:020000040000FA
:040000006FD00400B9
:101000006F1000140000000000000000902000207D
:10101000B2270020A9BDF9F56828002000000000D3
:101020000000000068280020902000200000000040
:101030000000000090200020000000009020002010
:101040000000000090200020902000209020002030
:101050009020002090200020B4300020902000201C
:10106000000000009020002090200020F4280020A4
:1010700090200020CE2800209020002090200020EA
:101080009020002090200020902000209020002020
:101090009020002001A04111B7170040985F3AC688
:1010A000945F3247E39CE6FE324541018280411164
:1010B000814601468145114506C6EF009014B727C9
:1010C000004011472383E780B7F700E003A707D16B
:1010D0006D9B23A8E7D003A707D15D9B23A8E7D08A
:1010E0007300501001000100B240410182800111E3
:1010F000814601468145114506CEEF009010B72785
:10110000004011472383E780B717004083C6E702FA
:1011100003C5E7041307800893F6C60F136535006F
:1011200093E61600733607801376860832C00100F6
:101130000100930570052380B704130680FA23800D
:10114000C70401000100238207022380070402482C
:10115000732808800100010073380780137888081D
:1011600042C2010001002380B7042380C7040100AC
:1011700001002387D7022387A70423800704924610
:10118000F3A6068001000100F336078093F6860877
:1011900036C4010001002380B7042380C704010086
:1011A000010083C6B70493E60602A385D704238013
:1011B0000704A246F3A6068001000100B7F600E08E
:1011C00003A506D11365450023A8A6D003A506D123
:1011D0005D9923A8A6D07300501001000100733759
:1011E0000780137787083AC6010001002380B704FF
:1011F0002380C7040100010003C7B7041377F70D6C
:10120000A385E70423800704B247F3A70780010002
:101210000100F240056182803971B7F5070022DCD8
:1012200081462A843010E105194506DE02D42316D2
:101230000102EF00007DB717004083C6E7041307E3
:10124000800893E63600733607801376860832C42A
:1012500001000100930570052380B704130680FA8E
:101260002380C704010001002382070223800704B2
:101270002245732505800100010073350780137531
:1012800085082AC6010001002380B7042380C70413
:10129000010001002387D70423800704B246F3A688
:1012A000068001000100F336078093F6860836C8F1
:1012B000010001002380B7042380C704010001005E
:1012C00003D50702F176FD16E98E2390D70223801D
:1012D0000704C246F3A606800100010037F500E0CE
:1012E000832605D193E646002328D5D083D607026E
:1012F0006575110593F60660C18EC98EC206C1825E
:1013000073350780137585082ACA01000100238000
:10131000B7042380C7040100010003C5F70013656B
:101320000504A387A7002390D70223800704D24691
:10133000F3A60680010001001165618D1DE9733778
:101340000780137787083ACC010001002380B70497
:101350002380C7040100010003C7B7041367070215
:10136000A385E70423800704E247F3A70780010071
:10137000010037F700E0832707D1DD9B2328F7D052
:10138000730050100100010013078008F337078035
:1013900093F787083ECE01000100B7170040930580
:1013A00070052380B704130680FA2380C704010068
:1013B000010083D60702C606C5822390D702238088
:1013C0000704F246F3A6068001000100F336078009
:1013D00093F6860836D0010001002380B7042380ED
:1013E000C7040100010003D80702F176FD16B3F629
:1013F00006012390D702238007048256F3A60680B5
:10140000010001000DED73370780137787083AD28A
:10141000010001002380B7042380C70401000100FC
:1014200003C7B7041377F70DA385E70423800704E8
:101430009257F3A70780010001005145ED2EF250AD
:10144000625421618280397152D481462A8A0146D0
:101450008145114522DC26DA06DE4AD84ED63714FD
:10146000004045238347E4020347E40493048008D3
:1014700093F7C70F1367370093E71700F3B604809D
:1014800093F6860836C60100010093097005230013
:101490003405130980FA230024050100010023020A
:1014A000040223000404B246F3A6068001000100F2
:1014B000F3B6048093F6860836C8010001002300C5
:1014C000340523002405010001002307F40223074B
:1014D000E40423000404C247F3A7078001000100CD
:1014E00013055002E128B7F700E003A707D11367FF
:1014F000470023A8E7D073B70480137787083ACA58
:10150000010001002300340523002405010001002F
:101510000347F40013670704A307E400230004044F
:101520005247732707800100010073B704801377C7
:1015300087083ACC0100010023003405230024056C
:10154000010001002167336AEA00231044032300ED
:1015500004046247732707800100010003A707D135
:101560005D9B23A8E7D07300501001000100814665
:101570000146814511457121F3B4048093F4840838
:1015800026CE0100010023003405230024050100BC
:1015900001008347640493E717002303F404230046
:1015A0000404F247F3A7078001000100F2506254DF
:1015B000D2544259B259225A216182800111130733
:1015C0008008F337078093F787083EC201000100C7
:1015D000B7170040930570052380B704130680FAFF
:1015E0002380C7040100010083C6B70493F6F60DFB
:1015F000A385D704238007049246F3A60680010042
:10160000010093760502D5CEF336078093F686085F
:1016100036C4010001002380B7042380C704010001
:101620000100B70614007D89558D88C701000100AF
:101630000100010023800704A246F3A606800100F2
:10164000010073370780137787083AC6010001004D
:101650002380B7042380C7040100010001000100BA
:101660003727004093061005A303D7802380070483
:10167000B247F3A707800100010093078008F3B782
:10168000078093F787083ECE01000100B71700409E
:10169000130770052380E704130780FA2380E7040B
:1016A0000100010003C7B70413670708A385E70417
:1016B00023800704F247F3A70780010001000561BA
:1016C000828093760504BDC6F336078093F68608BC
:1016D00036C8010001002380B7042380C70401003D
:1016E0000100B7061400938606047D89558D88C7CE
:1016F000010001000100010023800704C246F3A697
:1017000006800100010073370780137787083ACA03
:10171000010001002380B7042380C70401000100F9
:101720003727004093062005A303D78023800704B2
:10173000D24781B773370780137787083ACC010007
:1017400001002380B7042380C704010001009847EB
:101750001367070C98C723800704E24719BF0111DC
:10176000814601468145114506CE612C93078008CC
:10177000F3B7078093F787083EC601000100B7174B
:101780000040130770052380E704130780FA2380C5
:10179000E7040100010003C76704136717002383F0
:1017A000E70423800704B247F3A707800100010084
:1017B000F240056182804111814601468145114513
:1017C000892413078008F337078093F787083EC4FE
:1017D00001000100B7170040130670052380C704FD
:1017E000930680FA2380D70401000100FD5523965B
:1017F000B70223800704A245F3A50580010001007C
:1018000073370780137787083AC6010001002380E9
:10181000C7042380D7040100010003C767041367CE
:1018200017002383E70423800704B247F3A7078048
:101830000100010001A0BD473305F50201007D153F
:1018400075FD8280411122C426C206C6AA840144C5
:1018500063179400B24022449244410182800504FF
:101860001305803E4204C13F4180DDB7930500026D
:1018700073A0458082457390153492402242B24253
:101880004243D2436244F244025592552256B25624
:101890004257D2576258F25806499649264AB64AE4
:1018A000464BD64B664CF64C065D965D265EB65EA4
:1018B000465FD65F0961730020304111B7170040C1
:1018C000985F3AC6945F3247E39CE6FE3245410199
:1018D0008280B7170040130700032388E70285477B
:1018E00023A2F18673002030411122C406C63704BA
:1018F00000201C408297F5BF3737004083474700E0
:101900009146BD8B6389D70099466394D70083477E
:1019100057407300203083C6118993871600A3882F
:10192000F18803478700973700009387E7FBB69756
:101930002380E700B7E70400BC4F0946894503C58B
:1019400061828297F9B72303048015472303E4805B
:1019500001002302A480828083076480E3CE07FE17
:1019600023030480828083076480E3CE07FE03455F
:101970004480828083076480E3CE07FE2302A48034
:101980008280411126C44AC24EC006C61377F50BA9
:10199000AD47AA892E8995446306F7001945653736
:1019A000653F8D444E854537FD59FD1463983401DC
:1019B000B240A24412498249410182801355090173
:1019C0001375F50F453F2209CDB7011126CC06CE80
:1019D000B704080051371545BD37713769372AC636
:1019E000A53F32459377150089EB136515001375F4
:1019F000F50FF240E24405618280FD14E9FC0145E7
:101A0000CDBF397126DC4ADA4ED852D656D45AD2D6
:101A10005ED006DE62CE66CCB7E700E07D5783AAD3
:101A2000070022C603AA470023A0E71823A2E7184D
:101A3000B7170040130770052380E704130780FAE7
:101A40002380E70483C74704930B75FFB684E2073E
:101A500093FBFB0F8546AA892E8B328937240040E1
:101A6000E187015763FA76016308D50089461307B9
:101A700000026313D5000157D98F93F7F70FB71CF6
:101A800000402382FC0411472303E4801305F00F78
:101A90005D3D094CD135636D7C11B7050700DA95C2
:101AA00037870700795563F2E504B3879500636EC5
:101AB000F702370B0800A94733EB65016399F90674
:101AC00089E48144513D26850DA0DA850945553DBF
:101AD00005090345F9FFFD14050B693D81C49377A2
:101AE000FB0FFDF7DD3569FD7D55B7170040130786
:101AF00070052380E704130780FA2380E70403C7F7
:101B00004704418B2382E704F250B7E700E023A0AB
:101B1000571123A24711E25432445259C259325A42
:101B2000A25A125B825B724CE24C21618280A54713
:101B30006395F90685691309F00FB3069900B3742C
:101B40002B01B6941349F9FFB3749900856B33796F
:101B50006901416B9387F9FFB3F7270199E363FCB0
:101B6000340193D94900C147E3E637FF99BF0569BE
:101B7000C1697D19D9B71305800D63886901130503
:101B800000026384790113051008CA85DD3B353DE9
:101B900021DD4E99B3843441D9B7DA852D45D5334B
:101BA000CA94E30099F205097D3BA30FA9FED5BFB6
:101BB0009387F9FF93F7F70F6361FC0C83C71C044D
:101BC00013073008631FF70437070800636BEB0443
:101BD000B3079B00B706100063F5D704334BEB0047
:101BE00089476393F9068980D549E38C04ECDA854B
:101BF0000945413B11090327C9FF91472320E48090
:101C000003076480E34E07FE23033481FD17EDFBD9
:101C1000FD14110B81C49377FB0FE9FF7D3371F540
:101C2000E1B5B717004003C75704B707080013779B
:101C3000070219E3B78707007955E378FBEA330712
:101C40009B00E3FFE7F855B58547E382F9F2DA85B3
:101C50002D45053B9389F4FFE38504E6293393F78B
:101C6000390091EB8326048003270900930749007C
:101C7000E39AE6E43E89CE84F1BFB5476396F90066
:101C80001305900BC93135BDB1471305B00AE38B7D
:101C9000F9FE99476391F904B7050800B365BB00E5
:101CA0002D45C53181448D4BA14975396396740129
:101CB000832704802320F9008504E39834FF8327D9
:101CC000048013172B01635507002312F900D5BBBD
:101CD0002322F900FDB39D476399F902814513055D
:101CE000B0044531BD442320090023220900FD59D9
:101CF0009D3993F77400CA9703C70700FD14398D07
:101D00002380A700E39634FF6DBBA1476392F904DB
:101D10006D398144630D0B008D479304C003630844
:101D2000FB009304000563048B01930440041375C6
:101D3000C507E30895D819453931393905452131A9
:101D400026850D3909453D314931E31C05D669BB6E
:101D500091476399F90013056006F536F53E1305C2
:101D600090090DB7E38F09D4F154A9BBBD660147B3
:101D700017360000130606E4938606A685458347BA
:101D8000060093F7F70F91C382800507E3F9E6FE9B
:101D9000973700002380B7E2DDB77D1662066186C3
:101DA00093178601E18763D407000145828093176A
:101DB00026003307F500AE9718439C4363E7E7001E
:101DC0007D16E37FF7FC7D55828005458280FD15F9
:101DD000E205E18513978501618793F7F50F634865
:101DE0000700FD15139725002A97584365D71385DB
:101DF00017006205618582803308B5021C4283A802
:101E00000600B335B502C29733B50701AE984695C3
:101E100085486367B5006394A50063E307018148C3
:101E20000C43C6950CC388C21CC28280814713979D
:101E3000870161876343B7008280139727002A9741
:101E4000232007008507E5B781470147939687015F
:101E5000E18663C5B600133517008280939627008C
:101E6000AA9694428507558FD5B793D755408A07D0
:101E7000AA979C4305453315B5007D8D828017F3E5
:101E8000FFDFE702033B2A84993705C59317250036
:101E90003E940327C4FF814711EB7D1516053E953F
:101EA0004205418517F3FFDF6700E33A05838507A5
:101EB000E5B70145C5BF8147139787016187634334
:101EC000C700828013972700B386E50094422A97C3
:101ED000850714C3D5B77D1662066186014793173F
:101EE0008601E18763D507001335170082809317B9
:101EF0002600B306F500AE9794429C437D16B58F3D
:101F00005D8FF1BF8A05AA9501476363B5008280A2
:101F100083A6C5FFF11593D71600D98F9CC11397DF
:101F2000F601E5B72A830148014701456343D7001D
:101F30008280B387050183A80700B30706019C438D
:101F4000C697AA976384F80033B517010507B3084D
:101F50000301620723A0F80061871108C1BF2A832B
:101F600001478147014563C3D70082803388E5007C
:101F700083280800330EE600032E0E003388A840A5
:101F80003308C8416384080133B508018507B308E5
:101F9000E300E20723A00801E1871107E9B717F37F
:101FA000FFDFE70203290111B286B2842E86AA85DB
:101FB0000A8575372A84A6850A85793533348000E9
:101FC000060413351500018D056117F3FFDF670067
:101FD000832817F3FFDFE70243234111AA89AE8A62
:101FE000328BB68402C202C402C60144131C8401AF
:101FF000135C8C4163499C02939B1400FD1B0549B3
:10200000138CF4FFF15C3304890162046184634D35
:10201000740592478E04CE9423AEF4FE410117F36B
:10202000FFDF6700032213192400B30B2B01014AC1
:1020300093172A00D69783A50B00884378003400B5
:1020400050005D3B050A93178A01E187F11BE351BC
:10205000FCFE92474E9905042320F900A2473EC298
:10206000B24702C63EC459B7131A8901135A8A41AE
:10207000131D240093178A01E18763CF97009247CD
:102080000A044E941CC0A24705091379F90F3EC2F9
:10209000B24702C63EC485BFB3079A0313152A0090
:1020A00056950841780034005000050AEA97DA97FF
:1020B0008C439933C1B70000197106C212C416C609
:1020C0001AC81ECA22CC26CE2AD02ED232D436D658
:1020D0003AD83EDA42DC46DECAC0CEC2D2C4D6C648
:1020E000DAC8DECAE2CCE6CEEAD0EED2F2D4F6D638
:1020F000FAD8FEDA9385C1858841E7000500924051
:102100002242B2424243D2436244F24402559255C3
:102110002256B2564257D2576258F258064996494B
:10212000264AB64A464BD64B664CF64C065D965D43
:10213000265EB65E465FD65F096173002030000000
:1021400097210020938181E6174100201301816BC4
:1021500017F5FFFF130545EB97050020938585EAEA
:10216000171600201306C6FD63FAC500832205007A
:1021700023A0550011059105E3EAC5FE17A501004E
:102180001305C536971500209385C5FB138601847A
:1021900063FAC5008322050023A0550011059105AF
:1021A000E3EAC5FE1385018497450020938585ECFD
:1021B0006377B500232005001105E36DB5FEFD42F0
:1021C000739002BC8D4273904280B72200009382CC
:1021D000828873900230970200209382A2E293E2F9
:1021E000320073905230974200009382C2EA73909B
:1021F00012346FB0F46073002030397101436EC641
:1022000019A0397141536AC866CA62CC5ECE19A062
:10221000397101535AD056D252D44ED64AD826DA02
:1022200022DC06DE33016140828241114AC026C2AF
:1022300022C406C68282B24D4101024D924C224C0C
:10224000B24B4101024B924A224AB2494101024932
:1022500092442244B240410182803D432A87637305
:10226000C3029377F700BDEFADE5937606FF3D8A95
:10227000BA960CC34CC30CC74CC74107E36BD7FEDF
:1022800011E28280B306C3408A0697020000969648
:102290006780A6002307B700A306B7002306B70090
:1022A000A305B7002305B700A304B7002304B700B4
:1022B000A303B7002303B700A302B7002302B700AC
:1022C000A301B7002301B700A300B7002300B700A4
:1022D000828093F5F50F93968500D58D9396050131
:1022E000D58D61B793962700970200009696868257
:1022F000E78086FA9680C1171D8F3E96E374C3F877
:10230000A5B73367B500FD530D8B79E7B7877F7F9E
:102310009387F7F710419441B372F6003363F600E8
:10232000BE92B3E262006397720C6318D606504106
:10233000D441B372F6003363F600BE92B3E262009A
:102340006398720A631BD60410459445B372F60075
:102350003363F600BE92B3E262006391720A631EB9
:10236000D6025045D445B372F6003363F600BE92F0
:10237000B3E26200639A72086311D602104994496D
:10238000B372F6003363F600BE92B3E26200639369
:1023900072085105D105E30FD6F61317060193977E
:1023A0000601631CF7001357060193D70601330596
:1023B000F7409375F50F91E982804183C18333051E
:1023C000F7409375F50F91E182801377F70F93F73C
:1023D000F70F3305F74082800346050083C60500EA
:1023E000050585056313D60065FA3305D64082805E
:1023F00011059105E312D6FE014582802105A10554
:10240000E31CD6FC014582803105B105E316D6FCFC
:10241000014582804105C105E310D6FC014582805B
:10242000B717004003C777051377E70FA38BE704BF
:10243000130700F8A38DE7043D47238CE704130737
:102440005003A38CE70403C7A7051377D70F238D89
:10245000E7048280B717004003C7E7040D894111E4
:102460001377C70F498F93068008F3B6068093F65B
:10247000860836C601000100930670052380D70444
:10248000930680FA2380D704010001002387E70424
:1024900023800704B247F3A7078001000100410130
:1024A0008280B717004003C7E7020D8941111377F7
:1024B000C70F498F93068008F3B6068093F6860807
:1024C00036C601000100930670052380D7049306E9
:1024D00080FA2380D704010001002387E7022380CC
:1024E0000704B247F3A70780010001004101828081
:1024F00041112A83014E930E407E130F0019930F52
:10250000400663E56E129308001913034006B37882
:102510001503854E0D4FA14F337365020D89133599
:10252000150063EFBE121308F6FF79467298420851
:10253000135808013307C70213D61700BE07329796
:102540006146B3F6C60213068070B386C60236979C
:10255000A166F58F42075D8FB716004083C7F6026C
:1025600093F70708A303F1000346710083C7F6023F
:1025700093F70708E394C7FE83477100B71600403E
:1025800093F7F70F6388071293078008F3B7078064
:1025900093F787083EC401000100B7170040930677
:1025A00070052380D704930680FA2380D7040100A6
:1025B000010023AA070383C6170393E60608A3882E
:1025C000D70223800704A247F3A707800100010078
:1025D0001166B71700407D16D45BC85F938547032B
:1025E000A98EF18EF5FA93068008F3B6068093F66D
:1025F000860836C601000100930670052380D704C3
:10260000930680FA2380D7040100010098C103C714
:10261000170313670704A388E70223800704B24760
:10262000F3A7078001000100410182807D13336818
:10263000E3039308E016630E08003368F30393087E
:10264000D016630808009378330093B81800938875
:10265000D81633081E01131E0801135E0E0155B56E
:102660006393E5030548638608000148630303009C
:102670002A8871087298FD15131E0801C205135EA1
:102680000E01C18179BD13F8150063F4BF0079080C
:10269000D5B713381800E5BF83C7F60293F70708CC
:1026A000A303F1000346710083C7F60293F70708FE
:1026B000E394C7FE8347710093F7F70FF1DFE9B5A5
:1026C00031714AD966CB06DF22DD26DB4ED752D5E3
:1026D00056D35AD15ECF62CD6AC96EC7AA8C02D8D2
:1026E000EF00901C2A8993078008F3B7078093F7BF
:1026F00087083EDA01000100B71700401307700594
:102700002380E704130780FA2380E7040100010017
:1027100003C7F7021377770FA387E70203C7F70210
:1027200013678700A387E70223800704D257F3A724
:102730000780010001000545AD33130780C1334711
:10274000E902116A93070AE893065002BD69930BE8
:10275000A004814A014B13048008930470057D1A7C
:10276000B347F9023307D7023EC0FD873ECC9387BB
:1027700009A69309803E3347F7023AC27D873AC4DF
:10278000334739038549B399990193D93940B30641
:10279000D702B30B7703B3C6F602B3CBFB0236C640
:1027A000FD8636C893D6FB4136CEB7460F009386DA
:1027B00006243349D9028566938606FAB3969601B4
:1027C000B389E902130760553309D9029306001053
:1027D000B389E9023349D902B3C9F9029316390022
:1027E00036CA37190040FD8636D0930D090493D7B9
:1027F000F9413ED2F336048093F6860836DC0100B8
:102800000100930770052380FD00930680FA238062
:10281000DD00010001008346390593F6860FA30908
:10282000D9048346390593E61600A309D904238009
:102830000D00E256F3A6068001000100130C80FA99
:10284000116DF336048093F6860836DE0100010030
:10285000930770052380FD0023808D010100010096
:1028600083463905216693E60602A309D9048356F7
:102870000905B3E6A6012318D90483560905D18EAC
:102880002318D90423800D00F256F3A60680010018
:1028900001008346390593F60602638A061803464B
:1028A0003905218A6DDE0818EF00100473360480A4
:1028B00013768608B2C20100010023809D002380A8
:1028C0008D0101000100B717004003C637051376DC
:1028D000F60DA389C70403C6370513660602A3894C
:1028E000C704835609052166B3E6A6012318D90457
:1028F00083560905D18E2318D90423800D009646EE
:10290000F3A60680010001008346390593F606020E
:102910006386061483463905A18AEDFE97F0FF1FF2
:10292000E7806077AA8636D497F0FF1FE780A0760D
:10293000A256E30AD5FE835609054255B3E6A60121
:102940002318D904C12783463905A18AEDDE035631
:1029500009058346290582473376CA00B306DA02A1
:1029600093D5F641B296B388F640E24733B8C60035
:102970002E983308F840A247B3B616013308D84062
:1029800063C70701631DF800924763FA1701C24746
:10299000634DF80E63950701B24763E8F80E894668
:1029A00063E7660FF2469315180013D3F8015E86AD
:1029B00013951800B365B30042D646D4EF60E11B0F
:1029C0003258050B137BFB0F634700016312083875
:1029D000A258638F083613081500B336A800B695C1
:1029E00013D6F5013298B336C800AE9613581800C6
:1029F000FE06B3E606017336048013768608B2C677
:102A00000100010023809D0023808D010100010051
:102A10000356C902B296C206C1822316D902238088
:102A20000D00B646F3A606800100010019BDF3367D
:102A3000048093F68608B6C00100010023809D0043
:102A400023808D01010001008346390593E60602CB
:102A5000A309D90423800D00864605BDF336048002
:102A600093F68608B6C40100010023809D002380F0
:102A70008D01010001008346390593E60602A30992
:102A8000D90423800D00A646A5BDE30D0BF0F33657
:102A9000048093F68608B6C801000100930680FA08
:102AA00023809D002380DD0001000100834639055D
:102AB00093F5FC0F93F6860FA309D90483463905D5
:102AC000CD8EA309D90423800D00C646F3A6068047
:102AD00001000100130580FA034639059306390504
:102AE0001D8A631496297336048013768608B2CC47
:102AF00001000100130680FA23809D002380CD0091
:102B00000100010003C606001376F60D2380C600FF
:102B100003C60600136606022380C6008356090515
:102B20001166D18E2318D904835609052166D18EEA
:102B30002318D90423800D00E646F3A60680010081
:102B40000100130680FA8346390593F6060263886E
:102B5000062483463905130C3905A18AFDDA0818C5
:102B60006123F336048093F68608B6D00100010095
:102B7000930680FA23809D002380DD000100010080
:102B800083460C00116693F6F60D2300DC008346A5
:102B90000C0093E606022300DC0083560905D18E63
:102BA0002318D904835609052166D18E2318D90428
:102BB00023800D008656F3A606800100010013064F
:102BC00080FA8346390593F606026385062083461C
:102BD0003905A18AEDFE97F0FF1FE780C04B2A8CD4
:102BE00097F0FF1FE780204BE30C85FF8356090514
:102BF00011664255D18E2318D904292383463905FD
:102C000013063905A18AFDDAF336048093F68608A7
:102C1000B6D401000100930680FA23809D00238032
:102C2000DD00010001008346060093F6F60D230047
:102C3000D60023800D00A656F3A6068001000100F1
:102C40008356090503462905D247B376DA003306D1
:102C5000CA021305800C9355F6413696330DF640A3
:102C60008257333CD6002E9C3336A601330CFC40F1
:102C7000330CCC403308850392564E86B335A503FA
:102C80003305A503C295EF50516F63468001631E63
:102C90000C16630C0D16130615003335A6002E9581
:102CA0009356F5013696B335D600AA959396F5015D
:102CB00005828585D18E6346B000639D051A638BBE
:102CC000061A0356C90215823305D6003336C500ED
:102CD000B2956348B000639105241306F00F637D3D
:102CE000A622894663F3561593078008F3B7078039
:102CF00093F78708BED601000100371700409307FD
:102D000070052300F704930780FA2300F7040100FD
:102D100001008356C70289678117D58FC207C18317
:102D20002316F70223000704B657F3A70780010014
:102D30000100FA506A54DA544A59BA592A5A9A5A2E
:102D40000A5BFA4B6A4CDA4C4A4DBA4D29618280D3
:102D50001308F5FF3335A800FD152E951356F50120
:102D60003298B336C800AA9651B1F336048093F670
:102D70008608B6CA0100010023809D002380AD00B3
:102D80000100010083463905CD8EA309D9042380B3
:102D90000D00D646F3A606800100010035BBF336D0
:102DA000048093F68608B6CE0100010023809D00C2
:102DB0002380CD00010001008346390593E6060219
:102DC000A309D90423800D00F646F3A6068001006E
:102DD000010095BBF336048093F68608B6D2010055
:102DE000010023809D002380CD0001000100834667
:102DF000390593E60602A309D90423800D009656EF
:102E0000F3A60680010001006DBB9306F5FF33B504
:102E1000A600FD152E959355F501AE96B3B5B600F7
:102E2000AA951396F501858269B5F336048093F669
:102E30008608B6D801000100930680FA23809D0021
:102E40002380DD00010001008356C90205660116DA
:102E500093F6F60FD18EC206C1822316D9022380C3
:102E60000D00C656F3A6068001000100850A93FAFC
:102E7000FA0F49B233E6B60045C20356C90233051C
:102E8000D0403338A000B305B040B385054115826A
:102E90006345B000D1E16371A608894663F0560529
:102EA00093078008F3B7078093F78708BEDA01001D
:102EB0000100B7170040130770052380E7041307CC
:102EC00080FA2380E7040100010003D7C7027D8B4D
:102ED0002396E70223800704D65781BDF33604808A
:102EE00093F68608B6DC01000100930680FA238081
:102EF0009D002380DD00010001008356C9020566A4
:102F0000011693F6F60FD18EC206C1822316D9029E
:102F100023800D00E656B9B793078008F3B7078002
:102F200093F78708BEDE01000100371700409307C2
:102F300070052300F704930780FA2300F7040100CB
:102F400001000356C70293975600B297C207C18388
:102F50002316F70223000704F657C1BB914763EE1F
:102F6000B702178701001307278F8A05BA959C417E
:102F7000BA978287B717004003A7470B1345F5FFA1
:102F8000698F23AAE70A03A7070B698F23A8E70A1B
:102F900003A7070A798D23A0A70A8280B7170040EC
:102FA00083A6470B1347F5FFF98E23AAD70A83A6FA
:102FB000070B558D23A8A70A83A6070A758F23A0A0
:102FC000E70A8280B717004003A7470B498F23AA5F
:102FD000E70A03A7070B1345F5FF45BFB7170040E6
:102FE00083A6470B1347F5FF758F23AAE70A03A7AC
:102FF000070A598D4DB7B717004003A7470B498FF4
:10300000EDB7914763EEB7021787010013070786F4
:103010008A05BA959C41BA978287B717004003A7E3
:10302000470D1345F5FF698F23AAE70C03A7070D8A
:10303000698F23A8E70C03A7070C798D23A0A70CA1
:103040008280B717004083A6470D1347F5FFF98E1E
:1030500023AAD70C83A6070D558D23A8A70C83A6FA
:10306000070C758F23A0E70C8280B717004003A7D9
:10307000470D498F23AAE70C03A7070D1345F5FF5A
:1030800045BFB717004083A6470D1347F5FF758F5F
:1030900023AAE70C03A7070C598D4DB7B7170040BB
:1030A00003A7470D498FEDB7B71700408847420582
:1030B00041819377050491EB9377F5013755E8014A
:1030C000130505803345F50282809377050C1307BD
:1030D00000046397E7009377F50137459C1CCDB753
:1030E0002165130505D0828037E700E01C43544377
:1030F000A183E206D58F1CC1FD572320F718232298
:10310000F718828013178500B7E700E023A0E710C7
:10311000618123A2A7108280B7F700E08847CC47DF
:103120008280814737370040A14663C4C70032859B
:1031300082800345B740E38EA6FE3385F500034544
:10314000050085072304A740CDB797070020938784
:10315000E7659C43173700201307C7F13E95636E60
:10316000E500173700201307E7496368A700170732
:103170000020232DA7623E858280FD57EDBF4111BF
:1031800022C406C62A840D372947B307E502B24098
:103190008D83B3D7870222449507B3D7E702373729
:1031A0000040C207C1832316F70041018280716588
:1031B00041111305052006C6D937B737004013075C
:1031C00070F82381E7000D47A381E700130700048F
:1031D000A380E70005472387E700B24041018280D2
:1031E00037370040834727001A0593F7F703C98F45
:1031F00093F7F70F2301F7008280B737004003C72A
:10320000170019C9D98DA380B70003C7070013673A
:1032100087002380E700828093C5F5FFF98DA380A6
:10322000B7008280B73700402147B736004091E1B0
:10323000828003C6B700E30CC7FE05050346F5FF11
:10324000FD15C2052384C600C181D5B7411122C432
:1032500006C62A84913D2947B307E502B2408D8313
:10326000B3D7870222449507B3D7E7023737004028
:10327000C207C1832316F740410182807165411165
:103280001305052006C6D937B7370040130770F875
:103290002381E7400D47A381E74013070004A38083
:1032A000E74005472387E740B24041018280CC4197
:1032B000411106C6328503C6150083C505002206E6
:1032C0004D8E42068D654186138875A263080611EE
:1032D000634BC804138845A2630C060B634AC800FD
:1032E000938535A2630FB60623900600294669A888
:1032F000138855A26301060D938565A2E316B6FEF9
:103300008D451D4663E2E5081146198E63F3C7003B
:103310003E86B7E704002390C600FC47979501005E
:103320009385C516B9A8138895A2630F060F634A43
:10333000060D1388A5A2630C0611938505A5E31558
:10334000B6FA99451D4663E1E504198E63F3C7009B
:103350003E86B7E704002390C600FC479385818032
:103360000DA09D451D4663E1E5022146198E63F3DC
:10337000C7003E86B7E70400FC472390C60093854C
:103380000184BA9582970146B2403285410182801C
:10339000AD451D46E3EAE5FE3146198E63F3C700ED
:1033A0003E86B7E704002390C600FC4797750100EE
:1033B0009385C54EF9B7B1451D46E3E7E5FC3546B3
:1033C000198E63F3C7003E86B7E704002390C6005A
:1033D000FC47977501009385654D65B78D451D4682
:1033E000E3E4E5FA1146198E63F3C7003E86B7E7BA
:1033F00004002390C600FC47979501009385C509FA
:1034000049B78D451D46E3E1E5F81146198E63F392
:10341000C7003E86B7E704002390C600FC47979597
:10342000010093852509B1BFA5451D46E3EEE5F4EE
:103430002946198E63F3C7003E86B7E70400239040
:10344000C600FC4797750100938585441DBFB545AF
:103450001D46E3EBE5F23946198E63F3C7003E865D
:10346000B7E704002390C600FC47977501009385D9
:10347000254101BFB7E7040003A307139706002007
:10348000938646D54146A54517050020130585CBF3
:1034900002832D4559EF03C5050009476317E50869
:1034A00003A84500411106C60347180032850346AC
:1034B000080022074168518F930828FE630817030C
:1034C00063E9E80005186303070523900600294512
:1034D0001DA8130648FE630BC7021518E31707FF64
:1034E00015463E87637BF602154705A83E8691C3C5
:1034F0000546B7E70400FC472390C6004206CC45CA
:10350000418282970145B240410182801306700FCB
:103510003E876374F6001307700FB7E7040023902B
:10352000E600FC4713160701D9BF239006000545A6
:1035300082808280416779176302E504411122C4C9
:1035400006C685472A84639DF500B7E704002285F7
:103550002244B24003A387139385C18441010283AF
:1035600089476399F500B7E7040083A7070B8545F2
:10357000829761DDB240224441018280828079716C
:1035800022D452CC2E842A8A977501009385453423
:10359000177501001305853506D63AC626D24AD0DE
:1035A000B68432894ECEEF509128A685177501005A
:1035B0001305C534EF50B1272945EF50512B8347F0
:1035C000840093F70702F1E3834904008947054526
:1035D00032476394F908544083C7160083C6060037
:1035E000A207D58FC166138616FE638CC7028D169F
:1035F000638DD7068D66938626902945639FD704F1
:10360000B7E70400A285225403A34714B250F2493D
:10361000A6864A86925402595285624A8547456178
:1036200002832D451DEB9307700F354563E7970225
:10363000B7E70400FC4748441306700FCA85829719
:103640008149938781859C43014581CB9C4391C7E8
:103650004E852686CA8582970145B25022549254DF
:103660000259F249624A456182802D457DF79307F0
:10367000700F3545E3E397FEB7E70400FC47484485
:103680001306700FCA8582976DBF2145F9B74111A6
:1036900022C437E404008327841326C2AA84416528
:1036A00006C69385C1847D1582978327C40A1705B2
:1036B0000000130565E88588829795C003230413ED
:1036C0002244B240924497060020938666C2414647
:1036D000C545170500201305A5B041010283B2407E
:1036E0002244924401454101828009C523ACA18452
:1036F000014582804545828011476360A70A97761D
:1037000001009386A61B0A0536951841411106C68D
:103710003697AE87B28502871307700F6145639BAA
:10372000E700B7E70400FC471306700F1385C18B51
:1037300082970145B2404101828005476145E39B84
:10374000E7FEB7E70400FC47054613858184CDB743
:103750001307700F6145E39FE7FCB7E70400FC47E0
:103760001306700F1385419BE1B71307700F614576
:10377000E392E7FCB7E70400FC471306700F1385DC
:10378000C1AA7DB715476145E396E7FAB7E704009C
:10379000FC4715461385018561BF094582804111AB
:1037A00026C2B7E4040083A7C41322C44AC006C6D5
:1037B0002E849385C1842A898297058905C5970738
:1037C00000209387E7A183D7A70BA28503A3440D0D
:1037D0002310F4002244B24092444A850249014633
:1037E00041010283B24022449244024949454101C9
:1037F000828011456FE0DFEC411193962500AA8588
:103800002D4506C697F0FF1FE780A01FB240014577
:1038100041018280011122CC06CE3714004026CA15
:103820004AC84EC652C483447405034AB40583494A
:10383000840503499405EFE0BFBE8347A40593F4D4
:10384000F40F137AFA0F93E71700230DF40493F99A
:10385000F90F1379F90FB717004003C7A705058BB8
:103860006DFF03D5C705A38D4705238C3705A38CB2
:103870002705A38B9704F2406244D2444249B249DF
:10388000224A0561828041119397050122C406C630
:1038900026C2C1872E8463D00702B7E40400FC541B
:1038A000829719C1BC5482972165218DB240224470
:1038B00092444101828093F7150013C51500FDF76E
:1038C0009397250163D30702B7E4040083A7C41EBE
:1038D00082970537BC4C37F60200130606E089656F
:1038E00003C5018682970965C9B7939715010145FC
:1038F000E3DE07FA1775010013050507EF5071079E
:10390000B7E70400BC4F13060064916503C5018648
:103910008297116559BF2D71232A9110FD74E98C8E
:10392000232C811023282111232631112A84AE89CA
:103930003289930600100A86A6852D45232E111084
:1039400097F0FF1FE780E00B13154401B7E7040071
:10395000FC4751810A0513962900CA850A9582976A
:10396000A68585660146254597F0FF1FE78060091B
:103970000A86A68593060010294597F0FF1FE78069
:1039800040088320C111032481118324411103299C
:1039900001118329C11015618280B7F7070003C7A1
:1039A0000701411106C622C426C24AC0A547631AB0
:1039B000F7009537B2402244924402490145410143
:1039C000828013942500AA843289A286AA850146A2
:1039D000254597F0FF1FE780C002A2864A86A6858C
:1039E000294597F0FF1FE780C001E9B71D71A6CAFE
:1039F000B7E40400DC5CC85886CEA2CC4946977573
:103A000001009385E5F1829701E91775010013051F
:103A100065F2EF50017601A037F700E0795610CB40
:103A2000FD5654CBB7E700E0056423A0871093064A
:103A3000F00214C323A087180100010037070020FB
:103A4000184713060004814523AEE1844157A38A39
:103A5000E740BC440808829797170020938787E8BF
:103A60003EC89D673ECCB7070105938707103ECE41
:103A70009307B00F2310F10285472301F102970746
:103A800000009387A7D7BEC297070000938727F14E
:103A9000BEC485679387B7D32312F10297F7FFFF60
:103AA0009387C7673ED8970700009387E7D63EDC29
:103AB000B7F50700970700009387E7D33EDE8146FE
:103AC000970700009387E71B3000E10519453EDAB0
:103AD000231A810097F0FF1FE780A0F218088147A2
:103AE000994630003E960346060085070507A30B5E
:103AF000C700E398D7FEC24791C7035741018567C6
:103B00006373F70001A0B7E7040083A7470A08081A
:103B10008297AA8501C9177501001305E5E2EF50E8
:103B2000015101A0F6406644D644256182804111CE
:103B300026C2B7E4040083A7040806C622C41705FA
:103B40000000130585D48297138401862300A40006
:103B50008520E12A03450400224403A38405B240E2
:103B60009244130600328965410102834111930793
:103B70008008F3B7078093F787083EC6010001006D
:103B8000B7170040130770052380E704130780FA76
:103B90002380E70401000100C8DB23800704B2474B
:103BA000F3A707800100010023A201864101828062
:103BB000797106D622D413078008F337078093F76C
:103BC00087083EC201000100B71700409305700549
:103BD0002380B704130680FA2380C7040100010084
:103BE00083C6F70293F6A60FA387D70223800704A4
:103BF0009246F3A606800100010073370780137711
:103C000087083AC4010001002380B7042380C70459
:103C10000100010003C7F70213672700A387E7022B
:103C200023800704A247F3A7078001000100054590
:103C3000EFE03F877D3E0147814681470546854548
:103C40001305407EEFE0DF8A37E404003C4468005F
:103C5000514681458297B707C0A83EC8B787E80399
:103C6000938707D03ECA97F7FF1F938707C53EC6C5
:103C70007C5868008297B2502254456182800111BD
:103C800022CC06CE930730031304D5FC63E7A700CC
:103C90003704C0A81304D4FC2A946800EFF0CFC402
:103CA00097E0FF1FE780203FB307A4406376A4009E
:103CB000B707C0A8A297898F3747F6A681171307C1
:103CC00007C6637AF7003245EFF0CFC30945F240EB
:103CD0006244056182802285513D3245EFF08FC2FA
:103CE000373700408347574093F707048DCF9387BA
:103CF00041869C430D45E1FF1165690597E0FF1F73
:103D0000E78080510545EFE0EFF497E0FF1FE78083
:103D100080382AC497E0FF1FE780E037A247E30B13
:103D2000F5FE01456DB7010075BF4111130780080D
:103D3000F337078093F787083EC401000100B717E7
:103D40000040930570052380B704130680FA238092
:103D5000C7040100010083C6E70093E686002387BD
:103D6000D70023800704A246F3A6068001000100C5
:103D700073370780137787083AC601000100238054
:103D8000B7042380C7040100010003C717031367AA
:103D90000702A388E70223800704B247F3A707803E
:103DA00001000100B7E700E03707001023A0E7108B
:103DB000410182804111977501009385A52A1775ED
:103DC00001001305A5B206C6EF5061261775010064
:103DD0001305C543EF50A125B240294541016F505D
:103DE0000129411197750100938505291775010077
:103DF0001305C5AF06C6EF508123177501001305E3
:103E0000A53FEF50C122B240294541016F50212604
:103E1000411122C406C6834705002A849DC39775B5
:103E200001009385252B17750100130525ACEF5074
:103E300001204C401775010013058551EF50211FDB
:103E40001DA058411DE7977501009385A52817759A
:103E500001001305A5A9EF50811D17750100130579
:103E6000A550EF50C11C2244B240294541016F507A
:103E70000120A1679386D7036311D70297750100CC
:103E80009385452517750100130545A6EF50211AA6
:103E9000177501001305454EE9B7ED079775010049
:103EA0009385452317750100130545A46319F70091
:103EB000EF50E117177501001305454D5DB7EF5041
:103EC00001174C40177501001305454E85BF411180
:103ED000977501009385851B17750100130505A1D2
:103EE00006C6EF50C114B240294541016F50211858
:103EF000797122D426D24AD02E842A898145B2846F
:103F00004800714606D6EFE04FB597F7FF1F93873D
:103F1000A75DDC4783D70700231421012313F10099
:103F2000EF20206C9547A305F1009307401F3EC684
:103F3000FD572305A100230AF100EF20007C26860F
:103F4000A2854800EF20406CB2502254925402598E
:103F5000456182802399018823880188B7E704009E
:103F6000BC47411106C6414681451715002013057F
:103F7000A5958297EF109055EF1050340145EF2032
:103F8000507403C7417A9307F00A631BF700930745
:103F9000F00889451385417A2392F17AEF30401D6C
:103FA000EF30A02C81453705040023A4018823921B
:103FB000018823830188239F0186239E0186239104
:103FC000018823960188EF2000250145EF308020ED
:103FD000977501009385050E17750100130505916E
:103FE000EF50E1041775010013058542EF502104DD
:103FF000B240294541016F508107411122C406C6D4
:1040000026C293F715002E846389070C814617F6A4
:10401000FF1F1306E64A854503D58187EF80E068D8
:1040200005C5977501009385A5091775010013054E
:10403000E58BEF40D17F17750100130525ABEF40ED
:10404000117F2945EF50A10297750100938545071F
:104050001775010013058589EF40717D1775010003
:10406000130505AAEF40B17C2945EF50410017F533
:10407000FF1F130565475C4505472390E700EFE008
:104080003079977501009385A50317750100130515
:10409000E585EF40D179177501001305A5A7EF401D
:1040A00011792945EF40B17C930710F82382F17A0A
:1040B00083D74187A382F17A1385417AA183914501
:1040C0002383F17AA383017AEF30800A1345140029
:1040D000B240224492444101828093F72500D1C32B
:1040E00003D7418825CF9386818894429777010032
:1040F0009387073403C6618881451705002013059F
:10410000A57CEF40C067AA8431C9977501009385EB
:10411000E501176501001305657DEF405171A68526
:1041200017750100130585A0EF4071702945EF4018
:10413000117423920188930710F82382F17A83D7B0
:104140004187A382F17AA1832383F17A91458D4738
:104150001385417AA383F17AEF308001134524005F
:1041600085BF93F74500A1CF97750100938505FCA6
:104170001765010013058577EF40716B1775010016
:104180001305859CEF40B16A2945EF40516E9307B6
:1041900020F82382F17A83D7E187A382F17AA18381
:1041A0002383F17A8547A383F17AEF2000551385A5
:1041B000417A9145EF20D07B1345440011BF93F71E
:1041C00085009DCB97750100938545F61765010025
:1041D0001305C571EF40B16517750100130505980A
:1041E000EF40F1642945EF40916823920188EF4048
:1041F000E06513458400E9BD93F70501A1CF85452E
:1042000003D5E187EF00F12F97750100938505F243
:10421000176501001305856DEF4071611775010089
:1042200013050595EF40B1602945EF4051649307B0
:1042300030F82382F17A83D7E187A382F17A13855C
:10424000417AA1838D452383F17AEF207072134563
:104250000401BDBD93F70502B1CF977501009385A9
:10426000E5EC1765010013056568EF40515C1775B3
:10427000010013052592EF40915B2945EF40315F26
:10428000930740F82382F17A83D7C187A382F17A1A
:10429000A1832383F17A8547A383F17A239E018644
:1042A000EF20A0451385417A9145EF20706C1345AE
:1042B000040239BD93F70504D9CF977501009385A2
:1042C000E5E61765010013056562EF405156177565
:1042D00001001305A58DEF4091552945EF40315957
:1042E00083C7417A1307700A6384E7041307800ABF
:1042F0006380E7061307600A6395E702930760F897
:104300002382F17A83D72188A382F17AA183238340
:10431000F17A8547A387F17AB1451385417AEF2079
:104320003065EF20803D13450404239101884DB38F
:10433000930770F82382F17A83D72188A382F17AD8
:10434000A1832383F17A8547A384F17A9945F1B754
:10435000930780F8C5B793F705080145E38A07D6A8
:1043600097750100938585DC1765010013050558D5
:10437000EF40F14B177501001305C584EF40314B39
:104380002945EF40D14E9307A0F82382F17A83D7D5
:10439000C188A382F17AA1832383F17A8547A3831D
:1043A000F17A23960188EF2040351385417A9145B3
:1043B000EF20105C1345040821BB411122C49775FE
:1043C0000100938565D22A84176501001305055203
:1043D00006C6EF40D1454C40177501001305C5F4E2
:1043E000EF40F1442945EF4091480347040093070B
:1043F000F00F6319F702977501009385E5CE1765F5
:1044000001001305A54EEF4091424C401775010085
:10441000130585F2EF40B1412244B24029454101E4
:104420006F40F144B24022444101828085CD411168
:1044300022C4176501001305654B2E849775010092
:10444000938585C506C6EF40913EA285177501008C
:104450001305C5F9EF40B13D2244B2402945410161
:104460006F40F1408280411122C426C22E84AA846A
:1044700097750100938505C317650100130505476E
:1044800006C6EF40D13A177501001305E5F6EF4077
:10449000113A2945EF40B13D97750100938585C0DC
:1044A000239C918617650100130545448544239A92
:1044B0008186239B918623998188EF40513783D54C
:1044C0002189177501001305A5F3EF4051362945E1
:1044D000EF40F13923889188EF10405E2285EF206C
:1044E000501E0545EF20104F97F7FF1F9387C7FF1A
:1044F000DC4703D70700C167FD176310F7022244AA
:10450000B7E70400B240924403A3870503C5818640
:104510001306000A854541010283B24022449244B9
:1045200041018280011122CC37E404005C5C06CE9C
:1045300026CA354697750100938585CE177501000B
:104540001305C55A829701E9176501001305853ED9
:10455000EF40314201A097F7FF1F9387675F3EC48A
:10456000B7F507008567938707C081461386C18624
:10457000E10519453EC697E0FF1FE78080487C446F
:1045800019469385C186170500201305252D8297AE
:1045900034001386C186977501009385E51217755F
:1045A00001001305E513EF301076AA8415C997753D
:1045B00001009385A5B61765010013052533EF406B
:1045C0001127A68517750100130585C6EF40312612
:1045D0002945EF40D129F2406244D24405618280EE
:1045E000EFA0E00C17750100130585BBEF304011FB
:1045F000EF60307BEF00B11917F5FF1F130585EB56
:10460000EF00910617750100130585BAEF00F11947
:10461000AA84EF30E06BEFC0003FEF205139EF404C
:104620001008EF30304BEFE0F01B977501009385D9
:10463000E5AE176501001305652B89C8EF40311FF2
:10464000A685177501001305E5C049B7EF40311E77
:1046500017750100130545C2EF40711D2945EF4054
:104660001121EFE0807EEFB0C028630D050C854579
:1046700037050400EF10303A97750100938505AABD
:104680001765010013058526EF40711A17750100A3
:10469000130505C0EF40B1192945EF40511D97F7AB
:1046A000FF1F9387A7D483D707002399F1888547F5
:1046B0002388F188EF10405CEF10404003D521893A
:1046C000EF20300083C7F188B9EFA30301008327EF
:1046D000441713067100854513055030829797756E
:1046E00001009385A5A31765010013052520EF4060
:1046F0001114177501001305E5BBEF40511329454F
:10470000EF40F11697750100938545A117650100EB
:104710001305C51DEF40B11117750100130585BFC5
:10472000EF40F11075B5977501009385259F1765CA
:1047300001001305A51BEF40910F1775010013052C
:10474000E5BA65BF977501009385459D1765010022
:104750001305C519EF40B10D17750100130545CBC1
:10476000EF40F10C2945EF4091100145EF209026D4
:1047700051BF411122C437E404008327041A06C63E
:104780008297EF20C07C83270408170500001305DB
:10479000058782972384A18617F5FF1F1305C5D4CB
:1047A000EF2000212244B2404101ADBB411122C49F
:1047B00091462A84170600201306C6079D652D45DD
:1047C00006C697E0FF1FE780C023B7F7070003C7BF
:1047D0000701A5476313F70001A0930600100146E7
:1047E0009D65254597E0FF1FE780A02197070020E2
:1047F000238287042244B240914617060020130604
:1048000066039D652945410117E3FF1F6700631F8C
:10481000B7E704001171FC47CED79389417AA2DD36
:10482000CAD986DFA6DB2E8432892E86AA854E85DC
:10483000829783C70900130780029387E70793F7DE
:10484000F70F636CF77217670100130727128A07C7
:10485000BA979C43BA9782878D47977501009385D5
:10486000258E1765010013056508630BF400EF4002
:10487000017C176501001305654BEF40417BCDA21C
:10488000EF40E17A176501001305C54BEF40217A2F
:104890002945EF40C17D930720F811469385417A61
:1048A0004A852382F17AA383017AEFF06FE42A84A8
:1048B0000DC5977501009385A5881765010013053F
:1048C000E502EF40C176A285176501001305454B4F
:1048D000EF40E1752945EF40817997750100938597
:1048E00025861765010013056500EF4041741765C3
:1048F00001001305254AEF4081732945EF402177D8
:104900004165930730FA05469385417A7D152382E8
:10491000F17AEFF0EFDD2A840DC5977501009385DC
:10492000258217650100130565FCEF404170A285E3
:10493000176501001305C544EF40616F2945EF403D
:104940000173B7E70400BC4F0566130606C8A1450E
:1049500003C581868297FE506E54DE544E59BE596F
:104960001161828091476301F4029765010093858C
:10497000257D17650100130565F7EF40416B17654D
:10498000010013056544D5BDB7E70400FC4F914510
:1049900003C581868297976501009385657A1765BF
:1049A00001001305A5F4EF408168176501001305A8
:1049B0006543EF40C1672945EF40616BEF10F0534D
:1049C0009145C1A285476301F40297650100938573
:1049D000257717650100130565F1EF4041651765FF
:1049E00001001305A54151BD239F2187B7E70400AE
:1049F0000566BC4F130606C8C14599BF8D476301C4
:104A0000F402976501009385A573176501001305EE
:104A1000E5EDEF40C161176501001305E53FB1BD4C
:104A2000930740F811469385417A4A852382F17AAB
:104A3000A383017AEFF0CFCB2A84E30E05F09765CC
:104A400001009385E56F17650100130525EAEF4026
:104A5000015EA2851765010013058532EF40215DD7
:104A60002945EF40C160C5BD9147E31CF4F8B7E7A5
:104A70000400FC4F9305000203C581868297976569
:104A800001009385E56B17650100130525E6EF40EE
:104A9000015A176501001305A53921BF894763E154
:104AA0008702976501009385A569176501001305C5
:104AB000E5E3EF40C157176501001305A53875BB45
:104AC00083C4617A83C7517A9765010093854567EE
:104AD000A20417650100130565E1DD8CEF40215547
:104AE000A2851765010013052537EF404154C20424
:104AF0002945EF40C157C1849305D4FF9396040123
:104B0000C1824A8693F5F50F1385717AEF102074F0
:104B1000E35390E4930750F82382F17A83C7390076
:104B200022869385417A85074A85A383F17AEFF03F
:104B30002FBC2A84E30105E2976501009385456057
:104B400017650100130585DAEF40614EA2851775E0
:104B500001001305A58819B7894763E187029765A6
:104B600001009385E55D17650100130525D8EF4029
:104B7000014C176501001305E52F01B3EF10F03765
:104B8000A2851385417AEF20A05EF1B38D476301C2
:104B9000F402976501009385A55A17650100130576
:104BA000E5D4EF40C148176501001305652EF1B14A
:104BB000B76602000146B7750200054597E0FF1F82
:104BC000E78020E4930760F82382F17AA383017AD7
:104BD0009307002623A4F17AE5779387072123968C
:104BE000F17A3146A387A17A9385417A4A85238752
:104BF000017AEFF0EFAF2A84E30F05D49765010047
:104C00009385055417650100130545CEEF402142F9
:104C1000A285176501001305252989B5B1476301F0
:104C2000F402976501009385A551176501001305EE
:104C3000E5CBEF40C13F176501001305A52835B945
:104C4000B7E70400FC4F9305000403C581868297F3
:104C5000EF10B02AB14535B7914763E187029765F8
:104C600001009385E54D17650100130525C8EF4048
:104C7000013C176501001305A52601B183C4817AA3
:104C800083C7717AA204DD8C8E04B77702006D149D
:104C9000BE942286A685176501001305A525EF4061
:104CA0000139B7E70400FC4722869385917A2800F2
:104CB000829793160401C1823000A685094597E0CA
:104CC000FF1FE78000D42A8419C51765010013056A
:104CD0002524EF40014A930770F819469385417ADD
:104CE0004A852382F17AA384817AEFF06FA02A8427
:104CF000E30305C6976501009385854417650100A8
:104D00001305C5BEEF40A132A2851765010013054A
:104D10002521A9B399476301F41097650100938594
:104D2000254217650100130565BCEF40413017654A
:104D300001001305652091B6914763E187029765ED
:104D400001009385E53F17650100130525BAEF4083
:104D5000012E176501001305A51F05B683C4817ACE
:104D600083C7717AA204DD8C8E04B77702006D14BC
:104D7000BE942286A685176501001305A51EEF4087
:104D8000012BB7E70400FC4722869385917A28001F
:104D9000829793160401C1823000A6850D4597E0E5
:104DA000FF1FE78000C62A8419C517650100130597
:104DB000251DEF40013C930780F819469385417A01
:104DC0004A852382F17AA384817AEFF06F922A8454
:104DD000E30305B8976501009385853617650100E3
:104DE0001305C5B0EF40A124A28517650100130586
:104DF000651AADB199476301F40297650100938587
:104E0000253417650100130565AEEF404122176593
:104E100001001305A51995B4B7E70400FC4F9305ED
:104E2000000403C581868297EF10300D994591BB30
:104E30008D476301F402976501009385653017651E
:104E400001001305A5AAEF40811E17650100130597
:104E5000651725B4176501001305C517EF406131CB
:104E60001305C01297E0FF1FE780C09D0145EFE0EA
:104E7000AFA70D45EFF09F93294597E0FF1FE7800F
:104E8000609C97E0FF1FE780808DF1B49947630134
:104E9000F402976501009385A52A176501001305A3
:104EA000E5A4EF40C1181765010013056513F1B2C1
:104EB00003C7917A83C7817A22075D8F9166BA967C
:104EC000C2061166C1821306F6EF8D476363D602F0
:104ED00097E7FF1F938747619C4B03C6717A9386C0
:104EE000C70039C603D607004DCA8907E39CD7FE21
:104EF00089471307A0F811469385417A4A85238292
:104F0000E17AA383F17AEFE0BFFE2A84E30505A4EA
:104F1000976501009385C522176501001305059D5E
:104F2000EF40E110A285176501001305A50C3DB601
:104F300003D607006300E60A8907E39BF6FE8D4768
:104F40004DBF91476302F402976501009385451FA9
:104F50001765010013058599EF40610D1765010084
:104F60001305C50A6FF07F91B7E70400FC4F930566
:104F7000000803C58186829791B4976501009385E7
:104F8000251C1765010013056596EF40410A17655A
:104F90000100130525096FF05F8E2390E70017E5E8
:104FA000FF1F13056554EFE04008976501009385E6
:104FB00025191765010013056593EF404107176533
:104FC000010013052507EF4081062945EF40210A1E
:104FD000814705B72390070017E5FF1F1305C5504C
:104FE000EFE0A00497650100938585151765010022
:104FF0001305C58FEF40A1031765010013050505D3
:10500000D9B7411122C406C6834705002A849DC32F
:10501000976501009385850E176501001305058DC1
:10502000EF40E1004C401765010013056541EF407A
:10503000010065A05841B707CF009387777D6311C2
:10504000F706976501009385650B17650100130549
:10505000E589EF30D17D1C448356E4008355C400BC
:1050600003C60700176501001305053FEF30317CCB
:105070002945EF30D17F0357E40083D721896307A7
:10508000F7008355C4000844EFE0CF990356E400CD
:105090008355C40008442244B24041016FF04FF7E9
:1050A000B707CC009387777D631FF70297650100F0
:1050B0009385C5041765010013054583EF303177EB
:1050C0001C448356E4008355C40003C607001765DB
:1050D000010013056538EF3091752244B24029452F
:1050E00041016F30D178B707CE009387777D630297
:1050F000F7029765010093856500175501001305B8
:10510000E57EEF30D1724C40176501001305052A8A
:1051100039BFB2402244410182805171CAD137E97E
:1051200004008327C904A2D52E8686D7A6D32E8451
:10513000AA851385417A829783C7417A1307700A3B
:10514000638BE70C636CF7001307600A6382E70464
:10515000BE502E549E540E596D6182801307800AF2
:105160006380E7121307900AE394E7FE8D47630913
:10517000F41697650100938565FE17550100130528
:10518000E576EF30D16A176501001305659315A028
:105190008D476306F40297650100938525FC17553A
:1051A00001001305A574EF30916817650100130520
:1051B000658AEF30D1672945EF30716B51BF854764
:1051C000176501001305C58A2380F188EF30717AD5
:1051D000B7750200B76602000146054597E0FF1F5C
:1051E000E7802082930760F82382F17AA383017A13
:1051F0009307002623A4F17AE57793870721239666
:10520000F17AB1452387017AA387A17A1385417A80
:10521000EF10107635BF914763E187029765010073
:105220009385C5F3175501001305456CEF303160C8
:10523000176501001305C585ADBF83C4817A83C797
:10524000717AA204DD8C8327C9046D1422869385AC
:10525000917A280082978E0493160401B775020094
:10526000C1823000A695094597D0FF1FE78060797D
:10527000930770F82382F17A9945A384A17A79B7CC
:10528000914763E1870297650100938525ED1755E6
:1052900001001305A565EF3091591765010013054D
:1052A000A58001BF83C4817A83C7717AA204DD8C93
:1052B0008327C9046D1422869385917A28008297EA
:1052C0008E0493160401B7750200C1823000A695C2
:1052D0000D4597D0FF1FE780C072930780F859BF34
:1052E000175501001305057FEF30B1681305C01293
:1052F00097D0FF1FE78000550145EFD0FFDE0D4539
:10530000EFF0CFCA294597D0FF1FE780A05397D071
:10531000FF1FE780C0442DBDB7E704004111FC47E3
:1053200026C29384417A2E8606C622C44AC02E84A1
:105330002A89AA8526858297976501009385C5E30A
:10534000175501001305855AEF30714E83C5417A18
:105350001765010013058588EF30714D2945EF3041
:10536000115183C7040041479387070693F7F70F4E
:105370006363F74617570100130787698A07BA97CF
:105380009C43BA9782879D476303F40297650100A7
:10539000938585DE1755010013054555EF303149DA
:1053A0001765010013050584EF30714855AA83C7BE
:1053B000517AADC783D7817A03D7617AC207D98F73
:1053C00023A4F18883C76400976501009385C5DA3B
:1053D00017550100130585512383F188EF303145BE
:1053E000938781888C4303C6618817650100130584
:1053F0002581EF30D1432945EF307147A382017AEF
:105400002244B24092440249930700F82382F17A81
:105410009D451385417A41016F109055EF30A04EA4
:105420002393A17A935705012A842384F17A935711
:1054300085010145A384F17AEF30A04D2385A17A3F
:1054400097650100938545D3175501001305054A5B
:10545000EF30F13D03C6A17AA2851755010013056F
:10546000A57B41BFCD476301F40297650100938599
:10547000A5D01755010013056547EF30513B17556F
:1054800001001305E57A0DB737E404007C4441467A
:105490009385517A17F5FF1F13050543829717F57A
:1054A000FF1F13056542EF008076092D83C7617BDE
:1054B00003C7517BA20703238405D98F2392F18868
:1054C0001306000A89452244B2409244024903C5AA
:1054D0008186410102838D476301F40297650100D3
:1054E000938585C91755010013054540EF303134C8
:1054F000176501001305858345BD03C4617A83C721
:10550000517A97650100938525C72204175501003C
:105510001305C53D5D8CEF309131A2851755010013
:1055200013058572EF30B1302945EF3051340D4607
:105530009385417A2285EFE0BF9BAA8415C99765C0
:105540000100938565C3175501001305253AEF3017
:10555000112EA6851755010013054570EF30312D2A
:105560002244B24092440249294541016F30313012
:10557000239F8186B7E70400116603A387051306FE
:1055800006E8914589B78D476301F40297650100EC
:10559000938585BE1755010013054535EF30312938
:1055A000176501001305458701B503C4617A83C7F8
:1055B000517A97650100938525BC22041755010097
:1055C0001305C5325D8CEF309126A2851755010079
:1055D0001305056AEF30B1252945EF3051290D46F5
:1055E0009385417A2285EFE0BF90AA840DC197652B
:1055F0000100938565B8175501001305252FEF307D
:105600001123A685175501001305C56781BF239E89
:105610008186B7E70400116603A38705130606E831
:10562000930500024DB5894763E187029765010044
:10563000938585B4175501001305452BEF30311FB5
:10564000176501001305058085B383C4617A83C79C
:10565000517A97650100938525B2A2041755010080
:105660001305C528DD8CEF30911CA6851755010068
:105670001305C562EF30B11B2945EF30511F22865B
:105680009385417A2685EFE0BF862A846304051658
:1056900097650100938545AE175501001305052553
:1056A000EF30F118A28517550100130565607DB52F
:1056B000854763F18714834519002244B240924420
:1056C0000249B335B0002380B18817550100130596
:1056D000655F41016F30B115A2852244B24092440A
:1056E0004A85024941016FF05FA399476301F402C3
:1056F00097650100938545A8175501001305051FFF
:10570000EF30F112176501001305858D71B903C4DF
:10571000617A83C7517A976501009385E5A52204D4
:10572000175501001305851C5D8CEF305110A285C3
:10573000175501001305855AEF30710F2945EF30D9
:10574000111319469385417A2285EFE06FFAAA84F6
:105750000DC197650100938525A21755010013051A
:10576000E518EF30D10CA685175501001305055833
:10577000F5B323968188B7E70400116603A3870574
:10578000130606E8930500083DBB854797650100B1
:105790009385859E17550100130545156309F4008F
:1057A000EF30F1081755010013058555F5BEEF30B0
:1057B00011081755010013052556EF3051072945EB
:1057C000EF30F10A2244B240924402492392018808
:1057D00041016F30A007976501009385E599175542
:1057E00001001305A510EF309104176501001305A2
:1057F00065835DBEB24022449244024941018280E9
:10580000411106C622C4EFE0AFEE9377F50F95CBBA
:105810002A84976501009385A59717550100130504
:10582000E50CEF30D1009375F40F176501001305F7
:10583000E5BAEF30C17F2244B240294541016F30C3
:105840001103B24022444101828001114EC683D629
:105850002189B28903D6818226CA4AC806CE22CCC3
:10586000AA842E89CD2183C70189A9C703C4440016
:1058700083C7340017650100130545C222045D8CFF
:10588000EF30E17A4A86A68522859D3F638B090227
:1058900083C7E1889DC76306090283C7018895E332
:1058A0006244F240B249CA8526854249D244056124
:1058B0006F10100C176501001305C5BEEF30710B9A
:1058C000F1B7F2406244D2444249B2490561828054
:1058D0008347550083454500176501001305C5BA88
:1058E000A207DD8D6F30A174176501001305C5B8DF
:1058F0006F3031088D4763FAB708011126CA06CE0A
:1059000022CC0344350083C4F18897650100938558
:1059100025BAB3378000A387F18809C497650100D1
:105920009385C5B9176501001305C5B9EF3021701E
:1059300083C7F18863839700212C83C7F1889DC3B7
:1059400085472306F100B7E7040083A747177000D7
:10595000854513055030829717650100130585B7FB
:10596000EF3031019967938757EE2316F1006800F5
:1059700085479145A30781002307F100EF10407F81
:10598000F2406244D244056182808280894763FE8E
:10599000B706011122CC06CE26CA834425008547CE
:1059A0002A846396F404914763FEB70203454500D9
:1059B0008347340022055D8D2394A18209299967CC
:1059C000938767EE2314F100834734002305910089
:1059D000A305F10083474400954528002306F10004
:1059E000EF100079F2406244D24405618280FDF8F4
:1059F0009967938767EE2314F10083D78182A3050B
:105A0000F10023050100A183C1BF828001119967C4
:105A100022CCD517138401892314F1008347040095
:105A200026CA938421892305F10083D70400280026
:105A30009545A305F100A18306CE2306F100EF10E2
:105A4000207303D604008345040017650100130585
:105A5000E5A9EF30C15DF2406244D2440561828025
:105A60009D677971D9172316F10083C7018906D67E
:105A70002307F1009DCBB7E70400FC47414697F5AB
:105A8000FF1F938565E41305F10082976800CD45FB
:105A9000EF10006E83C5018917650100130505A885
:105AA000EF30E158B25045618280B7E70400BC474F
:105AB000414681451305F1008297C9BFB7670203CC
:105AC0006971938757AA3EC4856793871740231649
:105AD000F1009387018983C7070023248112A3075C
:105AE00001002307F1009387218983D7070037E45A
:105AF0000400232611122318F1009387818283D793
:105B00000700414648082319F1007C4497F5FF1F20
:105B1000938585DB8297F1452800F5222312A102A7
:105B20007C442C002810794682973C44130561047C
:105B30001306900D8145829730109305700F014533
:105B4000EFD09FBB8320C112032481125561828054
:105B5000B7C7A55A01119387C7333EC483C7F188DD
:105B60003EC6B7F7070003C7070106CE22CCA547FC
:105B70006313F70001A01164930504F0930600106D
:105B80000146254597D0FF1FE780A0E73000930529
:105B900004F0A146294597D0FF1FE78080E683C522
:105BA000F18817650100130525A8EF304148F24040
:105BB00062440561828001119165A14630009385A0
:105BC00005F02D4506CE97D0FF1FE78080E32247E2
:105BD000B7C7A55A9387C7336310F702B245176555
:105BE00001001305A597B335B000A387B188EF3046
:105BF0000144F2400561828081451765010013056B
:105C00002598A3870188EF3081429937DDB7B7C760
:105C1000A55A79719387F7353EC6B7E70400FC476C
:105C2000AA8506D622D4414608088297B7F707000E
:105C300003C70701A5476313F70001A0116493058B
:105C400004E8930600100146254597D0FF1FE78022
:105C500040DB7000930504E8D146294597D0FF1F2B
:105C6000E78020DA176501001305C59FEF3061500A
:105C7000B25022544561828079719165D14670009D
:105C8000938505E82D4506D697D0FF1FE78060D79E
:105C90003247B7C7A55A9387F73517650100130533
:105CA00025966310F702B7E70400FC4717F5FF1FBE
:105CB000130585C141460C0882971765010013053D
:105CC0002592EF30014BB25045618280B7F7070053
:105CD00003C70701A5476313F70001A091654111B0
:105CE000930600100146938505E8254506C697D022
:105CF000FF1FE78000D1B2401765010013054584FE
:105D000041016F300147C16769768146FD1705067D
:105D10001397060141836364B7003E858280330791
:105D2000D50003470700B98F214713F81700858373
:105D300063050800B18FC207C1837D171377F70F82
:105D40006DF78506F1B749C1A547054763FFB7065B
:105D500083471500034705003168A207D98F1397C1
:105D60008700A183D98FC207C1831308C85505478F
:105D7000639D0705411106C622C426C203442500BF
:105D8000914763FD8702930754006399F502A301CD
:105D9000C50021822302C5009304340091C6A302EA
:105DA000D500A1822303D5002A84A685A93F269485
:105DB0002300A4002181A300A4000147B240224493
:105DC00092443A854101828005473A858280B7C76F
:105DD000A55A01119387E7343EC42AC6B7F70700D6
:105DE00003C7070106CE22CC26CAA5476313F700D6
:105DF00001A091642A84938504EE93060010014665
:105E0000254597D0FF1FE780C0BF3000A14693858E
:105E100004EE294597D0FF1FE780A0BEA285176535
:105E2000010013056582EF308120EFF03FC9F24099
:105E30006244D2440561828001119165A14630001F
:105E4000938505EE2D4506CE97D0FF1FE78060BBFA
:105E50002247B7C7A55A9387E7346312F702B245C2
:105E6000175501001305C5732394B182C205C18182
:105E7000EF30E11BEFF09FC4F24005618280D14713
:105E8000D145175501001305A5732394F182EF3016
:105E9000011A03D58182253FC5B7011126CA06CE56
:105EA00022CC93F71500AE849DC7AD67371700402D
:105EB0009387A7AA1CC3B7E70400BC4F13060019B9
:105EC000854503C56182829713C51400F240624480
:105ED000D2440561828093F72500638B07109755A4
:105EE00001009385257C2D464800EF30E10883C5ED
:105EF0001189854793C4240063EDB70299C983C70C
:105F0000E18891CF8545170500201305A59DEF1069
:105F1000202613950401A3880188418145BF41656E
:105F20000546970500209385E59B7D15EFF05F8D75
:105F3000CDB7170400200344E49A9707002083C7D5
:105F4000779A22045D8CAD67C2059387B755C181EE
:105F50006302F40863E48702A9679387A755630285
:105F6000F40883C7E1888DE741652E867D15970586
:105F7000002093852597EFF0BF88A9A0B16793878C
:105F8000C755630EF400B5679387D755E31BF4FC40
:105F90001705002013050595EF10801D25A0054667
:105FA0001705002013050594EFF03F8A83C7018988
:105FB00091EB4800EF30A12393150501C181480002
:105FC000EFD04FA6A285175501001305A56BEF3042
:105FD000010681B7170500201305C590EFF05F8F0C
:105FE000D5B7170500201305E58FEFF0FF8FD9BF58
:105FF00093F745000145E38B07EC175501001305A6
:10600000A569EF300117EF10C02713C544007DBD0F
:10601000411122C437E404005C5C06C6354697553E
:1060200001009385E51F17650100130525AC8297D4
:1060300001E9175501001305A567EF30811301A091
:106040008327041C82972A840545EF80A065EF1002
:106050004159EF108137EF70301A2285B240224447
:10606000410182801567B71700401307575598C341
:10607000D8439D66558FD8C3D843FD76758FD8C356
:10608000D8431367F70FD8C335671307C7CC98C336
:10609000828041111305800406C622C426C24AC06C
:1060A00097C0FF1FE780805185457D55EFC01FEBEE
:1060B00085457D55EFC0FFF4371400408327840ADF
:1060C0008D451305002093E707202324F40AEFC031
:1060D000FFE8B7E40400EFD06F9AC8581309840CA6
:1060E0001304C40CEF30E10817650100130505A087
:1060F000EF3021088327C4FF8545414593E7070812
:10610000232EF4FEEFC0FFEF8D4513050008EFC00E
:106110005FEFEFD0CF890145EFD08F8C85450545E6
:106120008947238AF188EFD04F8D37070004B7E7FE
:1061300000E023A0E710EFD07F8BEFD05F9FC93D39
:10614000EFF07FA7EFF05FCFEFE0AFE28D450D6599
:10615000EFC03FEB170500201305C58885671CC5F8
:1061600089672320250140C12326250100C95CC978
:1061700083A7841E829783A70408170500001305D0
:1061800005D282972383A182BC4C13060064854507
:106190008297C93D97C0FF1FE78000750145828047
:1061A000B7F7070003C70701A547AE866316F700D8
:1061B0009397450191C301A0AA850146254517D3B0
:1061C000FF1F670003844111B2862E86AA852D45E4
:1061D00006C697D0FF1FE780C082B240014541014B
:1061E00082809307000463E6C7021D71A2CC2A8453
:1061F000080886CE32C6EF203158B2461008A28574
:10620000294597C0FF1FE780C07FF640664425619F
:10621000828039558280411126C2AE848D4522C4C8
:1062200006C62A84EFC0FFDDB717004099C803A552
:10623000C70C418D23A6A70CB240224492444101D1
:10624000828003A5870C418D23A4A70CF5B7834753
:10625000050003471500A207D98FC2076177C187E0
:10626000130727206397E7008345250037050400BF
:106270005DB782809387818918429C4383D645000D
:106280000345070083C5C700035646006396A50073
:1062900083D5E700638DD502011106CE2386A700C2
:1062A0002397D700B705CF00DC4B9385757D050795
:1062B0007D162EC2230001003AC42316C100231705
:1062C000D10099C30A858297F2400561828082805D
:1062D000DC4DDC4B91CBB7E70400904503A3870569
:1062E000914503C5C189028382806D713C083EC619
:1062F000B707E500232291103EC8AA843C083285E6
:10630000232611103ECA23248110232021112E8917
:10631000EF2010592A84975501009385A541174510
:1063200001001305A55CEF209150A28517550100CF
:1063300013054550EF20B14F2945EF205153B705C4
:10634000CB009385757D6800EF102035A28568002D
:10635000EF20B04A014781467000CA852685EF10BC
:10636000405415C52A84975501009385A53C1745CF
:1063700001001305A557EF20914BA2851755010089
:106380001305054CEF20B14A2945EF20514E8320DB
:10639000C11003248110832441100329011051618D
:1063A00082809387818918429C43797122D406D6D2
:1063B0000348070083C807012A8483D64500035594
:1063C00046006396080183D82701638DD80223888D
:1063D000070105072399D7003708CC00DC4B1308C9
:1063E000787D3ACC1307F5FF42CA23080100231E2B
:1063F000E100231FD10099C7080832C62EC4829736
:106400003246A2452285D535B2502254456182805C
:106410006D713C083EC0B707E5003EC23C083EC473
:106420002326111023248110232291102317010009
:106430002318010023190100231A0100231B010066
:1064400097D7FF1F83D7470E99E3C167FD17231620
:10645000F10097D7FF1F83D7470D81EB9387818981
:106460009C439C43DC4783D7070017D4FF1F1304CA
:10647000A40B584C2317F10083574400484B2318B2
:10648000F10005ED975501009385C53117450100D1
:106490001305C545EF20B139175501001305C53166
:1064A000EF20F1382945EF20913C8320C1100324CF
:1064B0008110832441105161828097D7FF1F83C7C9
:1064C000170789EBB7E70400BC5782975C4C23AAF7
:1064D0000700E1BFFD1797D6FF1FA38AF6040356F6
:1064E0000701834704014C470A85230BF100EF2085
:1064F000F02E938781899C430147814688430A8611
:106500006C00EF10003AAA841DC9975501009385CD
:106510006529174501001305653DEF205131A6851A
:10652000175501001305052AEF2071302945EF208A
:106530001134584CB7E70400BC57484B79B797D78C
:10654000FF1F83C7D7FEF5D7B7E70400BC4F104441
:10655000854503C5C189829789BF5C4EDC4BB9C7AD
:10656000B1C5411122C417450100130525382E84F9
:10657000975501009385452106C6EF20512BA28532
:106580001755010013054526EF20712A2945EF20F4
:10659000112EB7E704002244B24003A3870503C5C8
:1065A000C189130640069145410102838280411151
:1065B00022C417D4FF1F130424F51C4C06C689C738
:1065C000DC4399C34C488297584CB7E70400BC574A
:1065D000484B82975C4CB240224423AA07004101F9
:1065E00082801387A182834707009306F00B8507FB
:1065F00093F7F70F63E7F6002385F1820345070061
:106600008280930700F8CDBF835745006384070E4F
:1066100001114AC817D9FF1F130909F152C4032AEF
:10662000C90106CE22CC03274A0126CA4EC656C24D
:10663000F15721EF1307D00DFD576368C704B7E981
:10664000040083A709072A841305860042054181B7
:10665000B284AE8A8297232AAA000325C9015C4925
:106660009DEF9755010093852510174501001305EF
:10667000E527EF20D11B175501001305251FEF203B
:10668000111B2945EF20B11EDD57F2406244D24470
:106690004249B249224A924A3E85056182809387E7
:1066A0004400B705CF002319F5009385757D3105AA
:1066B000EF00B07E0325C901834564003105EF205A
:1066C000D0130325C9012686D6853105EF20101188
:1066D0007146A2854A85EF20310A504409CA83A732
:1066E0008905854503C5C1898297814779BFEFF048
:1066F0003FD2E5BFFD573E858280411126C297D427
:10670000FF1F938464E2D84C22C437E404003C5455
:10671000484B06C68297DC4C0323C4052244B24092
:10672000924423AA070003C5C1898545410102831C
:10673000411126C2938481899C4006C622C44AC066
:10674000C9C7DC43D9C35CC12300B5002A8497556F
:1067500001009385A5FC1745010013052519EF20BD
:10676000110D2945EF20B1109C4023A4070023A25E
:10677000070097D7FF1F938727D9DC4FDC4B81C7D2
:106780002955EFF0DFE297D7FF1F9387E7D9DC4F5A
:10679000DC4B91C39D3737E904008327C905894540
:1067A00003C5C18982978327C905914503C5C1895E
:1067B00082979C4003A3470163090300228522447A
:1067C000B2409244024941010283B24022449244C1
:1067D0000249410182800111328506CE22CC26CAAF
:1067E0002E84EF20F00BAA8497550100938545F67F
:1067F000174501001305850FEF207103030784007F
:106800000356640083554400A686175501001305FE
:10681000A5FFEF20D1012945EF20710597D7FF1F74
:1068200083C7E7CE639897000145EFF05FD88145B5
:106830000A85FD3DF2406244D244056182806D715B
:1068400023248110232611102322911093F7450051
:106850002E84638107123C083EC0B707E5003EC2A4
:106860003C083EC42317010023180100231901002E
:10687000231A0100231B010097D7FF1F83D7C7C826
:1068800099E3C167FD172316F10097D7FF1F83D740
:10689000C7C781EB938781899C439C43DC4783D79F
:1068A000070017D7FF1F130727C62317F100544F00
:1068B000835747002318F100DC4A95EF97550100F4
:1068C000938545ED1745010013054502EF2021761C
:1068D00017550100130545EEEF2061752945EF209E
:1068E0000179134544008320C110032481108324BF
:1068F00041105161828097D7FF1F83C757C125552B
:10690000BDC7FD1717D6FF1FA303F6C003D60601A8
:1069100083470701CC460A85230BF100EF20006C6A
:10692000938781899C4317D7FF1F1307E7BD97669D
:1069300001009386E6BA88430A866C00EF00707601
:10694000AA8445D1975501009385C5E417450100F8
:106950001305C5F9EF20A16DA68517550100130594
:1069600065E6EF20C16C2945EF2061702685EFF0C8
:106970001FC485BF93F725009DC3B7E70400BC473C
:1069800041468145280882972555EFF05FC22808C7
:106990009305F00FEFF0DFD913452400A9B793F763
:1069A00015000145A9D3EFF0BFA61345140025BF7C
:1069B0005C4D411106C688C323ACF188B7E70400DB
:1069C00083A70708170500001305A5E78297B240C3
:1069D000238EA18801454101828001119307700F28
:1069E0002316F10006CE83C7918A99EFB7E704001A
:1069F00083A7870D03C601836C0003D5C18A8297E4
:106A00003335A000A384A18AF24005618280411140
:106A10009397050122C406C626C2C1872E8463D27D
:106A20000702B7E40400FC5403C50183829719C12F
:106A3000BC5482972165218DB24022449244410189
:106A4000828093F715009DC3B7E7040083A7471A18
:106A500017D6FF1F130646AF97F5FF1F938585FDD9
:106A600003C50183829713451400F9B793F72500F6
:106A700089CFB7E70400BC4F13060064894503C5FE
:106A8000018382971345240045BF93F785009DC37A
:106A9000B7E7040003A8871A1307401F83C70183C1
:106AA000814613064006994503D5C18A02981345CD
:106AB000840059B793F745000145BDDFB7E40400F2
:106AC00083A7041803D5C18A8297BC4C13060064BF
:106AD000914503C50183829713454400B1BF83D715
:106AE000C18A6390A7022397B18A2398C18A239908
:106AF000D18A2E8617550100130505EDBE856F203E
:106B00000153175501001305A5ED6F20816603574A
:106B10004500011106CE22CC83D7C18A175501004A
:106B2000130505EC6316F704C167F91723A6F18A6C
:106B300037E4040023A8018A7C4C894503C50183FE
:106B400082977C4C914503C50183829783C7F18866
:106B500095C78547A307F100832744171306F10063
:106B60008545130550308297175501001305C5DC84
:106B7000EF202160F24062440561828083C7018971
:106B800017550100130505E0E5F78547A307F10058
:106B9000832744171306F10085451305503082976B
:106BA00017550100130585DBE1B77D15954763EEA9
:106BB000A716175701001307E7D40A053A951C4199
:106BC000011122CC06CE26CABA972E848287175589
:106BD0000100130565E1EF20C159FDA803C7250099
:106BE0009947631DF7002E85EFF07FF2834564001F
:106BF00017550100130545E0EF2061432387018805
:106C000017550100130505E1F9B703C7250095479E
:106C10006315F702C16703D7C18AF91703D5A50029
:106C20006305F702B7E7040083A7C71782971755D4
:106C30000100130525DFEF20C15385472387F18825
:106C400017550100130585E079B72396A18A83D7EC
:106C5000E500B7E4040009662397F18A83D70501AC
:106C60001306069003C501832398F18A83D7250173
:106C7000A1452399F18ABC4C8297BC4C1306006451
:106C8000914503C5018382970356E4008355A40010
:106C900017550100130545DAEF20613979BF175503
:106CA0000100130565DB05BF83C525009147639A85
:106CB000F502854717550100130585DBA307F10091
:106CC000EF20214BB7E7040083A747171306F10015
:106CD0008545130550308297F2406244D2440561E5
:106CE00082809947639EF5002285EFF05FE283453D
:106CF000640017550100130525D0EF204133E9BF8B
:106D00009547639FF500834714001755010013054D
:106D100025D6E39207EC17550100130525D765BD6D
:106D200017550100130505D7C9BF82806D71232453
:106D300081102326111023229110328401CD89471E
:106D40006306F5028320C1100324811083244110BF
:106D50005161828017550100130585D4AE84EF2060
:106D60004141A2852685EFE02FDBE9BFB7E70400AC
:106D7000FC472800829717550100130525D3EF2003
:106D8000413F8347810029C01307000B638EE70052
:106D90001387A7051377F70F8D4663E7E602A285F1
:106DA0002800EFE08FB779BF8547E3FD87F883457B
:106DB0009100174501001305E5F0B335B0002380BD
:106DC000B188EF20C126BDBF03479100A207D98F2C
:106DD00035671307D755638DE7066366F7022D679E
:106DE0001307B7556381E70631671307C7556386F5
:106DF000E70429671307A7556392E702A2852800D5
:106E0000EFE09FAE81B739679306E7656383D706E6
:106E100063E9F6001307E7556388E704A2852800B5
:106E200099B73D679306F755638AD7041307F7664A
:106E3000E396E7FEEFE0DFC231B70146A285280006
:106E4000EFE0BFA001B7A2852800EFE07FA8DDBD7D
:106E50008947E3F987EE9305E4FFC205C181130575
:106E6000A100EFC02FBCF9BDA2852800EFE09FA8CC
:106E7000D1BDA2852800EFE07FB1E9B5EFE01FB9F1
:106E8000D1B5411122C417C4FF1F1304A46DAA86F3
:106E900017560100130686A82285C14506C6EF20B5
:106EA000012E0357440097C7FF1F9387A76C2393B6
:106EB000E700035764002394E700B24022444101F5
:106EC0008280011106CE22CC6D3F37E40400832777
:106ED000841417C6FF1F1306E668D545014582973F
:106EE000832784179305F100130550308297834759
:106EF000F100A1C7A3070100832744171306F1007F
:106F000085451305503082978327441717C6FF1F06
:106F100013064666CD451305703082978547A30753
:106F2000F100832744171306F100854513055030FF
:106F30008297F2406244056182808327441717C616
:106F4000FF1F13062663CD4513057030D5B7130117
:106F500001DE232C812037E4040083270408232E3C
:106F60001120232A912023282121232631211705AE
:106F70000000130505AA8297138901839947854468
:106F80002300A9002318F10097550100938505A25D
:106F90009307400617450100130545952314F1108A
:106FA0002304910093892189EF20610883D509008A
:106FB0001755010013054597EF2061072945EF207C
:106FC000010B03D50900EFF0DFEB832744173000F6
:106FD00085451305503082978327441717C6FF1F36
:106FE00013064659CD451305703082978327441701
:106FF00017C6FF1F13060656B54513056030829766
:107000008327441710088945130510318297832779
:107010004417300289451305203182978327441590
:10702000930500050D4582978327441593050005B8
:1070300011458297A301910023029100230491003E
:107040002324011023080100832784163002914570
:1070500013057040829783278416130631008545F7
:107060001305004082978327841650008545130539
:107070001040829783278416100885451305204009
:1070800082978327841630008545130550408297E8
:10709000832704157D558297832744137D55829756
:1070A0007D55EFC0CFDE8327440C8297EFC08FBCA5
:1070B0008327841417C6FF1F1306C64AD54501450A
:1070C000829789471306700F814508082302F10053
:1070D000EFB0AF988D471306700F81452802230843
:1070E000F100EFB08F9791472304F11093878183CC
:1070F000984383C747003AC42306F100EFE01F9C82
:10710000500085450545EFC02FDF10089305700F2F
:107110000945EFC06FDE30029305700F0D45EFC0DB
:10712000AFDD300095451145EFC00FDDC167138716
:10713000C18AF9171CC3232207001385C182EFC03F
:10714000CFDA8327C41D1385018A82973C48034503
:107150000900854582978320C1210324812183244E
:107160004121032901218329C120130101228280A9
:107170000111C16726CA06CEAA8422CC03D5C18AD2
:10718000F9176304F50437E40400832784122E867C
:107190002315B10001478146ED4582977C44035693
:1071A000A1002AC6A68582972C0003D5C18AEFC00C
:1071B0000FDF01CD1755010013054580EF10717BDE
:1071C0008327C412ED4528008297F2406244D244DE
:1071D00005618280011106CE22CC2DC9854717C7D3
:1071E000FF1FA30EF73697C7FF1F238B073637E421
:1071F0000400832784179305F1001305503082970C
:107200008347F100A9CBA307010083274417130686
:10721000F10085451305503082978327441717C620
:10722000FF1F13062633B545130560308297854747
:10723000A307F100832744171306F10085451305C2
:1072400050308297F24062440561828097C7FF1FE9
:10725000A387073049BF8327441717C6FF1F1306AC
:10726000662FB54513056030E9BFC16703D5C18AF4
:10727000F9176307F500B7E7040003A3C7170283F4
:10728000828001118547A30701002384F18AB7E7B3
:10729000040083A7471706CE1306F10085451305A2
:1072A00050308297F24005618280EFA27FF62A84F7
:1072B00008452E89B28909C900C197050000938548
:1072C000C5746105EF00810181447D5AEF10C0094A
:1072D00063C3A4048144EF10200A63C6A40497E7A3
:1072E000FF1F9387E7759C43DC47B307F9409187FD
:1072F0002302F400638109048327C900B307F44023
:107300009587A302F4001C4C89C79C4799C322852A
:1073100082976FA03FF35C44139714008504BA97DB
:107320002390470165B71C48139714008504BA974A
:10733000239007004DB7832789000547B307F44022
:107340009587A302F40083570400638EE7028DC380
:1073500009476384E7040D47E397E7FA975701006D
:10736000938787C71CCC975701009387E7C711A85D
:10737000975701009387C78D1CCC975701009387BF
:10738000278E5CC849B797470100938767791CCC63
:10739000974701009387C779EDB797570100938707
:1073A00067C81CCC975701009387C7C8D9BF85E130
:1073B000EFA2BFE7004618448347940075839D8B76
:1073C0006315F700EF00501C48C46FA05FE882808F
:1073D000EFA21FE413893500C16442094111AA8953
:1073E0000144F11413590901054A2EC6EF00D07764
:1073F000B2456346A400014541016FA0BFE483A7E5
:10740000090013171400BA9783D707006388B700E1
:107410006394970063742A010504C1BF0545E9BF61
:10742000EFA23FDEAA892E89328BB6843A8ABE8AC1
:10743000EF80204C55C12685EF1030368D4763E52F
:10744000A7007D556FA07FDF83DB4400EF00D0777E
:107450002A84EF00B0789307740031443305850225
:1074600063C5A702EF005076EF0010762A84EF0084
:10747000F0769307740031443305850263CDA7028B
:10748000EF0090749307450019A8EF00307533059D
:1074900085021307F0179307C017E357A7FC2D5574
:1074A000E3C277FB63000B02D6865286A6854A8527
:1074B000EFE0106341BFEF00707233058502930760
:1074C000C5FFF1BF832749001385C90083D5270075
:1074D000EFF01FF071F9B5B76955ADB797E7FF1F2A
:1074E0002392A75697E7FF1F9387875590438147BD
:1074F0000C463307F500420741836393B70082804F
:107500005446139847008507C2962390E600D5B7E6
:1075100097E7FF1F9387C7529C4303C5870082806C
:1075200017E5FF1F035505528280EFA21FD0C167E8
:107530001387D7FF6307E5026368A700F117630E9F
:10754000F50001456FA0BFD01387E7FF630EE5008C
:10755000FD171D8D13351500F5B7EF40003D7D1566
:10756000D5BFEF40801AE5BFEF40E018CDBFEFA2D6
:10757000DFCB4111AA8401442EC6EF00F05FB24573
:107580006346A400014541016FA07FCC9C481315C0
:1075900014003E9583570500E387B7FE0504E9BF55
:1075A00003485500814693F7F60F63E507018147CD
:1075B0003E858280584593975600BA9703D7270097
:1075C0006316B70003D70700E304C7FE8506E1BFD3
:1075D0008346450001479377F70F63E4D70081475F
:1075E00011A81C45131657000507B29703D60700CC
:1075F000E313B6FE3E858280EFA29FC1931705017B
:10760000C18797EAFF1F938AAA436355F00883A7AF
:107610000A00C0479C4703570400198D4205418169
:107620006366F500014422856FA0DFC112052A942C
:10763000DDBFDC4713944900014A3E948347440070
:107640006341FA02014A834754006347FA028509FD
:10765000C20993D9090183A70A009847E3EBE9FC23
:10766000D1B71C4413195A00A6853E994A85EFF0FC
:107670001FF011ED050AD9B75C4413195A00A6850D
:107680003E994A85EFF0BFEE19E1050A6DBFE300B0
:1076900009FC51BFAA8481497DBFEFA21FB91C45D7
:1076A0002A8481E79307C5001CC51C4423120400EB
:1076B0001CC09307F00F63E9B70093F5F50F22851F
:1076C000EF10B0136FA0BFB893940501C167C180DC
:1076D00063F7F500A6852285EF10D015E5B7C181C7
:1076E00093F5F50F2285EF105011A6852285EF1036
:1076F0001012C9BF97E7FF1F9387873488438280A2
:107700001C4599C797E7FF1F23ACA732014582802C
:107710007D55828097E7FF1F938787329843834781
:107720004500484792073E958280EFA21FB06171E5
:1077300000451C183EC6B70780013EC81C183ECA4B
:107740008357440002CE02D002CC231EF1008347AF
:1077500084002A8902D22301F1023C083ED402D6D9
:10776000EFF05FFB835705002316F102EF30706BDB
:107770002307A1025C4003556400F18313F717004F
:107780008347F10252055181F99BD98FA307F1027A
:10779000EFE0702639C5AA8403550500EF80401636
:1077A00083D704002AD26800231CF10083D7240069
:1077B000231DF1001C4803D647008C43EF10100234
:1077C0008347B400CA86174601001306E62E8117C8
:1077D000A305F4006C004810EFE090305D616FA0ED
:1077E0001FA72155E5BF1C45B1CF03C5A70089469A
:1077F00013576500630BD7028D46630ED70285468B
:107800006300D702130740063305E50203C7B7003C
:10781000418B15CB83C7B700BD8B3355F5408280B4
:107820001375F5031307803EC5B709671375F50394
:1078300013070771D1BF372709001375F503130725
:10784000077CD9B701458280EFA23F9E03A985003E
:10785000630509048347B900AE8493F7070E91CFFF
:1078600003459900930520030D810505B305B50275
:1078700088446105EFF0B0320DA02E85EFF0BFF621
:107880002A8401CD11238325C900B307B54063F8CD
:1078900087002E94B305A440E1FD6FA05F9B854552
:1078A000C1BFEFA29F982A8403D50500011132C6FB
:1078B00036C43AC22EC002CA02CC02CEEF804004C7
:1078C00082452ACA22852ECCEFF0DFE4035705005B
:1078D000231EE100EF30F054A24632469247230FB8
:1078E000A10036874C08B28622850146EFF05FB3CF
:1078F00005616FA0DF95EFA25F9361711C183EC612
:10790000B70780013EC81C183ECA3C0800453ED45B
:10791000AA8402CC02CE02D002D202D6EFF09FDFC0
:107920008357050035592316F102EF30904F230796
:10793000A10209C48357440091E721594A855D613A
:107940006FA0FF900355640052055181EFE0B00A2B
:107950002A8965D58347B40093F7070E89C71305B5
:107960008401EFF0502583574400231EF100834724
:1079700084002301F1025C4003550900D98313F709
:10798000070883471102231CA10093F7F707D98F3B
:10799000A300F10283572900231DF1005C40F1830D
:1079A00013F717008347F102F99BD98FA307F10260
:1079B000EF7010752AD251D1834794006800139755
:1079C00057008347B400FD8BD98FA305F4001C48F2
:1079D00003D647008C43EF106060A687174701006D
:1079E0001307870D740005464C102685EFF05FA342
:1079F0002A8929D58347B400A685FD8BA305F40009
:107A0000EFF09FE425BFEFA25F82832485FE2A84E6
:107A100041112685EFF03FDD834734FF93F7070ED2
:107A20009DC32AC62685EFF05FD019C9834734FF6E
:107A3000B245FD8BA309F4FE81C52285EFF0301617
:107A400041016FA0DF806DDD8327C4FF268582970B
:107A500065F9834734FF93F7070E81C72285EFF05E
:107A60009015032584FEEFF01FE9D9BFEFA2EFF8D0
:107A70009C4141112A8903C7070089472E849356E8
:107A80006700638CF6020D466382C6049307F00715
:107A90006302F7022E85EF10A060AA848149C16BB2
:107AA000130C490097E7FF1F938787F99C4398477A
:107AB00063ECE90241016FA00FF803D74500854749
:107AC000E3FAE7FE2E85EF108061C1BF03D74500C2
:107AD000E3F2E7FE2E85EF10A05CAA842285EF106A
:107AE000805DC204C98C5DBFDC470355A900139AB1
:107AF00049003E9A93170501C187635DF0008357E3
:107B00000A006395A70263E574038327CA00034D47
:107B10005A001DA0A1672167A98F1307F7EFE3742F
:107B2000F7FE63950900EFF05FA071FD85099DBF29
:107B300083278A00034D4A00835DA900035769002B
:107B4000216A138BC7003AC6814A33CA4D01631EAE
:107B50005D0197E7FF1F938727EF9C43E1DBA28638
:107B60006286814526858297D1B7A1679387F7EF13
:107B7000930C4BFF63F04703B2455A85EFF05F85E6
:107B800019CD03278B00104719CA10436380C40224
:107B90003107D5BFEE856685EFF07F9D71FD938639
:107BA0001A0093FAF60F130B0B0255B783564400D5
:107BB0005C43E3EDF6F622853AC6EF10603DA1671F
:107BC0009387D7042A8A035D4400324763E897000D
:107BD0008347D90093E707F8A306F9001C47668599
:107BE0002286E2858297C1670844FD17337AFA003E
:107BF000529508C02312A40115BF97E7FF1F938772
:107C000027E49843814715C31447814763FFD50094
:107C1000939745004C47BE9519C903C75500814746
:107C20006375E600DC451606B2973E85828003C781
:107C300045008147E37BE6FE16069C45F5B7EFA2BB
:107C40002FDDAA892E8A814497EAFF1F938A4ADF93
:107C500083A70A00984763E4E4006FA0AFDEDC4727
:107C60001394440001493E9413BB1400834744001D
:107C7000634BF900014913BB140083475400634F61
:107C8000F9008504F1B70844931759005287DA8642
:107C90000146A2853E9582990509C9BF48449317BC
:107CA00059005287DA860546A2853E9582990509D4
:107CB000E9B7EFA28FD7814517F5FFFF1305255FC1
:107CC00097E7FF1F239007D8EFF07FF76FA02FD81B
:107CD00097E7FF1F9387C7D69C4381CFEFA2EFD4CE
:107CE000814517F5FFFF1305855CEFF05FF56FA089
:107CF0000FD68280EFA2CFD137E40400832784120D
:107D000041112315E100AE893289368A3A868146CF
:107D10000147ED45AA8482972AC621C50356A100D2
:107D2000D285EF1061258327C413CE8526858297DF
:107D3000058915C58327440D2314210101462C0014
:107D4000268582972A8401C9B7E7040083A7C71252
:107D5000ED4528008297228541016FA0AFCE4944AE
:107D6000E5B76554CDBF5C41FD175CC18280EFA2D1
:107D7000CFCBB7E70400FC5F829795473305F50248
:107D800081450D816FA0AFCCEFA22FCAB7E70400E9
:107D9000FC5F829795473305F5020D816FA02FCBCD
:107DA000EFA2AFC8B7E7040083A7870B0355050010
:107DB00082976FA0CFC9EFA24FC703550500328746
:107DC000AE8617C6FF1F0356068197E5FF1F9385F2
:107DD000E5C7EFF03FF26FA08FC7EFA20FC5B7E77F
:107DE000040083A7C71782976FA06FC6EFA2EFC3E7
:107DF000B7E7040083A7871397E5FF1F938505C5A1
:107E0000829701456FA0AFC4EFA22FC2B7E704006D
:107E100083A7C71F814517B5FF1F0355C5778297F5
:107E20006FA0EFC2EFA26FC0B7E7040083A787136C
:107E300097E5FF1F938585C2829701456FA02FC1EB
:107E4000EFA2AFBEB7E7040083A7C71F814517B5F0
:107E5000FF1F0355457A82976FA06FBFEFA2EFBC5B
:107E60002E85EF600055EF60900D6FA04FBEEFA222
:107E7000CFBBEF60D0176FA08FBD5C49E1175CC925
:107E80005CC583572501A1072319F5008357050118
:107E9000A1072318F5008280F1473305F50297E723
:107EA000FF1F9387A7BD9C433E9582808D47631734
:107EB000F60603D74600854763F2E706EFA2EFB662
:107EC000368536842E89EF10A01D39C183574400B2
:107ED00093140501C18063ED97022285EF10401CC9
:107EE000FD14231294009307A002630EF50093077C
:107EF000B0026301F50293079002631BF50022852F
:107F0000EFC0B07E31A00146CA852285EF80000F08
:107F10006FA0EFB32285EF001059DDBF828097E696
:107F2000FF1F9386E6B59C42014599CF9843D44202
:107F300017E6FF1F2326E6B46396D70097E6FF1FD8
:107F400023A2E6B41385C7FE8280EFA20FAEE92616
:107F50007144330585029145EF70606201E5655516
:107F60006FA0EFAE97E7FF1F23A8A7B075263305D4
:107F700085029145EF70A0607DD197E7FF1F23AF89
:107F8000A7AE592E97E7FF1F2392A7AE712697E75A
:107F9000FF1F239EA7AC97470100938727B717E7DA
:107FA000FF1F2329F7AC97070000938747ED17E7DA
:107FB000FF1F232FF7AA014565B7EFA20FA7AA85D8
:107FC00017E5FF1F130585AAEF1060216FA02FA8EA
:107FD000EFA2AFA5EFF07FFEEF10E02197E7FF1FC4
:107FE000938707AA9C4381CF1387C7FE09CB83D50C
:107FF000C7FF17E5FF1F130525A9EFF0403A6FA053
:108000000FA5EFA28FA2EFF09FF119C9834785005A
:108010002A8493F7070499E70355E500EFF05FFB27
:108020006FA0EFA28347C5009304450117E9FF1F26
:10803000130909A585E3832709005CC997E7FF1F9A
:1080400023A097A483274900E1FF97E7FF1F23ABF5
:1080500097A2F9B7FD172306F5006105EF60E07EF2
:108060008307840063CB07048347840093E707F802
:108070002304F400B7E704009C5F82974205A947F8
:1080800041813375F5028347840093F707FCC98F5C
:108090002304F4008347D4003E951C402318A40019
:1080A00089CF984319CB8347C40050408145850749
:1080B0003305F502420541810297832709005CC818
:1080C00097E7FF1F23AE979A8327490089E797E731
:1080D000FF1F23A9979A8347C400B9D3835504018E
:1080E00017E5FF1F1305459AEFF0602B15BFEFA2B0
:1080F000CF9397E7FF1F938767BE9C470144858313
:10810000858B81EFAE84B2853A86EF1020142A84E5
:1081100009C5EF10200B829408CC22856FA02F9305
:10812000EFA20F8F41112E8932C6AA89712C3247D6
:1081300013060502CA8697050000938525D617E524
:10814000FF1F1305A592EFF09FFA2A8429CD93040F
:10815000C50065261946AA852685EF003068854545
:108160002685EF001065174501001305E5974E952C
:10817000834505002685EF0050685C4831468145FF
:10818000A1075CC85CC483572401E1172319F400DC
:1081900083570401E1172318F4001C4C3E85EFA01F
:1081A000CF8BA3042501228541016FA0AF89EFA2E7
:1081B000CF874111AA842EC632C4EF100003004DB0
:1081C000B2452246834784000CC050C093F7F703A2
:1081D00093E707042304F400231804002685EF0026
:1081E000707E83479400A9462317A40013D7370055
:1081F00005073307D7029D8B85072306F400A306E6
:10820000E40083C70401D8488507230FF7FE17E76A
:10821000FF1F1307E7865843232A040093074401EE
:108220001DEB17E7FF1F232FF78417E7FF1F2329F5
:10823000F78417E4FF1F130424852285EFF0A00BB9
:108240001C44858B5D8D09E581452285EFF0201565
:1082500041016F90DFFF1CC317E7FF1F2324F78244
:10826000C9BFEF929FFC97050000938565C4014547
:10827000EFF0DFBE01456F909FFDEF921FFBEFF027
:108280001FBF6F90DFFC8347C500A1E7EF92FFF9A6
:108290002A840355E500EFF05FD215C983478400B7
:1082A00093F7F7FB2304F4001C4091C7DC4381C71C
:1082B0004C4001458297EFF09FC617D5FF1F13056D
:1082C000A57CEFF0400F0355E400EFF07FD06F90F6
:1082D0001FF88280EF927FF597D7FF1F9387477A29
:1082E00097050000938525D217D5FF1F1305C57983
:1082F00023A0070023A20700EFE0507E6F903FF518
:108300001C4D91CBDC4381CBEF923FF283450700BC
:1083100082976F90DFF3828097D7FF1F938707794B
:108320009C4303C50700828097D7FF1F9387077878
:108330009C4303C51700828097D7FF1F9387077759
:108340009C4303C52700828097D7FF1F938707763A
:108350009C4303C54700828097D7FF1F938707750B
:108360009C4303C53700828097D7FF1F938707740C
:108370009C4303C55700828097D7FF1F93870773DD
:108380009C4303C56700828097D7FF1F93870772BE
:108390009C4303C57700828097D7FF1F938707719F
:1083A0009C4303C58700828097D7FF1F9387077080
:1083B0009C4303C59700828097D7FF1F9387076F61
:1083C0009C4303C5A700828097D7FF1F9387076E42
:1083D0009C4303C5B70011E11D45828097D7FF1F5D
:1083E0009387C76C9C4303C5C700828097D7FF1F44
:1083F0009387C76B9C4303C5D700828097D7FF1F25
:108400009387C76A9C4303C5E700828097D7FF1F05
:108410009387C7699C4303D50701828097D7FF1FC5
:108420009387C7689C4303C52701828097D7FF1FA6
:108430009387C7679C4303D54701828097D7FF1F67
:108440009387C7669C4303D56701828097D7FF1F38
:108450009387C7659C4303D58701828097D7FF1F09
:108460009387C7649C4303C5A701828097D7FF1FEA
:108470009387C7639C4303C5B701828097D7FF1FCB
:108480009387C7629C4303C5C701828097D7FF1FAC
:108490009387C7619C4303C5D701828097D7FF1F8D
:1084A0009387C7609C438857828097D7FF1F938725
:1084B000E75F9C4303D5C702828097D7FF1F93874E
:1084C000E75E9C4303D5E70219E11305800C828027
:1084D00097D7FF1F9387875D9C4303C5070382805F
:1084E00097D7FF1F9387875C9C43C85B828097D791
:1084F000FF1F9387275B8843828097D7FF1F93874F
:10850000A75A8843828019E17D558280F5DE984222
:1085100065DFFDD917D7FF1F1307477C1847AA87C8
:108520007155058B6319072203C507001547E37DC5
:10853000A7FC03C737001305F0057D171377F70F66
:10854000E364E5FC03C35700E30003FC83C8670052
:10855000E38C08FA03C77700494579171377F70FBB
:10856000E364E5FA03C7A70011481305F7FF137585
:10857000F50FE36BA8F803CE97000D481305FEFF37
:108580001375F50FE362A8F803C8B7006309080084
:1085900065181378F80F1305600DE36705F703C539
:1085A000C700794879151375F50FE36FA8F403C870
:1085B000D7000D457D181378F80FE36705F503D84C
:1085C0000701930E40175118420813580801E3EDB4
:1085D0000EF303C8E7007D181378F80FE36605F380
:1085E00003C827017D181378F80FE36F05F103C85E
:1085F0008700C54E75181378F80FE3E70EF103D81E
:108600006701856E938EBEE06D184208135808010D
:10861000E3EC0EEF03D847016D1842081358080128
:10862000E3E40EEF03D887017918420813580801D4
:10863000E36C05ED03C8A7017D181378F80FE36517
:1086400005ED03C5B7011D487D151375F50FE36DE5
:10865000A8EA03C5D701714879151375F50FE365CD
:10866000A8EA03D5E7011308E00F7D154205418113
:10867000E36CA8E803C50702494879151375F50F9F
:10868000E364A8E8C85301C937C834005915130872
:1086900058BFE36BA8E603A8870237C5340013056B
:1086A00055BF5918E36205E717D5FF1F232EC53EB6
:1086B00003C6050117D5FF1F232AF53E0545E375BF
:1086C000C5E403D82501D04933760603E31E06E24C
:1086D00003C61501E30A06E217D6FF1F2324B63CA2
:1086E00083C5270001466387A50003C61700F1452F
:1086F0003306B60283C707039305C00272971A07B1
:108700001307C70516031A9796084697B387B7024B
:1087100041553E97329742074183636EE802EF92DC
:10872000DFB03685EF60D06FEFD0B0212A84EF80C4
:10873000B01D2A94EFC090252A94EF7040072A9428
:10874000EFF0BF802A94EF2050632A94EF504066E8
:1087500022956F90DFAF8280EF923FAD4111A3076A
:10876000A100EF80801E9305F1001705000013059E
:1087700065B9EFF0CFCC014541016F905FADEF924D
:108780005FA817D4FF1F1304645503288400795988
:108790009368180097D4FF1F23A614551378180068
:1087A000631E0800BA84BE89368B328A2E89AA8A53
:1087B000EFE01FD67D15269509E531594A856F9062
:1087C000DFA7EFE0FFD47D152695A167E357F5FEFF
:1087D00097E7FF1F9387878798433E8C814B11C78C
:1087E0000145EFC0B03E933B15004A85DA865686B8
:1087F000D285EF7070372A8911CD1C44F99B17D7A9
:10880000FF1F2321F74E83270C00CDDBE3880BFAF3
:1088100082976DB7268597D7FF1F23A3074CEFE0FC
:10882000FFCB4146CE8517D5FF1F1305A554EF009A
:10883000A174EFA070080325040BEFA0700A054592
:10884000EFA070100545EFF03FF18DBF97D7FF1FE8
:108850009387C7489C47858BD5C7EF921F9D17D537
:10886000FF1F1305654F97D7FF1F23A9074697D70B
:10887000FF1F23A7074697D7FF1F23A50746EFE053
:108880009033EF40C002EFE0F00AEFE0700F97D7AF
:10889000FF1F938727439C4381C70545EF60B03393
:1088A00097D7FF1F9387C72B9C4389C741657D15C9
:1088B000EF50A06BEFC0703AEFA0F00097D7FF1F0A
:1088C0009387C7569C431397170163540700EFC063
:1088D000A04597D7FF1F23AF074897D7FF1F23ADAA
:1088E000074897D7FF1F23AB074897D7FF1F23A938
:1088F0000748EFF09F984923EFF0AFBBEFC08067C8
:108900006F90FF94828097D7FF1F9387273D8843FE
:108910008280EF929F91EF60B07EEF7080006F9049
:108920001F93EF92FF8E2A849304140201112E8567
:10893000B289A685214636C63A89EF0081611DE1DC
:10894000B24638082686CE8513059404EF4060436E
:1089500021462C084A85EF00C15F133515000561DB
:108960006F905F8E0145E5BFEF923F8C9305450602
:1089700017D5FF1F1305C513EFE070226F903F8DD1
:10898000EF92BF8A41112EC6EFF00FC0B24588C1E9
:1089900041016F90DF8BEF92BF87AA842E84EF6036
:1089A0005078AA8985452285892D83C7E4011389DA
:1089B000940899E313890403CE8522853D2D214631
:1089C000930519022285192D97D7FF1F9387073129
:1089D0008C432285EF00E06821469385840222853E
:1089E000F52B6F903F86EF92DF813971EFC0E04E3B
:1089F0009305400645EDEF60D06F630E051097D7E5
:108A0000FF1F83C7A70C13B7170097D6FF1F238F2D
:108A1000E60A014489CFC16417D9FF1F1309092C45
:108A20009309400EFD14EFF03F986348A408EFF05F
:108A3000AFB54169B7290900096AFD7A2A8B8144DB
:108A40007D199389F97B130A0A71938A8AC7EFF01B
:108A5000BF9563D5A4041304400EB387840217D7CF
:108A6000FF1F1307A7270324070B3E948357C40156
:108A70006386270918403307EB4063EAE900834720
:108A800044008507B3874703D6976369F706014615
:108A900081450945EFF0CFE8AA8B29E1EF20105A74
:108AA0008547631FF50489659385057117D5FF1FF9
:108AB00013050500EFE0B00EA1A8B30734030327A8
:108AC000090BBA9703D7C7016308970003C757007C
:108AD000A38207002382E7000504B1B79305C50010
:108AE0002285EFF05FEB5E85228697350100938546
:108AF000E500EFF0CFEB5E85EF00E06F850481BF0E
:108B000097D7FF1F9387871D9C478D83858BC1FF58
:108B100021616F908FF201468545094502D002D24E
:108B200002D402D6EFF0CFDFAA847DD1EFC0203A85
:108B30001389C4002A8481454A85C1210C404146DD
:108B40004A85692983294400638809084E8502D82B
:108B500002DA02DC02DEEF0081692ACE141005463B
:108B60002C0808184ECCEF4060191375F50F2DE551
:108B70008355840093E525004A856D2911460C1024
:108B80004A85A9290146973501009385A5F72685D1
:108B9000EFF0EFE12685EF0000665C40B5DB0146B3
:108BA00085450D45EFF0CFD7AA843DD148401389C4
:108BB000C400EF00C1632AC64A85C5263246636AEF
:108BC000C5004C404A851929014681452685EFF0AC
:108BD0000FDE26850D252DBF8355840071BFEF92D2
:108BE000CFE497D7FF1F9387670F9C4719CD93E773
:108BF000870017D5FF1F1305A5EB17D7FF1F2323EA
:108C0000F70EEFE060786F908FE4DD9B17D7FF1FC2
:108C1000232AF70CEF2090427DF517D5FF1F13058F
:108C200025E9EFE04079C5B7EF92AFDD4169AA8948
:108C30002E8AB28A368BBA8B814417DCFF1F130C45
:108C4000EC09930C400E7D19EFF00FF663C4A400FD
:108C500001442DA03384940383270C0B3E94835747
:108C6000C401638027055A87D6865286CE851305B0
:108C70000403EFF01FCB11C523800B0022856F90FA
:108C8000CFDB8347F40191CF5A87D6865286CE85B3
:108C900013059408EFF0FFC809C585472380FB0042
:108CA000F1BF850455B783574500638D0716EF92D2
:108CB0002FD601112A84ED2619C58547630AF504CC
:108CC00005616F902FD8EFC040217DF98357440094
:108CD0004947ED9BE396E7FEC14522854524AA84DA
:108CE0002285F52E0357440002CE91472A89631747
:108CF000F700228539293C082ACC3ECEEFC0201D42
:108D00005C55DDDF74084A86A685054582974DBF10
:108D100003574400D147E3F5E7FA032A0400C16989
:108D2000014997DAFF1F938A6AFB130B400EFD1966
:108D3000EFF08FE76344A90C2285032A04008D26F7
:108D4000A1452A8922851D2CAA842285D926144072
:108D50002A86AA8978082685CA85EFF0FFECAA84BE
:108D600025D103C7F40189476315F7008347C10183
:108D7000A1DB5546D28513856400EF00E11F014554
:108D8000EF60103801C583D7C401B1EB97D7FF1F3F
:108D90009387C7F49C4793551900858913D73700EB
:108DA000058B11CB8983858B6397B70001452EC650
:108DB000EFF0FFE2B2454E85EF60703C0346C10123
:108DC0002A84937519002685EF70703131C9268584
:108DD000EF607037268511C00145EF60D061EF204C
:108DE000F0258547E31EF5EC83C754001307F00F09
:108DF000E388E7EC8507A382F400D9B5B3046903DF
:108E000083A70A0BBE9483D7C401638937015546F3
:108E1000D28513856400EF00C11371D1050909BF24
:108E20005DDC5DBF8280EF92AFBEEF60902C11CD14
:108E3000C164014417D9FF1F130949EA9309400E81
:108E4000FD14EFF06FD6634AA40017D5FF1F13057A
:108E500025C6EFE060536F90EFBE330534038327E0
:108E6000090B3E958357C5016386970023120500C1
:108E7000EF60702D0504F1B797D7FF1F938707E6C2
:108E80009C478D83858B99EBEF922FBA17D5FF1FE7
:108E9000130505C2EFE020526F906FBB8280EF9206
:108EA000CFB897050000938545B417D5FF1F13056C
:108EB00025C0EFE0A0426F908FB9EF920FB78841C5
:108EC000B7E70400BC5B050542054181829709C5EF
:108ED00085472300F50005056F906FB783C7F5FF41
:108EE0002E858507A38FF5FE828083C7F5FFFD17CA
:108EF00093F7F70FA38FF5FE99EBEF920FB3B7E758
:108F00000400BC571385F5FF82976F904FB48280A1
:108F10001C41035745008D8FBA951CC12312B50023
:108F20003E85828093D78500A2051441DD8D83574D
:108F300045001387E6FF18C189072312F50013D6F1
:108F400085004111238FB6FEA38FC6FE41018280AA
:108F500018419307F7FF1CC183574500850723126B
:108F6000F500A30FB7FE8280835745008D8F231233
:108F7000F5001C41BE950CC12E858280AA8703D7BF
:108F8000470008410D8FAA952392E7008CC3828089
:108F9000184108453305A740828083574500035791
:108FA00065001D8F1C4108453385A7403305A74048
:108FB0008280EF928FA741112EC62A84EFF0FFFD29
:108FC000B2456373B50001A0835744000840BE95C5
:108FD0002312B4003E9541016F906FA7EF92EFA46A
:108FE00041112E84B28532C6EFF0BFFC3246A28515
:108FF000EFF0907841016F908FA5EF920FA32E8430
:109000008545EFF01FFB230085006F904FA4EF9282
:10901000CFA141112317B1008945EFF09FF9834794
:10902000E1002300F5008347F100A300F5004101B2
:109030006F90EFA1EF926F9F93D78500A20541112A
:10904000DD8D2317B1008945EFF0BFF68347E100BE
:109050002300F5008347F100A300F50041016F9064
:109060000F9FEF928F9C1397850193D78501C1665F
:10907000938606F0D98F13D78500758FD98FA205F7
:109080003707FF00F98D4111DD8D2EC69145EFF0B8
:109090005FF26C001146EFF0306E41016F902F9B34
:1090A000EF92AF981C41854503C40700EFF0DFEB5A
:1090B00022856F90CF99EF924F971C4141118945BE
:1090C00003C7070083C717002307E100A307F100C8
:1090D000EFF09FE90355E10041016F904F97EF9248
:1090E000CF941C414111894503C7070083C717006E
:1090F0002307E100A307F100EFF01FE78357E1002A
:10910000410113D58700A2075D8D420541816F9013
:109110000F94EF928F910C4141112A8411466800FF
:10912000EFF0906591452285EFF01FE4B247C166EC
:10913000938606F01397870113D58701598D13D7AE
:109140008700758F598DA2073707FF00F98F5D8D56
:1091500041016F90CF8F1C45BE950CC18280AE87B8
:10916000944391E6584101EF0CC15CC1828003C772
:10917000570013671700A382E700B687D5B70CC363
:10918000EDB7AA87084119CD1841D44398C363139A
:10919000D500D8C32A87034657009376160081E688
:1091A000232007008280944381CA8C4203A8470091
:1091B0008CC363930601CCC3799A14C3A302C7007E
:1091C0003687D1BF1C45DC471D8DB777DBB693874B
:1091D00077DB09853305F502420541818280F1473D
:1091E000B385F50248452E95828083474500850763
:1091F0002302F5008280EF924F832A8419E06F905A
:109200000F8583474400E5DFFD1793F7F70F23022F
:10921000F400F5F71C4403D7270005072391E70066
:10922000DC4399C3228582974C4889CD83475400FB
:10923000898B99E71C4422859C479C439C478297D5
:10924000232A04000040232004004DBFEF82FFFDCD
:109250008357250041112EC691E701442285410123
:109260006F80FFFE035705008147F146E307F7FED5
:10927000B385D702404585072E948345440008C432
:10928000F5F5B247AA8481E7232A040009A81C4502
:109290006C0022859C439C43829748C85DDD8547CE
:1092A0002312F400B24723200400231804002319DA
:1092B000F4005C485CC483D72400FD172391F400BC
:1092C00071BFEF829FF697D7FF1F93876780884310
:1092D00023260500232405004105EFE0C00D6F8023
:1092E0001FF7EF829FF417C4FF1F1304647E1C4016
:1092F000411189CF9C472300B5002AC65CC1EFF01D
:109300005FFC1C40DC4399C33245829741016F806A
:109310001FF4034745001DEB584DAA877D550DCB23
:10932000EF82BFF01CC3DC4797C6FF1F23A2E67A7B
:10933000F156130507012390D70097050000938588
:109340008501EFD0B07901456F807FF07D55828037
:109350008280EF829FED0111614681452800EF80F8
:10936000DFEF97C7FF1F9387A7769C4328009305DD
:10937000F00FDC473EC6EFF0DFF605616F803FED92
:1093800097C7FF1F9387C7749C43D847A1679387EC
:10939000C7026312F70A397106DE22DC26DA800082
:1093A0004AD84ED652D456D23285B284EFF05FCF2F
:1093B000AA892685EFF03FD02318A4FC2685EFF07C
:1093C0009FCF2319A4FC2685EFF0FFCE83D744005E
:1093D0000A8A231AA4FC858393F7F70F230EF4FC63
:1093E0008607BD0793F7073F3301F1408A8A014999
:1093F0008347C4FD6365F902CE85130584FC232CE5
:1094000054FDEFF01FEE5281130104FCF250625440
:10941000D2544259B259225A925A216182802685E9
:10942000EFF07FC993171900D69705092390A7007D
:109430001379F90F75BF828097C7FF1F938747691C
:109440009C43D847A1679387A7026310F70A397135
:1094500006DE22DC26DA80004AD84ED652D456D216
:109460003285B284EFF0DFC3AA892685EFF0BFC44E
:10947000FD572318A4FC26852319F4FCEFF0BFC385
:1094800083D744000A8A231AA4FC858393F7F70F35
:10949000230EF4FC8607BD0793F7073F3301F14025
:1094A0008A8A01498347C4FD6365F902CE851305A5
:1094B00084FC232C54FDEFF0DFE25281130104FC05
:1094C000F2506254D2544259B259225A925A2161EE
:1094D00082802685EFF03FBE93171900D6970509C5
:1094E0002390A7001379F90F75BF828097C7FF1FDC
:1094F0009387075E9C43D847A16789076318F708DD
:10950000397106DE22DC26DA80004AD84ED652D4E3
:1095100056D232853289EFF0BFB8AA894A85EFF07A
:109520009FB9835749000A8A2318A4FC858393F7BF
:10953000F70F230CF4FC8607BD0793F7073F3301B1
:10954000F1408A8A8144834784FD63E5F402CE8535
:10955000130584FC232A54FDEFF0BFD85281130178
:1095600004FCF2506254D2544259B259225A925ACF
:10957000216182804A85EFF01FB493971400D6973B
:1095800085042390A70093F4F40F75BF828097C7DA
:10959000FF1F9387E7539C43D847A1679387E7044E
:1095A0006312F70A397106DE22DC26DA80004AD817
:1095B0004ED652D456D23285B284EFF07FAEAA890D
:1095C0002685EFF05FAF2318A4FC2685EFF0BFAE31
:1095D000231AA4FC2685EFF01FAE83D744000A8A25
:1095E0002319A4FC858393F7F70F230EF4FC860759
:1095F000BD0793F7073F3301F1408A8A014983474A
:10960000C4FD6365F902CE85130584FC232C54FD4B
:10961000EFF03FCD5281130104FCF2506254D2545A
:109620004259B259225A925A216182802685EFF01E
:109630009FA893171900D69705092390A7001379BF
:10964000F90F75BF828097C7FF1F938767489C43B8
:10965000D847A1679387C7046310F70A397106DEFC
:1096600022DC26DA80004AD84ED652D456D2328531
:10967000B284EFF0FFA2AA892685EFF0DFA3FD57A1
:109680002318A4FC2685231AF4FCEFF0DFA283D76D
:1096900044000A8A2319A4FC858393F7F70F230E4D
:1096A000F4FC8607BD0793F7073F3301F1408A8A30
:1096B00001498347C4FD6365F902CE85130584FC27
:1096C000232C54FDEFF0FFC15281130104FCF25032
:1096D0006254D2544259B259225A925A216182801C
:1096E0002685EFF05F9D93171900D6970509239003
:1096F000A7001379F90F75BF828097C7FF1F938763
:10970000273D9C43D847A167DD07631BF702EF8223
:10971000DFB1797132853284EFF09F982AC62285B5
:10972000EFF07F992311A1022285EFF07F97B245D8
:109730002300A1022808EFF0DFBA45616F803FB136
:10974000828097C7FF1F9387A7389C43D847A1679C
:1097500093878704631BF702EF823FAD79713285EF
:109760003284EFF0FF932AC62285EFF0DF942311B5
:10977000A1022285EFF0DF92B2452300A102280862
:10978000EFF03FB645616F809FAC828097C7FF1FA7
:10979000938707349C43D847A1679387A704631C2A
:1097A000F700EF829FA8011128008145EFF07FB3F9
:1097B00005616F80DFA9828097C7FF1F93874731BC
:1097C0009C43D847A167938757026311F702EF8242
:1097D000DFA501113285EFF0BF8C2308A100814580
:1097E0002800EFF01FB005616F807FA6828097C7C9
:1097F000FF1F9387E72D9C43D847A1679387E70214
:10980000631FF702EF827FA2011132853284EFF0ED
:109810009F8AAA842285EFF01F8A854719E5228551
:10982000EFF01F884205B337A000280081452318B8
:1098300091003ECAEFF0FFAA05616F805FA18280B0
:1098400097C7FF1F9387C7289C43D8479947631F33
:10985000F704EF829F9D797132853284EFF05F8447
:109860002AC62285EFF03F852310A1022285EFF062
:109870003F832301A1022285EFF09F82A301A10271
:109880002285EFF0FF812302A1022285EFF05F81A4
:109890002313A1022285EFF0BF80B2452314A10259
:1098A0002808EFF01FA445616F807F9A828097C7D8
:1098B000FF1F9387E7219C43D847A1679387C7037E
:1098C000631FF704EF827F96797132853284EFF05F
:1098D0002FFD2AC62285EFF00FFE2310A10222855C
:1098E000EFF06FFD2311A1022285EFF06FFB230241
:1098F000A1022285EFF0CFFAA302A1022285EFF0A8
:109900002FFA2303A1022285EFF08FF9B245A303BA
:10991000A1022808EFF0FF9C45616F805F93828071
:10992000EF82BF9001112A84EFF08FF7AA8422857D
:10993000EFF06FF82285EFF00FF8035744008D47E2
:1099400063F5E7002285EFF00FF72285EFF0AFF621
:109950002800A685EFF0FF9805616F805F8F97C79D
:10996000FF1F9387E7169C43D847A167FD0763193C
:10997000F700EF829F8B3285EFF09FFA6F803F8D6B
:10998000828097C7FF1F9387A7149C43D847A1677E
:10999000E5076311F706EF825F89797132853284BA
:1099A000EFF00FF02AC62285EFF0EFF02285EFF0FE
:1099B0008FF02310A1022285EFF0EFEF52055181C5
:1099C0002311A102228523020102EFF06FEDA30211
:1099D000A1022285EFF0CFEC2303A1022285EFF054
:1099E0002FECB245A303A1022808EFF09F8F456139
:1099F0006F80FF85828097C7FF1F9387670D9C4309
:109A0000D847A1679387E7036319F700EF82FF81C7
:109A10003285EFF0FFF06F809F83828097C7FF1F32
:109A20009387070B9C43D847A16793874704631428
:109A3000F702EF828FFF797132853284EFF04FE6C3
:109A40002AC62285EFF02FE7B2452808EFF07F897C
:109A500045616F80CFFF828097C7FF1F93874707BD
:109A60009C43D847A167938787026316F702EF826A
:109A7000CFFB797132853284EFF08FE22AC62285DE
:109A8000EFF00FE2B2452300A1022808EFF07F8536
:109A900045616F80CFFB8280EF822FF90111EFF0DB
:109AA0002FE0AA852800EFF0DF8305616F802FFA91
:109AB00097C7FF1F9387C7019C43D847A167D1076A
:109AC0006319F700EF826FF63285EFF0FFFC6F80CD
:109AD0000FF8828097C7FF1F938787FF9C43D84763
:109AE000A167C5076319F700EF822FF43285EFF005
:109AF000BFFA6F80CFF5828097C7FF1F938747FD1E
:109B00009C43D847A167B9076319F700EF82EFF1CB
:109B10003285EFF07FF86F808FF3828097C7FF1F49
:109B2000938707FB9C43D847A167AD076319F700EC
:109B3000EF82AFEF3285EFF03FF66F804FF182801A
:109B400097C7FF1F9387C7F89C43D847894763107F
:109B5000F702EF828FED0111328532C8EFF04FD45A
:109B6000AA852800EFF0EFF705616F804FEE828045
:109B700097C7FF1F9387C7F59C43D847A1678D07F9
:109B80006317F702EF826FEA011132853284EFF03A
:109B90002FD113066100AA844C002285EF20D00C3F
:109BA0002800A685EFF0EFF305616F804FEA828011
:109BB00097C7FF1F938707F29C4381CBDC4391C774
:109BC000EF82AFE682976F808FE88280EF82EFE5C9
:109BD00079713C08AE843ED2A165B7070A002A8499
:109BE0003ED448103C08DD053ED636C432C63AC2E3
:109BF000EFD0BFAA12474810BA85EFF00FC0324627
:109C00004810B285EFF0AFC0A2464810B685EFF01D
:109C1000CFBE501001478146A6852285EFD07FC870
:109C200045616F80CFE2EF824FE001117C00032994
:109C3000C501AE843ECAA165B70707002A843ECCA1
:109C400048087C00C5053ECEEFD03FA58345D9002E
:109C50004808EFF08FBA500801478146A685228553
:109C6000EFD03FC405616F808FDEEF820FDC83C7CA
:109C7000950093F7F707A384F500EFF0DFFA6F8004
:109C80000FDDEF828FDA79713C08AE843ED2A16598
:109C9000B70709002A843ED448103C089385450440
:109CA0003ED632C636C4EFD05F9FA2464810B68576
:109CB000EFF0AFB432464810B285EFF04FB5501018
:109CC00001478146A6852285EFD0BFBD45616F80E3
:109CD0000FD8EF828FD583C7950041112A8493F75F
:109CE000F707A384F50032852EC6EFF0CFBC856759
:109CF0002AC4637CF500EF50B0402246B24509E922
:109D0000114781462285EFF07FEC41016F802FD40F
:109D100001478346F501FDB7EF828FCF01113C006B
:109D20003ECAB7070A003ECC3C003ECE83C7950032
:109D3000AA89328593F7F707A384F5002E84EFF004
:109D40008FB785676371F504A165AA84938585043F
:109D50004808EFD09F942685EF50903A2A891DE558
:109D600091454808EFF06FA9A6854808EFF02FAAA3
:109D7000CA854808EFF06FA8014781465008A285C0
:109D80004E85EFD01FB205616F80CFCB814548086B
:109D9000EFF0AFA603490902C1BFEF826FC7797127
:109DA0001C103ECAB7070F003ECC404D1C10AA84C1
:109DB000AE894808994532C636893ECEEFD0FF8D30
:109DC00032464808B285EFF04FA363040902A54567
:109DD0004808EFF00F9E2546CA85EFF0E0195008BD
:109DE00001478146CE852685EFD0BFAB45616F80A8
:109DF0006FC58355C4024808EFF06FA10355E40214
:109E0000814515C185478545630FF500C167FD177D
:109E10009305F00F6309F5007D15EF50207493054D
:109E2000150093F5F50F4808EFF02F9D83450403C7
:109E30004808EFF08F9C834514034808EFF0EF9B30
:109E4000835524034808EFF08F9C8355440348084A
:109E5000EFF0EF9B69B7EF824FBD83C79500814656
:109E6000014693F7F707A384F500EFF01FF36F8027
:109E70000FBEEF828FBB79713E841C103ECA2E89C3
:109E8000B7070F00A1653ECCFD051C10AA84480849
:109E900042C03AC23ECE36C432C6EFD01F803246F0
:109EA0004808B285EFF06F95A2464808B685EFF0F6
:109EB0000F9612474808BA85EFF06F950248630481
:109EC000080291454808EFF0CF8E1146A285EFF0C9
:109ED000A00A500801478146CA852685EFD07F9C9D
:109EE00045616F80CFB689454808EFF08F8C834776
:109EF00004002300F50083471400A300F500D1BF40
:109F0000EF820FB183C7950001112A8A93F7F707F3
:109F1000A384F5003285AE8432C6EFF0CF99324685
:109F20002A893285EFF0CF978567637FF900AA8988
:109F30004A85EF50F01C2A8419E9114781464A8668
:109F4000A6855285EFF09FC805616F80AFAF9387FC
:109F5000E9FF93F7F70F0547E368F7FE8347F5013D
:109F600095E78947E382F9FE8346F401528501476C
:109F70004A86A685EFF09FC5A167D90748083ECC61
:109F8000230A010002CEEFF0BFC27DBF639CE70051
:109F90008947639CF90093071020231FF500EF50B9
:109FA000901AD9B70947E391E7FC8D47E39EF9FA88
:109FB0002285EF50D03B97C7FF1F9387A7D09C43C4
:109FC00099E797C7FF1F9387A7B99C4389C703D514
:109FD0000400EF60300C231F04002285C9B7EF8214
:109FE000CFA401113C003ECAB7070B003ECC3C0099
:109FF0003ECE83C795002A89328593F7F707A3845D
:10A00000F500AE84EFF02F8B93170501C187635ED7
:10A01000F004A1652A849385E5024808EFD0EFE7B4
:10A02000A2854808EFE0BFFE97C7FF1F938747B39D
:10A030009C439DEF01449375F40F4808EFE0FFFB4C
:10A040009355844093F5F50F4808EFE01FFB9355B7
:10A05000044193F5F50F4808EFE03FFA01478146C8
:10A060005008A6854A85EFD0DF8305616F802F9E5B
:10A07000416585460546A2857D15EF3070675DD93F
:10A080005105EFD04027130440063344850265B7DD
:10A09000EF82AF990111B70706003EC683C795004E
:10A0A00021642A8993F7F707A384F500AE8428007A
:10A0B0009305A4040AC40AC8EFD02FDE300001477C
:10A0C0008146A6854A85EFD0CFFDEFE02FF8130437
:10A0D0009404480822CC230A010002CEEFF05FADC1
:10A0E00005616F80CF96EF82AF92C1642A890144E7
:10A0F00097C9FF1F938989BE130A8002FD14EFE000
:10A10000AFAB6345A40001456F80CF93B307440311
:10A1100003A7C90ABA9703D707006306970083D736
:10A120002700638427010504D9BF0545F1BFEF82ED
:10A130002F8E2A8A2E8999C123A005008149814446
:10A1400097CAFF1F938A4A99614BEFE02FAD63C511
:10A15000A4004E856F800F8F3384640383A70A00A9
:10A160003E948357040099E7630409002320890083
:10A170008504E1BF4146D28513054400EFE0705DE0
:10A1800065F9A289F5B7EF82AF8839717C083ED4B2
:10A19000B7070A003ED67C083ED883C795002A8AB6
:10A1A000328593F7F707A384F5002E8932C6EFE0D6
:10A1B0009FF085676373F5063246AA843285EFE027
:10A1C0003FEE8547AA8963EAA704A16593858504C4
:10A1D0002810EFD08FCC2685EF5080722A8429E199
:10A1E00091452810EFE07FE1A6852810EFE03FE2DF
:10A1F000CE852810EFE07FE0014781463010CA8508
:10A200005285EFD00FEAA1679387770448183EDCA8
:10A21000230A010202DEEFF0BF9921616F808F8275
:10A2200081452810EFE07FDDA6852810EFE03FDEB6
:10A2300097C7FF1F938747E19C4391C72285638798
:10A240000900EFB0600C8345040265B7EFB0200B46
:10A25000DDBFEF72FFFB83C795004111AA8993F719
:10A26000F707A384F5003285AE84328AEFE0BFE4BD
:10A270008567637BF5022A89EF5080682A849146BE
:10A2800021C18347F50105476383E70291C70D4765
:10A29000636EF702AD462DA09305050303250A0062
:10A2A0004146EFE0104B1DE141016F70BFF993058E
:10A2B000950803250A004146EFE0B049814679F947
:10A2C0004A86A6854E85EFF0DF9BF9BF83250A00FD
:10A2D00013059408EF60600119C1C146D5B797C74F
:10A2E000FF1F9387279E9C4399E797C7FF1F93877C
:10A2F00027879C4389C72285EF60A05479FD854755
:10A30000A30FF4002285EF80B05D2285EF50A0639B
:10A310004E8581464A86A685EFF0BF96A167938752
:10A32000570448003EC42302010002C6EFF05F88D4
:10A33000A5BFEF721FED83C795004111AA8993F75E
:10A34000F707A384F50032852E89B28AEFE0BFD6E5
:10A3500085676370F50CAA84EF50805A2A841DE942
:10A36000416B014A97CBFF1F938B4B97130C400E09
:10A370007D1B19A833048A0383A70B0B3E948357D4
:10A38000C401638D6703050AEFE00F82E344AAFE70
:10A39000954639A88357C501639297029305050333
:10A3A00003A50A004146EFE0D03A994611E1814603
:10A3B0002686CA854E85EFF0DF8CA1A883A50A000A
:10A3C00013050403EF507072C1467DF12285231EF0
:10A3D0009400EF80F0502285EF50E05697C7FF1FA2
:10A3E000938787C69C438DCB230004022285EFA070
:10A3F00090614E8581462686CA85EFF09F88A167C9
:10A400009387070448003EC42302010002C6EFF010
:10A410002FFA41016F707FE289472300F402D1BF18
:10A42000397106DE22DC4AD8800052D456D25AD086
:10A4300026DA4ED65ECE2E8A32892A8BEFD0DFF313
:10A440000605710541998A8A3301A140232224FC23
:10A45000231404FCEFD05FF283479A00060535050C
:10A4600093F7F7072315A4FCA304FA004A852326D3
:10A4700024FCEFE05FC493170501C1876340F0023D
:10A480005681130104FCF2506254D2544259B2591D
:10A49000225A925A025BF24B21618280AA844A8539
:10A4A000EFE07FC1AA894A85EFE0FFC0A1659385EF
:10A4B000C5022A89130544FCEFD02F9E2685EFD0D4
:10A4C000AF93854501C94A86CE85EFD06F8DAA8BA3
:10A4D00015ED8945130544FCEFE03FB2A685130551
:10A4E00044FCEFE0DFB2CE85130544FCEFE03FB261
:10A4F000CA85130544FCEFE09FB10147814613066E
:10A5000044FCD2855A85EFD0CFB99DBF8145130554
:10A5100044FCEFE09FAEA685130544FCEFE03FAF9F
:10A52000CE85130544FCEFE09FAECA85130544FCBD
:10A53000EFE0FFAD8144EFD03FE4E3D0A4FC83A77C
:10A540000B0113971400BA9783D5070089C513052B
:10A5500044FCEFE0DFAB8504F9BF797106D622D465
:10A560004AD000184ECE52CC56CA26D25AC8AE890E
:10A570003289AA8AEFD05FE00605690541990A8A07
:10A580003301A140232A24FC231C04FCEFD0DFDE8E
:10A5900083C7990006052D0593F7F707231DA4FC33
:10A5A000A384F9004A85232E24FCEFE0DFB0931743
:10A5B0000501C187634FF0005281130104FDB250C1
:10A5C000225492540259F249624AD24A424B45619E
:10A5D0008280AA844A85EFE01FAEA1659385A5021B
:10A5E0002A89130544FDEFD04F8B2685EFD0CF800D
:10A5F000854519C5CA85EFC0BFFD2A8B0DE9894580
:10A60000130544FDEFE07F9FA685130544FDEFE0B1
:10A610001FA0CA85130544FDEFE07F9F01478146D7
:10A62000130644FDCE855685EFD0AFA771B781459F
:10A63000130544FDEFE07F9CA685130544FDEFE084
:10A640001F9DCA85130544FDEFE07F9C8144EFD038
:10A65000BFD2E3D5A4FC83270B0113971400BA974C
:10A6600083D5070089C5130544FDEFE05F9A850493
:10A67000F9BFEF729FBB83474500404DD5E7FD57BB
:10A680004DC0834694000947636DD7080346B40064
:10A69000854663E8C6088306E40063C406085C4593
:10A6A000F9562390D70097B7FF1F83C7274399E335
:10A6B000A304E40097B7FF1F9387874A9C4381E771
:10A6C0008947A306F40097C7FF1F9387E7979C432A
:10A6D00081E789472306F400970500009385450527
:10A6E000AA8413050401EFC0703FFD57231AF4023A
:10A6F00081471CDC014897B7FF1F23AD873C97B704
:10A70000FF1F9387673D232E040304C08043EFD0CF
:10A71000FFD061463306C50281452285EF70FFB345
:10A7200081473E856F70BFB2FD57E5BFEF72FFAF47
:10A730002A8403554502EF50A01C09E5231E04009E
:10A740006F70FFB08357E401E5DF930504FF171531
:10A7500001001305E574EFB01063DDB7EF72FFACD5
:10A760002E89A16541119385E5032A8436C432C63A
:10A77000BE843AC2EFC07FF212472285BA85EFE06D
:10A78000DF8732462285B285EFE07F88A2462285A8
:10A79000B685EFE0DF87630D090091452285EFE084
:10A7A0005F811146A685EFE0207D41016F703FAAD1
:10A7B00089452285EFE0EFFF83C704002300F50001
:10A7C00083C71400A300F500CDB7EF721FA683C79F
:10A7D0009500444D054793F7F707A384F5001C4205
:10A7E000411183C70700636DF7042E842A8985CC45
:10A7F00003C7D4006309F70217B7FF1F13074736D3
:10A80000184301CFA386F400EF80902B83C7D400B8
:10A8100089E741657D15EF30407583D72403918B1F
:10A8200099C3EFB0B0624A85A285EFF0CFBFA167B0
:10A83000C10748003EC42302010002C6EFF04FB733
:10A8400041016F70DFA0EF725F9E03D745008D4717
:10A85000AA8441112E8432892E8563EDE700EFE052
:10A860009F85AA85230009002685EFC07FD6410178
:10A870006F70FF9DEFE03F842AC62285EFE0BF8323
:10A88000B24585472A862300F9002685EFC05FD1AF
:10A89000F9BF397106DE22DC26DA80004ED652D4AA
:10A8A00056D24AD85AD05ECEAE89B284AA8AEFD0A8
:10A8B000BFAB06051305250241990A8A3301A14061
:10A8C000232224FC231404FCEFD01FAA83C7990081
:10A8D00006054D0593F7F7072315A4FCA384F9009B
:10A8E0002685232624FCEFE00FFD93170501C18781
:10A8F0006340F0025281130104FCF2506254D254BE
:10A900004259B259225A925A025BF24B216182801B
:10A91000AA8B03AB0400EFC03FCE35E983D74400D8
:10A9200001498544F11793B71700A301F4FC83474D
:10A9300034FCA165BDC79385E504130544FCEFC055
:10A94000DFD5A685130544FCEFE02FEBDE8513056C
:10A9500044FCEFE0CFEB834734FC114691E309461A
:10A96000DA85130544FCEFE06FE7814463080900D2
:10A97000416B7D1BEFD05F9F63C8A40201478146F6
:10A98000130644FCCE855685EFC0BFF1A5B7A6855A
:10A99000130634FCEFF03FEB933415002A8986044C
:10A9A00079B79385C50451BF8327C9001397140055
:10A9B000BA9783D5070063866501130544FCEFE071
:10A9C0000FE5850445BFEF72DF8379711C103EC42B
:10A9D000B7070F003EC61C103EC883C79500AA8A61
:10A9E000328593F7F707A384F500AE893284EFE050
:10A9F0008FEC93170501C1876350F0062A8A2285E0
:10AA0000EFE06FEB2A895285032B0400EFC0DFBE15
:10AA100039E58357440081440544F11793B7170083
:10AA2000A303F10083457100DA872287CA86528624
:10AA30002800EFF0BFD2014781463000CE85568511
:10AA4000EFC03FE6A1679387D70348083ECC230AAF
:10AA5000810026CEEFF0CF9545616F700FFEA28585
:10AA600013067100EFF03FDEAA84094445DD35444A
:10AA7000E30A55FB4A85EFF00FE70D4445D5014445
:10AA8000EFD09F8E634BA400C16B0144FD1BEFD040
:10AA9000BF8D634EA400154471B7DC441317140036
:10AAA000BA9783D70700638127030504D1BFD84431
:10AAB00093171400BA9703D70700631977012390FF
:10AAC00027012685EF80C0540144A9BF0504C1B702
:10AAD000EF720FF483C7950041112A8A93F7F707A5
:10AAE000A384F50032852E893284EFE0CFDC931702
:10AAF0000501C187635BF004AA892285EFE0AFDB23
:10AB00002311A1004E85832A0400EFC0FFAE29E186
:10AB10008357440085440144F11793B71700A300FD
:10AB2000F1000348110003572100D6875285CE86D5
:10AB30002686CA85EFF0EFB3A167F10748003EC44F
:10AB40002302910022C6EFF0AF8641016F708FEFB4
:10AB5000A28513061100EFF01FCF2A84894471D11A
:10AB60008357210011678544BA97C2071167C183D3
:10AB70001307F7EFE367F7FA97B7FF1F9387871479
:10AB80009C4391C7854513052100EF40300E835546
:10AB9000210022858144EFC09F9D41D523100500EF
:10ABA0002285EF808048B5BFEF72AFE583C795007F
:10ABB00041112A8B93F7F707A384F50032852E8A7B
:10ABC0003284EFE04FCF93170501C1876359F0043A
:10ABD000AA8A2285EFE02FCE2A895685832B04008E
:10ABE000EFC09FA121E18357440081440544F11740
:10ABF00093B71700A301F10003483100DE875A859F
:10AC00004A87D6862286D285EFF0AFA6A167ED07E8
:10AC100048003EC42302810026C6EFE07FF94101CF
:10AC20006F70AFE1A28513063100EFF0DFC1AA8497
:10AC3000094479D19167CA97C2071167C183130785
:10AC4000F7EF0544E36AF7FACA85EFC05F92014463
:10AC500045F58149EFD04FF263DBA90098489397FF
:10AC60001900BA9703D7070015E723902701EFD003
:10AC7000AFF01544E382A9F82685EF80003B97B733
:10AC8000FF1F938727049C430144BDD74A85EF40AB
:10AC900040769DB785097DBFEF728FD779713E846D
:10ACA0007C083EC82E8AB7071400A1653ECAE50598
:10ACB0007C08AA89080836C4428932C6BA8AC68482
:10ACC0003ECCEFC09F9DCA850808EFE00FB3324627
:10ACD0000808B285EFE0AFB3A246630E09029D45B6
:10ACE0000808EFE00FAD1D468145EF700FD7638771
:10ACF0000A0691450808EFE0CFAB1146A685EFE0C4
:10AD0000A027100801478146D2854E85EFC07FB944
:10AD100045616F702FD3B6850808EFE04FAF1C4038
:10AD20000808D8439355C701858912075183B20596
:10AD3000D98DEFE0CFAD1C40080883C58700EFE058
:10AD4000CFAB1C40080883C5A700EFE00FAB1C4049
:10AD5000080883C59700EFE04FAA51BF894508084E
:10AD6000EFE02FA583C704002300F50083C714007C
:10AD7000A300F50079B7EF72AFC983C79500411101
:10AD8000AA8993F7F707A384F5003285AE8432844D
:10AD9000EFE06FB293170501C1876357F0042A896A
:10ADA000032A0400EFC05F8519E983574400054872
:10ADB000F11793B71700A307F100814621A81306E6
:10ADC000F100A285EFF03FA81DC11C459DC383D6AD
:10ADD000470001480347F10093078500D2884A865F
:10ADE000A6854E85EFF05FEB41016F70AFC5094856
:10ADF000E9B71D48D9B7EF72AFC165715C083EC4B1
:10AE0000B7077B013EC65C083EC883C795002A8A07
:10AE1000328593F7F707A384F500AE89EFE04FA8DA
:10AE20008357E100C5C389452800EFC01F878145CE
:10AE30002800EFE08F9CEFC0FF8B97B7FF1F938731
:10AE4000A7209C4317B4FF1F034444C9AA8433348A
:10AE5000800099C31364240097B7FF1F938747D0DE
:10AE60009C4399C31364440097B7FF1F938787E5FA
:10AE70009C4399C31364840083D5040028000149CE
:10AE8000EFE0EF9883D524002800EFE04F9883D5BA
:10AE900044002800EFE0AF97EFD00FC993150501EC
:10AEA000C1812800EFE0AF96A2852800EFE02F9641
:10AEB0009C44636CF900014781463000CE85528581
:10AEC000EFC03F9E59616F70EFB7DC441314490027
:10AED00028003E94EFE06F8C834744000347540002
:10AEE00089070607BA978607E36EF5FC83552400A9
:10AEF0002800814AEFE0AF91834544002800EFE04D
:10AF0000CF8F834554002800EFE02F8F8347440004
:10AF100063C9FA00814A8347540063CFFA000509E8
:10AF200041BF1C4413975A002800BA9783D50700E5
:10AF3000850AEFE0CF8DD9BF032BC40093975A0049
:10AF400028003E9B83552B00850AEFE04F8C8355EC
:10AF50000B002800EFE0AF8B7DBFEF720FAD5C49B7
:10AF600093E717005CC9EF8020336F704FAEEF722C
:10AF7000CFAB2E848145EFF08F9B05C18357050031
:10AF8000FD172310F50009C4835725002310F40092
:10AF9000EFF0BFFC01456F708FAB31456DDC2310C6
:10AFA0000400D5BFEF72CFA683C7950041112A8A4E
:10AFB00093F7F707A384F50032852E893284EFE0FA
:10AFC0008F8F93170501C187635EF004AA89C1457D
:10AFD0002285EFD0BFFA2A8B4E85832A0400EFC06A
:10AFE000AFE121E583574400231101000544F11727
:10AFF00093B71700A300F1008144034811000357E1
:10B000002100D6875285CE862286CA85EFE07FE66C
:10B01000A1679387170248003EC42302810026C619
:10B02000EFE01FB941016F70EFA113061100A28577
:10B03000EFF07F81AA8409E523110100094475BF5F
:10B04000930521005A85EFF09FF2835721002A844F
:10B05000CDD797B7FF1F9387E7C69C4391C7854518
:10B0600013052100EF40804083552100268531449F
:10B07000EFC0EFCF59D1231005002685EF70F07A8D
:10B080000144A5BFEF726F9A41112E896C00AA840A
:10B0900002C6EFF0CF8909CD03570500050723103D
:10B0A000E500EFF09FEB81473E8541016F702F9ADD
:10B0B0003247954775DBCA852685EF20D008C14702
:10B0C000E34405FE3244854741462310F40083578C
:10B0D0000900A685130544002311F400EFD0D069C0
:10B0E0002285C1B7EF72CF9283C795004111AA8A1A
:10B0F00093F7F707A384F5003285AE893284EFD049
:10B100009FFB93170501C187635EF0042A8AC1453E
:10B110002285EFD0BFE6AA845285032B0400EFC03E
:10B12000AFCD21E583574400231101008544F11779
:10B1300093B71700A300F10001440348110003571F
:10B140002100DA875685D2862686CE85EFE07FD22B
:10B15000A1679387070248003EC42302910022C6DC
:10B16000EFE01FA541016F70EF8DA285130611005E
:10B17000EFF06FED2A8409E523110100894475BFC2
:10B18000268593052100EFF0FFEFAA845DF5835536
:10B1900021002285EFC0AFBD4DF10149EFD0CF9D19
:10B1A000635DA900184893171900BA9703D70700E1
:10B1B0001DE7035721002390E700EFD0EF9B6302C8
:10B1C000250397B7FF1F9387E7AF9C4389C70355B4
:10B1D0002100EF4000222285EF703065B9BF0509DC
:10B1E00075BF954499BF05C19307F00F630FF50034
:10B1F000C547630CF5009307F5FF05453315F500CA
:10B200004205418182800145828041657D158280B1
:10B21000B9E1EF728F81034506033284EFF0BFFC82
:10B220009305803EB305B502C205C18191C903579C
:10B23000E402854763F6E70013050401EFC020161A
:10B240008357E40241677D176385E700FD172317E5
:10B25000F4026F60DFFF8280EF62BFFA004283C7B3
:10B260009500444D0349140093F7F707A384F500B4
:10B2700083470400220911673369F900A167B347C6
:10B28000F90041112A8BAE8A63ECE70C8347240056
:10B290001307C00EB91793F7F70F6371F70E034743
:10B2A0003400C14763ECE70C834744001307E00711
:10B2B00093C707086373F70A8349840083477400C0
:10B2C000A209B3E9F900856763F9F908034A640044
:10B2D000834754004E85220A336AFA00EF404062E9
:10B2E00045C123962403834B3400137AFA00239A32
:10B2F0003403238874032399440393890401631A54
:10B30000090023A60402239804024E85EFC0A00A78
:10B310001DA0034924004A85EFF0FFEC2397A40207
:10B32000834744004E85A388F402E3810BFEE30FBC
:10B3300009FCEFC06005EF70907981460146D68523
:10B340005A85EFE09FA5A167938797033EC4230228
:10B350000100480002C6EFE0BF8541016F60FFEDCC
:10B360008544A2862686D6855A85EFE01FA3A1676D
:10B37000938797033EC423029100E1BFBD44D5B734
:10B380009144C5B7EF62DFE801111C08404D3EC291
:10B39000B7070F003EC41C083EC62A89AE89EFC01D
:10B3A0001F9D585C1C5C634CB70A6394E50063E81E
:10B3B000A70A3385A740B3B7A700B305B740130664
:10B3C000803E81469D8DEFD0407B93140501C18066
:10B3D000A1659385C5034800EFC02FAC81454800A7
:10B3E000EFD0BFC1835504044800EFD05FC283553E
:10B3F00024044800EFD0BFC1814599C8C167FD173B
:10B400009305F00F6386F4002685EF402015AA858A
:10B410004800EFD09FBE03554404814511C9C16760
:10B42000FD179305F00F6305F500EF402013AA8583
:10B430004800EFD09FBC834564044800EFD0FFBBB9
:10B44000834574044800EFD05FBB5000014781463C
:10B45000CE854A85EFC0EFC405616F60BFDE8144D1
:10B4600085BFEF629FDC83C7950093F7F707A3843E
:10B47000F500EFF03FF16F609FDDEF627FD983C78A
:10B4800095004111404D93F7F707A384F5002A8AF0
:10B490003285B284AE89EFD01FC22A8B2685EFD0C9
:10B4A0009FC12A892685EFD0BFBF93170B0163CABE
:10B4B0000702E177CA97C207C183116763E3E70216
:10B4C00093070910C207C1831307B00F637BF7000E
:10B4D00093170901C187AA8A6348F000C54763FA38
:10B4E000570141016F601FD6EFC08F83E31B25FF1B
:10B4F000F5B763060B0263040902814463870A02FD
:10B50000B7077F0023106405231124057CC05685EE
:10B51000EFF07FCD9304803EB304950239A0B707C6
:10B520007F00232004047CC0814403552404EFB031
:10B53000101095CCEFC0BF83269593D7F4413337D5
:10B540009500AE97BA9708DC5CDCCE855285EFF0AB
:10B550007FE399E023220404A1679387B70348009F
:10B560003EC42302010002C6EFE08FE49DBF814785
:10B5700001481CDC232E0403C9BFEF621FCBEFC0C0
:10B58000FFE9E1473305F5029145EF30507FE5577C
:10B5900011C597A7FF1F23A1A75481473E856F6060
:10B5A0001FCB854717A7FF1F230AF7528280EF6240
:10B5B000DFC797A7FF1F9387E75180432DC08357AD
:10B5C0000404639EA70483572404639AB70436894E
:10B5D000B284EFC0CFF95C5C63C3B7046395B70076
:10B5E0001C5C63EEA7028347640463F3F400A68740
:10B5F0002303F4048347740463F39700A687A3032B
:10B60000F4048357440441677D176385E700850789
:10B610002312F4043C4481C7CA85268582976F6053
:10B620001FC397A7FF1F9387E74A9C43014599C310
:10B6300003C587008280EF625FBF0111B707070073
:10B640003EC683C79500584D0AC493F7F7070AC84A
:10B65000A384F5002A89AE8401CB1C4283C707006E
:10B660002304F700EF70D0452164930554022800AD
:10B67000EFC0AF82EFF0FFFAAA852800EFD0FF9766
:10B68000300001478146A6854A85EFC08FA113048B
:10B690004402480822CC230A010002CEEFE04FD139
:10B6A00005616F60DFBAEF625FB801117C003ECACE
:10B6B000B70707003ECC7C003ECE83C795002E84A2
:10B6C000AA8493F7F707A384F500A1659385550233
:10B6D0004808EFB09FFCEFF0DFF4AA854808EFD0F0
:10B6E000DF91500801478146A2852685EFC06F9BF8
:10B6F00005616F60DFB597A7FF1F9387A73D9C4348
:10B70000094599C303C59700828097A7FF1F9387B8
:10B71000673C9C43094599C303C5D700828097A71E
:10B72000FF1F9387273B9C43014599C303C5A7008F
:10B730008280EF62FFAD0111B70708003EC683C7E4
:10B740009500404D0AC493F7F7070AC8A384F50093
:10B750002A89AE8429C01442854703C7060063EED8
:10B76000E7068347940009468149638EC700B30703
:10B77000F740A304E400B339F00083C716002305A3
:10B78000F400EF70F03303572403058B09C763847B
:10B790000900EFA0B06B2164930584022800EFB08C
:10B7A000DFEFEFF05FF5AA852800EFD01F85EFF0FF
:10B7B0001FF7AA852800EFD05F840147814630003B
:10B7C000A6854A85EFC0EF8D13047402480822CC89
:10B7D000230A010002CEEFE0AFBD05616F609FA6B6
:10B7E000EF62BFA401117C003ECAB70708003ECC3F
:10B7F0007C003ECE83C795002E84AA8493F7F7077A
:10B80000A384F500A165938585024808EFB0FFE8A1
:10B81000EFF07FEEAA854808EFD02FFEEFF03FF063
:10B82000AA854808EFD06FFD500801478146A285E0
:10B830002685EFC00F8705616F607FA197A7FF1F67
:10B84000938747299C43014599C303C5B70082806C
:10B85000EF62BF9D0111B70707003EC683C7950081
:10B86000404D0AC493F7F7070AC8A384F5002A8954
:10B87000AE8405C41C42054783C70700636AF7040A
:10B880000347B400630BF700A305F400EF705023E7
:10B890008347B400A9C3EFD00FD921649305B40046
:10B8A0002800EFB09FDFEFF07FF9AA852800EFD0E6
:10B8B000CFF4014781463000A6854A85EFB07FFE70
:10B8C0002904480822CC230A010002CEEFE04FAE43
:10B8D00005616F60DF97EFD02FDAC1B7EF62FF9499
:10B8E00001117C003ECAB70707003ECC7C003ECE6B
:10B8F00083C795002E84AA8493F7F707A384F500E5
:10B90000A165AD054808EFB05FD9EFF03FF3AA8518
:10B910004808EFD08FEE500801478146A285268562
:10B92000EFB03FF805616F609F9297A7FF1F938765
:10B93000671A9C43094599C303C5C7008280EF621B
:10B94000DF8E01117C00AE843ECAA165B7070700F7
:10B950002A843ECCD1057C0048083ECEEFB0FFD310
:10B96000EFF0BFFCAA854808EFD02FE95008014747
:10B970008146A6852285EFB0DFF205616F603F8DBD
:10B98000EF62BF8A83C7950093F7F707A384F5009A
:10B99000EFF0FFFA6F60BF8BEF629F8783C7950060
:10B9A0000329C501411193F7F707A384F5001C4251
:10B9B00083C90700854763EC370597A7FF1F938767
:10B9C000A7689C432E84AA8495C7EFF01FF6894789
:10B9D0006302F502630009028347C900638C3701E3
:10B9E00023063901EF70D00D83572903898B99C342
:10B9F000EFA0D0452685A285EFF07FF4A167CD07A3
:10BA000048003EC42302010002C6EFE06F9A4101E4
:10BA10006F605F8397A7FF1F9387C70B9C431D45EC
:10BA200099C303C5E7008280EF623F800111B70729
:10BA300007003EC683C79500584D0AC493F7F70721
:10BA40000AC8A384F5002A89AE8405C71C4283C7AF
:10BA5000070093968701E18663C8060485466385DF
:10BA6000D7048346E7006386F6002307F700EF70EC
:10BA7000300521649305E4002800EFB01FC2EFF009
:10BA80007FF9AA852800EFD04FD7014781463000C3
:10BA9000A6854A85EFB0FFE03504480822CC230A8A
:10BAA000010002CEEFE0CF9005616F604FFAEF62C8
:10BAB000CFF701117C003ECAB70707003ECC7C00DF
:10BAC0003ECE83C795002E84AA8493F7F707A384FC
:10BAD000F500A165B9054808EFB03FBCEFF09FF352
:10BAE000AA854808EFD06FD1500801478146A2854A
:10BAF0002685EFB01FDB05616F606FF5EF624FF1D8
:10BB0000AA84014417A9FF1F130909FDE149EFC0E9
:10BB1000FF906344A400014519A83305340383272B
:10BB200009003E95835725006395970011056F60C6
:10BB30006FF10504E9BF032E850063040E1017A3FF
:10BB4000FF1F130323180323030063150300294376
:10BB5000639A060E03234E01631503001D4363938E
:10BB6000070EEF620FEAC689428A3E89BA8AB68416
:10BB7000328BAE8B2A84A1E903554E0009E50143BF
:10BB80001A856F608FEBA167A98F116763F7E700D4
:10BB9000EFF0DFF68145EFF08FBD0844B70700E016
:10BBA0005841F98F18455CC1B707001FF98F1CC5B4
:10BBB0005C4981C76105EFB01000E38209FC228572
:10BBC000EF70606E6DBF3285EFA0E0620D434DD91E
:10BBD0001C44116703D54700A167A98F63F7E700ED
:10BBE000EFF0DFF18145EFF08FB803238400931667
:10BBF0004B01D1828347B300035663008588FD8BD8
:10BC0000A305F300FD777D8E558EFD76FD16B204FB
:10BC1000F18E83274301C58E231273012313D300B2
:10BC20002304530123052301A3044301D9D722850B
:10BC3000EFB07FBBAA850844B5DD6105EFB0207683
:10BC4000ADBF1D431A858280EF628FDC0569AA842F
:10BC5000AE89328A0144FD5A7D19EFC0EFF0634589
:10BC6000A40001456F600FDED84493171400BA9703
:10BC700003D70700631B37032390570163050A00AE
:10BC80002685EF70E0389C448DC383D76700B3F7F7
:10BC90002701639C3701D2880148814701478146CB
:10BCA000014681452685EFF01FE905047DB7EF6267
:10BCB0002FD679711C103EC4B7070F003EC61C106A
:10BCC0003EC883C79500AA8A328593F7F707A384F5
:10BCD000F5002E893284EFD00FBE93170501C1877E
:10BCE0006350F006AA892285EFD0EFBC2A8A4E85E0
:10BCF000032B0400EFB05F9039E583574400814483
:10BD00000544F11793B71700A303F10083457100B1
:10BD1000DA872287D2864E862800EFE03FA40147CB
:10BD200081463000CA855685EFB0BFB7A1679387BB
:10BD3000F70348083ECC230A810026CEEFD05FE708
:10BD400045616F602FD0A28513067100EFE0BFAF91
:10BD5000AA84094445DD5285EFE0EFB80D445DD576
:10BD60000546D2852685EFF03FEE2A8445B7EF627F
:10BD7000CFCB835507000346270041112A842E8527
:10BD800032C62EC4EFE02FB611C53246A245228539
:10BD9000EFF09FEB41016F608FCBEF628FC683C7DF
:10BDA00095004111AA8A93F7F707A384F50032851D
:10BDB000AE893284EFD02FB093170501C187635746
:10BDC000F008C1452A8A2285EFD04F9B2A8D228513
:10BDD000EFD06FAE2A892285EFD08FAC930705F89C
:10BDE00093F7F70F1307E007AA8B6371F706228515
:10BDF000EFD00FAB2A8C2285EFD08FAAAA8C528568
:10BE0000032B0400EFB04FFF29E5835744002311B3
:10BE100001008144F11793B71700A300F100054416
:10BE20000347110083562100938784005685DA88E2
:10BE300022885286CE85EFE03FE6A167E9074800F9
:10BE40003EC42302810026C6EFD09FD641016F6019
:10BE5000CFBE13061100A285EFE0FF9EAA8409E57C
:10BE60002311010009446DBF930521006A85EFF09D
:10BE70006FA12A8455F5835521009356C9001316E6
:10BE8000490185486688E2875E87858A51822685D2
:10BE9000EFF07FCA2A8469B7EF62AFB683C7950017
:10BEA00041112A8B93F7F707A384F5003285AE89F9
:10BEB0003284EFD04FA093170501C1876352F00879
:10BEC0002A8A2285EFD02F9FAA8A2285EFD0AF9EA3
:10BED0002A892285EFD0CF9C930705F893F7F70FB7
:10BEE0001307E0072A8C637DF7042285EFD04F9B70
:10BEF000AA8C2285EFD0CF9A2A8D5285832B0400FD
:10BF0000EFB08FEF29E18357440085440144F117D6
:10BF100093B71700A301F100034731009307840092
:10BF20005A85DE882688D6865286CE85EFE0DFD613
:10BF30008D4748003EC42302910022C6EFD05FC760
:10BF400041016F608FAFA28513063100EFE0BF8F14
:10BF50002A84894471D19356C90013164901854832
:10BF60006A88E6876287858A5182D685EFF0BFBCF2
:10BF7000AA845DB7EF62CFA92A8981440144617A1E
:10BF8000916A17ABFF1F130BEBD3EFC0EFBE63C576
:10BF9000A40022856F600FAB8327090093991400DA
:10BFA000CE9703D5070033074501420741836362FB
:10BFB000570311CD03270B0009C785453E85EF3098
:10BFC000E04A832709000504CE97239007008504E3
:10BFD0006DBFEFF0BFB2832709000504CE97239011
:10BFE000070075D58145EFE09FF8D5B7EF624FA206
:10BFF00083C7950041112A8A93F7F707A384F500B8
:10C0000032852E893284EFD00F8B93170501C187BB
:10C010006354F004AA89832A0400EFB0EFDD21E124
:10C020008357440085440144F11793B71700A301D7
:10C03000F10003483100D68752850147CE86268617
:10C04000CA85EFD01FE3A167F50748003EC423026D
:10C05000910022C6EFD0DFB541016F60AF9EA2858F
:10C0600013063100EFE02FFE2A84894479D197A787
:10C07000FF1F938727C59C4381CB0449EFC0CFAFF7
:10C08000AA852685EF30803E13050401EFF09FEE70
:10C090002285EF609079814469BFEF628F9683C7F4
:10C0A00095004111AA8A93F7F707A384F50032851A
:10C0B000AE89328423110100EFC0FFFF9317050101
:10C0C000C187635CF0042A8AC1452285EFC01FEB5B
:10C0D000AA8B5285032B0400EFB00FD231E18357B6
:10C0E000440085440144F11793B71700A300F10001
:10C0F0000348110003572100DA875685D286268629
:10C10000CE85EFD01FD7A1679387270248003EC492
:10C110002302910022C6EFD0BFA941016F60EF91C9
:10C12000A28513061100EFE00FF22A84894469D139
:10C1300097A7FF1F938707B998433E8901CB04490E
:10C14000EFC08FA3AA852685EF3040321305040186
:10C15000EFF05FE2EFC04FA2954459D9930521005B
:10C160005E85EFE03FF2AA8441F51C4803572100A9
:10C1700022852390E700EF60506B83270900ADDB39
:10C1800003552100EF30E026A5B7EF628F8783C704
:10C1900095004111AA8A93F7F707A384F500328529
:10C1A000AE893284EFC03FF193170501C18763590F
:10C1B000F0042A8A2285EFC01FF02A895285032BBA
:10C1C0000400EFB06FC321E183574400854401446C
:10C1D000F11793B71700A301F10003483100DA8784
:10C1E00056854A87D2862686CE85EFD09FC8A1671E
:10C1F000F90748003EC42302910022C6EFD05F9B9E
:10C2000041016F608F83A28513063100EFE0AFE339
:10C210002A84894479D19167CA97C2071167C1837B
:10C220001307F7EF8544E36AF7FA97A7FF1F938791
:10C2300067A99843BE8B01CB0449EFC0EF93AA8551
:10C240002685EF30A02213050401EFF0BFD2EFC026
:10C25000AF92954459D11C482285814423902701EF
:10C26000EF60B05C83A70B00ADDB4A85EF30601850
:10C27000ADB7EF529FFB2A844105B284EFF09FCF08
:10C2800001C52285EF60705A81460146A685228548
:10C29000EF70C00B1C4C89C7DC4799C3228582977D
:10C2A0006F50FFFA97A7FF1F9387C7829C430145F2
:10C2B00099C313850701828097A7FF1F9387878102
:10C2C00088438280EF527FF69317C600DD8DC2054A
:10C2D0004111C1812A8432C6EFC07FD33246228504
:10C2E00011829375F60FEFC05FD141016F503FF699
:10C2F000EF521FF279713C083ED2B7070C003ED4D2
:10C300003C083ED683C79500AE842A8993F7F70789
:10C31000A384F500A165938535044810EFB0EFB70D
:10C32000C165FD15014417AAFF1F130A2A9B930A32
:10C33000400EAE892E8B2EC6EFC00F874205931795
:10C3400004014181C183B24563E3A702C167FD17C0
:10C350006385F5004810EFC09FCB50100147814620
:10C36000A6854A85EFB0EFD345616F50BFED330727
:10C37000540383270A0BBA9703D6C7016308360113
:10C38000638835014810EFF0FFF3DA85050465B7DF
:10C39000B285EDBFEF52FFE679717C083EC8B70762
:10C3A00011003ECA7C083ECC83C79500AA8932851D
:10C3B00093F7F707A384F5002E89EFC0DFCF8567D9
:10C3C000637EF502A165AA8489050808EFB0EFAC89
:10C3D0002685EF30E052133415000A04A2850808C0
:10C3E000EFC0BFC1A6850808EFC07FC235C00147B6
:10C3F00081461008CA854E85EFB0AFCA45616F50BF
:10C40000DFE3B30754030327CA0ABA9703D7070029
:10C41000631A970003D62700638A65030808EFF0C4
:10C420007FEADE8505042EC6EFB01FF9420593179B
:10C4300004014181C183B245E3E5A7FCC167FD1753
:10C44000E387F5FA0808EFC09FBC55B7B285D9BF9E
:10C45000C165FD15014417AAFF1F130A2A88930A14
:10C4600080022E8BAE8BC1B7EF523FDC1841834761
:10C47000170083460700A207D58FD207D1832390E8
:10C48000F50083472700034717008D45A207D98F82
:10C4900091832310F600EFC03FAD6F505FDBEF528A
:10C4A0003FD7C164014417A9FF1F130929839309CA
:10C4B0008002FD14EFB05FF06345A40001456F50AA
:10C4C0007FD8330534038327C90A3E958357050077
:10C4D000E38797FE0504F9BFEF529FD32A8AAE89FE
:10C4E000B284B68AEF30C04109E591473E856F506E
:10C4F0007FD52A894E85EF9010502A84638A0A04DA
:10C500008D476DD503570500C547E31147FF034726
:10C51000F9018546AD47E31BD7FC8347450091CB26
:10C520004146A6855D05EFC0D022814761D1AD4768
:10C5300075BF130965012302E500CA852685EF1042
:10C54000202D15CDA547E3830AFA2302040079BF05
:10C5500011CD83570500E39A47F94146A685190591
:10C56000EFC0301F814759D1994749B74E85EFF049
:10C570001FF32A8495473DD9130955007DBF4146D5
:10C58000A685231044012311340113051900EFC0BF
:10C59000B01E2285EF60B03C814789BFEF52FFC8D3
:10C5A00079717C003ECCB7070A003ECE7C003ED0BD
:10C5B00083C79500B2842E8493F7F707A384F50010
:10C5C0001306A1002A892C002685EFF0FFE9A1655A
:10C5D00028088D05EFB06F8C90408355A10003555E
:10C5E00081008546EFF05FEFAA84AA852808EFC096
:10C5F000DFA00356A100835581002808EFF09FCCEF
:10C60000300801478146A2854A85EFB08FA985474A
:10C6100048103ED42302910202D6EFD06FD9456173
:10C620006F50FFC2EF527FC079717C003ECCB707DC
:10C630000A003ECE7C003ED083C79500B2842E8493
:10C6400093F7F707A384F5001306A1002A892C00AD
:10C650002685EFF07FE1A16528088D05EFB0EF8317
:10C6600090408355A100035581008146EFF0DFE63D
:10C67000AA84AA852808EFC05F980356A1008355B5
:10C6800081002808EFF01FC4300801478146A285C9
:10C690004A85EFB00FA148102302910202D402D6BE
:10C6A000EFD00FD145616F509FBAEF521FB8EFF036
:10C6B000BFE26F50DFB99797FF1F9387E741884329
:10C6C0008280EF529FB6835725004111AE842A84A1
:10C6D0002307B10017F5FFFF1305A5696C002316AA
:10C6E000F100EFB0CFD581C42285EF60B02DFD57AA
:10C6F0002310F40013062002814513055400EF5067
:10C70000DFB541016F50BFB4EF529FB079717C002B
:10C710003ECCB7070A003ECE7C003ED083C79500D2
:10C72000AA89AE8493F7F7073285A384F500130630
:10C73000A1002C00EFF05FD3035581001144EF30CE
:10C74000201C15C10355A1000144EF90D02A01CD52
:10C75000035705008357810045446316F70085455C
:10C76000EFF03FF601442169930539002808EFA056
:10C77000DFF2A2852808EFC05F880356A100835529
:10C7800081002808EFF01FB4300801478146A685D4
:10C790004E85EFB00F9148104AD42302810202D691
:10C7A000EFD00FC145616F50FFA9EF527FA6979759
:10C7B000FF1F938727322A8488432E8915C1035788
:10C7C00045038357C401631DF70023260502231880
:10C7D00005024105EFA0303E63040900EF60302FF1
:10C7E00081449799FF1F9389694F130A8002EFB024
:10C7F000BFBC63CCA4029797FF1F938767369C4307
:10C8000089C70355C401EF104076630509002285EE
:10C81000EF6050031306400E81452285EF50FFA3C1
:10C82000FD57231EF4006F50FFA13385440383A7F7
:10C83000C90A3E95035705008357C4016315F700E5
:10C84000CA85EFF01FE885045DB7EF527F9C83C770
:10C8500095004111AA8993F7F707A384F500328563
:10C86000AE84EFC05F8585676370F5042A89EF3079
:10C870002009014411C983D704003144638627018C
:10C880008545EFF09FF201444E85A2864A86A68533
:10C89000EFD02FBFA1679387170448003EC423023F
:10C8A000810002C6EFD0CFB041016F50BF99EF5267
:10C8B0003F969797FF1F9387E72180431DCC014543
:10C8C000EFA0E05681470148C1641CDC232E04031D
:10C8D000232004041799FF1F1309494001449309B9
:10C8E000400EFD14EFB05FAC634BA400814517050B
:10C8F000000013054598EFB08FB46F50BF94330517
:10C9000034038327090B3E958357C5016385970040
:10C910008545EFF09FE90504F1B79357050113D75B
:10C920008700A380F50093170501C183A1832380AD
:10C93000E5002381F500A381A5008280EF52FF8EE0
:10C940002300050083C71500A300F50083C7250059
:10C950002301F50083C73500A301F50083C7450017
:10C960002302F50083C75500A302F50083C76500C5
:10C9700093059500A30305002303F5002304050098
:10C980003285EFF09FF96F509F8CEF527F884111F5
:10C99000E9541DC995C993F9C5FF2E842A89AA8433
:10C9A000338AA900B7EA040063149A020D8885440B
:10C9B00001CCB7E704009C5F82972AC622866C00F0
:10C9C00033053901EFC0405B268541016F509F87D9
:10C9D00083A78A039104829793170501C183A183DA
:10C9E000A38EF4FE93570501238FF4FEA183238EBB
:10C9F000A4FEA38FF4FE4DBF63E0D502EF52FF8289
:10CA0000B28741113686BE8536C6EFC0E056B246C3
:10CA1000410136856F50BF8381463685828083878A
:10CA200005001387F5003D05FD8793F777088346DA
:10CA300007007D158606B58FA300F5006307B700D4
:10CA40007D17834717009D83DDB78280EF52EFFD8E
:10CA5000B7E7040083A7070932872A863A858297B9
:10CA6000133515006F50AFFE01CD814799C9EF52C4
:10CA7000CFFB4146EFC0405085473E856F502FFDAC
:10CA800081473E8582801DC5EF522FFA4146814580
:10CA90002A84EF508FFC4146814513050403EF5073
:10CAA000CFFB0147C1672322040438C87CC8054571
:10CAB0006F50EFF901458280814729CDA1CDEF521A
:10CAC000CFF6B2842E891306800581452A84EF5063
:10CAD000CFF8CA8524C42685EFF01FF94146814569
:10CAE0002285EF508FF73044A2852285EFF01FF6A4
:10CAF00093040401A2852685EFF07FF2A685130535
:10CB00000402EFF0DFF12285EFF0FFF785473E8565
:10CB10006F50EFF33E858280EF528FEF4111E95461
:10CB20001DC995C993F9C5FF2E842A89AA84338A21
:10CB3000A900B7EA0400639444030D88814401CC42
:10CB4000B7E704009C5F82972AC622866C003305F3
:10CB50003901EFC06042268541016F50AFEE83A7D7
:10CB60008A039104829793170501C183A183A38E41
:10CB7000F4FE93570501238FF4FEA183238EA4FEB8
:10CB8000A38FF4FE4DBF71CDEF528FE8B28401E662
:10CB900005456F502FEB2A842E890145FDD93C486D
:10CBA0007848B3E6E700F5D69386F7FFB3B7F6000B
:10CBB0007D17032A4404BA9734C87CC8630F0A045B
:10CBC000C14913050A03B38949412295637B3601A4
:10CBD000B2862E86A685EFF03FE27C40BE9464C00C
:10CBE00045BFCE862E86CE85EFF01FE1C114D294CC
:10CBF0004E9923220404A2879306040103C7070069
:10CC000003C607038507318FA38FE7FEE398F6FE7F
:10CC10003044A2852285EFF07FE32699C14933068F
:10CC2000994063EA9900ADD4A686A685130504034E
:10CC3000EFF09FDC6DB78147B306F4003307F600D1
:10CC40000347070083C5060085072D8F2380E60074
:10CC5000E39437FF3044A2852285EFF03FDFC11413
:10CC60007DBF0145828019C9EF522FDC1306800574
:10CC70008145EF508FDE05456F506FDD01458280A5
:10CC800081473DC9B5C9EF524FDAFC4141462E8478
:10CC9000AA846393C70413860501A2878146C14510
:10CCA00003C7070003C507038507298F3305D6008F
:10CCB000034505008506298FA38FE7FEE392B6FEA4
:10CCC0003044A2852685EFF07FD82285EFF0BFF9AA
:10CCD00085473E856F50AFD7138507031D8E81456D
:10CCE0002295EF508FD77C40130700F813060402FB
:10CCF000A2972388E70255B73E858280EF52EFD294
:10CD00006D712E84B284AA85901028003689EFF0C8
:10CD1000BFDA19E9D55705A050400C402800EFF0C4
:10CD20009FE66DD9FD142104E5F82C004A85EFF04B
:10CD30003FF5814765D13E8551616F504FD1EF522C
:10CD4000CFCE41112EC432C62C000546EFF01FFB9A
:10CD500041016F50CFCFEF524FCD01112A842EC623
:10CD600002C802CA02CC02CEEFC06048B2462A8690
:10CD7000A2850808EFF0BFFC1375F50F05616F5031
:10CD80000FCDEF528FCA7971B2872A8421462308CA
:10CD9000B10013051101BE853AC436C6EFC0C01DEF
:10CDA000B246930591013685EFF03FB72285141006
:10CDB00035460C08EFF0BFF82A84224711E52146DA
:10CDC0000C103A85EFC0401B228545616F502FC87B
:10CDD000EF52AFC57171AE84AA850A853284EFF037
:10CDE000BFC801C90A86A6852285EFF03FC68147E4
:10CDF00011E1C5473E854D616F506FC5EF52EFBFE2
:10CE00001D712A8AB289BE843546854713051101F2
:10CE10002E8CB68A3A8BC28C468D2308F100EFC067
:10CE2000A01510100C085285231F0100EFF05FFAC7
:10CE30002A842DE9A147631BFD069307900591E025
:10CE4000E5473546E2851305110113990A012308C8
:10CE5000F10013590901EFC020121357890093976D
:10CE60008A00D98F90080C085285231FF100EFF03B
:10CE70003FF62A8405E9A1E09387FA0091831379AC
:10CE8000F9003EC6631309004149668B8144C14BDA
:10CE9000854DB2476397970C6A868C0033855C0199
:10CEA000EFC0800D228525616F50EFB89307900485
:10CEB000C9F8A54779B7834701050947C14B23083E
:10CEC000F10083471105A58FA308F1009387240083
:10CED000814463EFFB02014714083386E6008C08A7
:10CEE000B386E400BA95DA9683C6060083C50500CA
:10CEF0000507AD8E2300D600E390E7FE4147639817
:10CF0000E70490080C085285EFF09FEC35D535A862
:10CF1000B3069B00BA871008B305F60090083E964A
:10CF200003C506000346060085078506298E238073
:10CF3000C500E39277FF998F90080C085285BE9444
:10CF4000EFF01FE98947014749D52A84A1BF90081E
:10CF50003E96034606001408BE962380C600850749
:10CF600079BFB2478504638B971281471808B306CF
:10CF7000F70098083E973386F900034707000346F9
:10CF800006008507318F2380E600E39177FF900844
:10CF90000C085285EFF0DFE34DF93546E2851305C5
:10CFA00011012308B101EFB0307D139704014183D3
:10CFB000939784002183D98F10180C085285231F62
:10CFC000F100EFF0FFE051F1814710183387F900CD
:10CFD0003E960347070003460600B306FB0085079D
:10CFE000318F2380E600E39277FF75A01808B3061F
:10CFF000F70098083E973386F90003470700034679
:10D0000006008507318F2380E600E3E127FFCA870A
:10D010006398770990080C085285EFF07FDB15F5CF
:10D0200081479800B306F700900818103E973E9687
:10D0300003470700034606008507318F2380E6007B
:10D04000E39177FF3546E285130511012308B1010D
:10D05000EFB090721397040141839397840021836A
:10D06000D98F10180C085285231FF100EFF05FD6FE
:10D07000E31D05EC814710183387F9003E960347FE
:10D08000070003460600B306FB008507318F2380A7
:10D09000E600E3E227FFC109410BE5BB8147B5B7D5
:10D0A0009408BE9683C6060018083E972300D70052
:10D0B0008507B9BF638E062CEF522F9459712A84CD
:10D0C000BE89B28B85473546130511022E8B468CDF
:10D0D0004289BA8A368A2300F102EFB0F06910184B
:10D0E0000C10228523170102EFF09FCE631E05105E
:10D0F000A1476319FC069307900563930900E54770
:10D100003546DA851305110293140A012300F10252
:10D11000C180EFB0706693178A0013D78400D98F4F
:10D1200090080C1022852317F102EFF07FCA69EDF9
:10D13000639009049307FA00BD88918391E0C1448C
:10D14000C207C183DE8C814A3EC6414DB24763EAC5
:10D15000FA0C6286B3854B018810EFB0905F4DC525
:10D160003D555DA093079004E39C09F8A54749BF8E
:10D17000834701050947C14C2300F102834711058C
:10D18000B3C7F900A300F10293872900814963EF37
:10D19000FC02814618103306D7008C083387D9006B
:10D1A000B69556970347070083C5050085062D8F62
:10D1B0002300E600E390D7FE4147639AE704900816
:10D1C0000C102285EFF0DFC035D53DA8B3863A01BB
:10D1D000BA871010B305F60090083E9603C5060006
:10D1E0000346060085078506298E2380C500E39245
:10D1F00097FF3387EC4090080C102285BA99EFF026
:10D200003FBD8947014741D565616F50CF82900886
:10D210003E96034606001410BE962380C60085077E
:10D2200069BFB247850A93990A01939D8A0093D9F1
:10D2300009016399570D85473546DA8513051102B3
:10D240002300F10293D98900EFB01053B3ED3D01F3
:10D2500090000C1022852317B103EFF07FB74DF536
:10D260008147A68963E6970626860C084A85EFB0B3
:10D27000B05081471810B306F700100898083E9781
:10D280003E9603470700034606008507318F23803B
:10D29000E600E3E197FE639DA90590080C10228546
:10D2A000EFF01FB335F181479810B306F7009008EF
:10D2B00018183E973E960347070003460600850769
:10D2C000318F2380E600E391A7FF4109C10CBDBD6A
:10D2D00018089000B306F7003E963387FC0003471A
:10D2E0000700034606008507318F2380E60095BFBF
:10D2F00098084E97034707001C10CE972380E7003D
:10D30000850951BF85473546DA851305110223008B
:10D31000F10293D98900EFB03046B3ED3D019000A2
:10D320000C1022852317B103EFF09FAAE31E05EC32
:10D33000814718089000B306F7003E963387FC003B
:10D3400003470700034606008507318F2380E60068
:10D35000E391A7FF41460C084A85EFB0F0418147B1
:10D360001810B306F700100898083E973E9603473A
:10D370000700034606008507318F2380E600E3910E
:10D38000A7FF90080C102285EFF09FA41DDDADBD16
:10D390007D558280EF427FE901112A842E85930515
:10D3A0005100328902C002C202C402C69304740052
:10D3B000EFF0AFD61D46A68513059100EFB0D03B28
:10D3C00010088A854A85EFF0BFA019ED9307140075
:10D3D000180883C607000346070085070507B18EB6
:10D3E000A38FD7FEE397F4FE05616F405FE6EF423F
:10D3F0003FE22E848C414111AA898387150032892E
:10D40000914463D30700A1449797FF1F9387C7C335
:10D410009C43B1C3B5CE8D472310F10083C72500CF
:10D420004A852301F10083C73500A301F10083C7BA
:10D4300045002302F10083C75500A302F10083C712
:10D44000650093059100A30301002303F100230469
:10D450000100EFF08FCC0C404A860A85EFF00FCE2A
:10D460000328040083564400A6881D08814701470D
:10D47000E51642868A854E85EFF05F982A8909E590
:10D48000A6852285EFB0FFB24A8541016F409FDB40
:10D490004A860A85EFF08FCA7DBFEF427FD72E8480
:10D4A0008C414111AA89838715003289914463D345
:10D4B0000700A1449797FF1F938707B99C43B1C307
:10D4C000A5CE8D472310F10083C725004A8523018F
:10D4D000F10083C73500A301F10083C74500230293
:10D4E000F10083C75500A302F10083C765009305CF
:10D4F0009100A30301002303F10023040100EFF0D6
:10D50000CFC10C404A860A85EFF04FC383564400D2
:10D51000032804008A85858EC2061D08C182231255
:10D52000D400A68881470147E51642864E85EFF074
:10D530007FB841016F401FD14A860A85EFF00FC0C6
:10D54000C9B7EF429FCEB335B000011185052A89D6
:10D550001315F601336515012308B1009305110178
:10D5600036843AC632C03EC442C2EFF00FBBA24777
:10D570001248425593D68700230BF1009305910181
:10D5800093578800A30AD100A30BF100230C0101DB
:10D59000EFF0AFB83247024603280400B337E0008B
:10D5A000835644009207914411C2A1444A85A6883B
:10D5B00042860C08EFF09F842A8909E5A68522851A
:10D5C000EFB03F9F4A8505616F407FC8EF425FC45F
:10D5D00001113EC68647B335B0008505AA891315EB
:10D5E000F6015D8D2308B1009305110136843A8957
:10D5F000B28442C446C2EFF04FB222489248164568
:10D6000093578800A30AF1009305910193D78800EE
:10D61000230B0101A30BF100230C1101EFF0EFAF7D
:10D620003247104083564400B337E0009207032886
:10D630000900914891C0A1480C084E85EFF09FA7C2
:10D64000AA8411E5835544004A85EFB09F9626854C
:10D6500005616F403FBFAA959307F00F17F70000D1
:10D66000130787876317B50013C5F7FF1375F50F09
:10D67000828005058346F5FFB58FBA9783C70700FB
:10D68000D5B70357450014419307F00F17F6000074
:10D69000130686843697420741831395060141811C
:10D6A000631BE500AD8FB29703C50700130515F3A3
:10D6B000133515008280850603C5F6FFA98FB29742
:10D6C00083C70700D9BFEF425FB6B28736842E8684
:10D6D000BA86AA853E85BA84EFF06FE6634B0500F3
:10D6E0002285EFB0D0302A86A686A2852685EFF067
:10D6F0000FE56F40DFB5EF42BFB15D712A8BAE8A97
:10D7000017E500001305C57A2C00B284368ABA8961
:10D710003E89EFF04FE42A8459E534104146DA851A
:10D720002800EFF0CFE12A843DED8547A303F10007
:10D73000A6C2930771002408BEC4A68685470D467D
:10D740002C18281002DC02DED6C0BEC6EFF00FDBBC
:10D750002A8431E983477102A6860D4693F7F707BD
:10D760002300FA00C1473EDE2C188947281026DC2A
:10D77000A303F100EFF08FD82A8415E54146A68572
:10D780004E85EFB0607F8D47A6860D462C18281079
:10D79000A303F100EFF08FD62A8411E54146A68558
:10D7A0004A85EFB0607D228561616F40BFA9EF427D
:10D7B000DFA797D7000093876709984383C747007F
:10D7C00079712A89AE8417E500001305E56E0C080F
:10D7D0003AC42306F100EFF00FD82A8415E514109F
:10D7E0004146CA850808EFF08FD52A8411ED140848
:10D7F00015462C000810EFF08FD42A8411E521463D
:10D800002C082685EFB04077228545616F403FA404
:10D81000EF42BFA197D70000938747039C477971D8
:10D82000AA842E8417E50000130585690C083EC6FE
:10D83000EFF06FD20DE514104146A6850808EFF011
:10D840000FD011ED140811466C000810EFF02FCF27
:10D8500019E58347F10193F7F7032300F4004561CD
:10D860006F40FF9EEF427F9C3688A1488147014769
:10D87000E546EFF0AFD86F409F9DEF421F9B368883
:10D88000A14881470147E546EFF0DF826F403F9CAA
:10D89000EF42BF9901112A842E850C0832C6EFF0A1
:10D8A0008FCB19E9324797E600009386E65F1008B0
:10D8B000C1452285EFF03FE105616F405F99EF427E
:10D8C000DF964111C1472EC032C48A8509463EC247
:10D8D0003EC6EFF0AFC241016F407F97EF42FF9429
:10D8E0004111AE8613061009AA850A8502C002C23C
:10D8F00002C402C6EFF0AFC441016F405F95EF4232
:10D90000DF92328797E600009386065C2E869305A9
:10D910000002EFF05FDB6F409F93EF421F91797140
:10D92000C1472ACC2ED032D42C080D4628003ECE3A
:10D930003ED23ED602C402C602C802CAEFF00FBCF5
:10D9400045616F40DF90EF425F8E0111AA842E8403
:10D9500017E500001305C5578A85EFF0CFBF05E531
:10D9600014084146A6850A85EFF06FBD09ED83478F
:10D97000E1010347F101A207D98FCA07C983617783
:10D98000D98F2310F40005616F407F8C05C9EF42E9
:10D99000DF899787FF1F9387A71890439785FF1FFD
:10D9A000938545181785FF1F13058513EFB0800970
:10D9B0001785FF1F1305C5126F407F891785FF1F4D
:10D9C0001305051282809DC5EF423F869787FF1F92
:10D9D00093870715944301112E840A869785FF1FAC
:10D9E00093854514EFB0800A0A85029401450561CC
:10D9F0006F40FF857D558280EF423F83EFB08014FA
:10DA00009787FF1F23AEA71017F5FFFF130525F813
:10DA1000EF90D0406F40BF831787FF1F1307871217
:10DA20009317150008433E95FD572310F50082809B
:10DA3000EF42AFFF2A84084019E16F405F811C412B
:10DA400058401CC06313E5005CC083475500232089
:10DA50000500F99BA302F500EFB0EFF9E9BFEF4233
:10DA60002FFB9787FF1F9387E70F98432A8411CBDB
:10DA70008347350093F7070289C703550500894599
:10DA8000029713054401EF901013835504000355CA
:10DA9000E400EF20701B485809C5EFB0CFF5232AEA
:10DAA000040213058403EFF0BFF88144B149EFA0ED
:10DAB000FF9A63C5A402834734002320040493F72C
:10DAC00027FCA301F4000048EFA05F9A131615008D
:10DAD00081452285EF406FF86F40CFF6B38734035E
:10DAE0000329040385043E994A85EFF07FF423045B
:10DAF000090075BF8347350093F7070299E3014595
:10DB000082808357E500E39CB7FEC167FD1763166B
:10DB1000F600054582800545B9A0EF420FF1931745
:10DB20000601C187B2842A8401496359F0028357F0
:10DB300005008DCB01456367F600034584003E95E3
:10DB40003325A6001375F50F39A81C4813171900C3
:10DB5000BA9783D70700E38097FC0509EFA01F91D0
:10DB6000E345A9FE01456F408FEEEF426FEAAE89B3
:10DB7000AA84EFA07F852A84EFD0BFAAAA86014796
:10DB80001306840197050000938545E91785FF1F5B
:10DB9000130585FBEFA0AFD52A8921CD8C44130452
:10DBA000C50022859E0593F50508EFB00FC5CC4052
:10DBB00083877400E18163D1070493E5050822851A
:10DBC000EFB0AFC30D46938544002285EFB00FC17F
:10DBD00083D504002285EFB0EFC583D524002285CC
:10DBE000EFB04FC503D6490083A509002285EFB0E9
:10DBF000EFBE4A856F400FE593F5F507C9B7EF42D1
:10DC0000CFE201112A84328532C6EFB06FB4EF90B3
:10DC10003F91835704001787FF1F1307270C3246D5
:10DC2000231BF100930700F8A30DF1001C471843D4
:10DC3000231AA1008983858BB307F740B285480872
:10DC40003ECE231C0100230D0100EFF01FF2056101
:10DC50006F40EFDFEF42CFDB0041014529CC930459
:10DC6000C40026853289AE89EFB08FB295452A8AE5
:10DC70002685035B0401EFB02FAF2685EFB02FC6DA
:10DC80008D45AA8A2685EFB02FAE2685EFB02FC529
:10DC90005C48420A135A0A01D2975CC423186401F3
:10DCA000814763983A0146054D81330625419337F4
:10DCB000160013F5F70F6F40EFD8EF428FD4896944
:10DCC0002A8BAE8B328AB68A81440144314CFD19CD
:10DCD000EFA0CFF863C9A400EFA04FFB018D33B5CF
:10DCE000AA006F408FD53389840383270B003E99A8
:10DCF00063170A008347890085043E94D1BF035609
:10DD00000A00DE854A8533F6C900EFF0BFF47DD105
:10DD10000545C1BFEF426FD101112A847C00035534
:10DD2000E5003ECAB70707003ECC7C003ECEEF10B0
:10DD3000303D2A8985454808EFB0EFC1994548082C
:10DD4000EFB02FA7AA844A85EF10B03D2380A4002E
:10DD50009787FF1F938787F89C434166130606F059
:10DD60009396870113D78701558F93D68700F18E3D
:10DD7000558FA207B706FF00F58FD98F11462C00EB
:10DD8000138514003EC4EFB0201F5008A382040086
:10DD900089452285EFF0BFE609C9AA8513058403EA
:10DDA000EFB0EFBB3C4085073CC005616F402FCA18
:10DDB000EF42AFC7EFA08FED2A840504EFA00FEC70
:10DDC0003305A402F14791453305F502EF10207B9E
:10DDD00001E565556F40AFC79787FF1F23ACA7D6F6
:10DDE000EFA0CFEA2A840504EFA04FE93305A4028F
:10DDF00089450605EF10A07869DD9787FF1F23A3EB
:10DE0000A7D4EFA0AFE82A840504EFA02FE73304DE
:10DE1000A4029787FF1F239987D2EFA02FE72A84B8
:10DE2000EFA0CFE5930714003385A7029787FF1F64
:10DE3000239DA7D097E70000938747CD1787FF1F43
:10DE40002328F7D0014579B7EF428FBCAA842E89E9
:10DE500001449789FF1F938969E8130A8006EFA0A0
:10DE6000EFE16345A40001456F40CFBD3305440396
:10DE700083A709024A86A6853E95EFF0BFC719E140
:10DE80000504F1BF0545CDB7EF42AFB7AA8A2E8B87
:10DE9000B28B368C3A8A814401448149978CFF1FAA
:10DEA000938CCCE3130D8006EFA04FDD63C7A40075
:10DEB00011E085494E856F404FB83389A40383A78D
:10DEC0000C025E86D6853E994A85EFF0BFC219CD19
:10DED000EFA0CFDB0544636B4501D2866286DA850D
:10DEE00013050903EFF07FDD11C1854985046DBF7E
:10DEF000EF420FB2C16441112A8901449789FF1F83
:10DF00009389C9DD130A8006FD1436C632C42EC2B9
:10DF1000EFA0CFD692452246B2466346A400014503
:10DF200041016F402FB23305440383A709023E9598
:10DF300009C683473500C18B9DC791C6834735000D
:10DF400093F707028DC3630699008357E500639C2E
:10DF500027010357050001CB63E7E50083478500F0
:10DF6000BA97E3CFF5FA05044DB7EF426FAAC16443
:10DF70002A8901449789FF1F938949D6130A80068D
:10DF8000FD14EFA0AFCF6344A4006F40AFAB3305E7
:10DF9000440383A709023E958357E50063889700F1
:10DFA0006304990063942701EFF07FAB0504D1BFB0
:10DFB000EF42AFA489692A8AAE8A328BB68B81443C
:10DFC000178CFF1F130C8CD1930C8006314DFD195B
:10DFD000EFA0CFCA63C4A4006F40EFA533899403B8
:10DFE00083270C028355CA015A863E994A85EFF071
:10DFF0007FB005CD814D05A03384AD038327090390
:10E0000003D60B00D68533F6C9003E942285EFF087
:10E010007FC419E5850DEFA06FC4E3CFADFC31A03F
:10E020002285EFF0FFA023040400850455B7EF42DA
:10E030004F9D4169AA8A014A178BFF1F130B0BCA18
:10E040007D19C14B054CEFA06FC36344AA006F401C
:10E05000CF9E93098006B3073A0383290B02BE992A
:10E0600083D7E900638C270163842A0163985701F1
:10E0700003A4890311E44E85EFF0DFC9050AE1B777
:10E0800083570401639977079304C4002685EFA0A2
:10E090003FF085452A8D2685835C0401EFA0DFECE7
:10E0A0002685EFA0FFFF62056185635F05028D4550
:10E0B0002685EFA07FEB89452685EFA0FFEA8945FD
:10E0C0002685EFA07FEA85452685EFA03FEB8347B5
:10E0D0000500094793F7F7076398E70099452685F8
:10E0E000EFA0DFE9A30285014848337D2D01231805
:10E0F00094016A9548C40040B5BFEF420F9337E4DE
:10E1000004008327041D82979787FF1F83C707AAF0
:10E110001755FF1F13058553A300F5008327441CE3
:10E1200082978327841C81461306F00F81450145A1
:10E1300082976F40CF911787FF1F130727971843C8
:10E140009785FF1F83C585A69787FF1F938787A4A1
:10E1500083468703034697036397D5009787FF1F7E
:10E160002386C7A4828083C587010347A70363175B
:10E17000B6009787FF1F238BE7A2828003C6870123
:10E180006317C7009787FF1F2382D7A2828083C6A9
:10E190008701130750026319D7009307600217879E
:10E1A000FF1F2305F7A0828083C687011306600244
:10E1B0006315D60093077002DDB783C7870155BF8B
:10E1C0009787FF1F9387079DD44B09476385E60810
:10E1D000EF42AF851789FF1F130909993E848347D2
:10E1E0000900918B9DCFB7E4040083A7041D82979B
:10E1F00083A7441C1785FF1F13058597829783A764
:10E20000841C81461786FF1F034686988145014579
:10E21000829721C183470900ED9B1787FF1F2305C4
:10E22000F7948347040093F7F70F85C79147178743
:10E23000FF1F232BF796EFF05FECEFF0DFEFB7E770
:10E240000400BC4F414691451785FF1F03450595C6
:10E2500082976F30DFFF8280EF323FFD8D474111A3
:10E260006304F504C5476306F50285476310F502AC
:10E270009787FF1F238EA792B7E70400BC4B930537
:10E2800000101785FF1F03456591829741016F308C
:10E290001FFC85471787FF1F230CF790B7E7040083
:10E2A000BC4B93050020F1BF9787FF1F9387878E94
:10E2B000D44B1147638DE600B7E7040083A7071D21
:10E2C0008297B7E70400BC4B930500045DBF054986
:10E2D0001787FF1F232A278D83C7070032C62E8486
:10E2E00093F7F70FC5D7B7E4040083A7041D7D1487
:10E2F0001374F40F8297E37689FCB245994703C6FD
:10E300001500E3F0C7FCFC4409061785FF1F130541
:10E31000658A8297BC48930500081785FF1F03454F
:10E32000E587829779BFEF325FF01787FF1F1307EA
:10E3300067864047184B1C409786FF1F23A2F6862E
:10E340006316E4001787FF1F232EF784130584FE4E
:10E35000EF907FF3035564FFEF903FC6EFA0BFE956
:10E360006F30FFEEEF327FEC9787FF1F9387878236
:10E37000D84BDC4799C3EFF01FFB85471787FF1F7A
:10E380002324F7829777FF1F938747729C43930557
:10E3900000021785FF1F0345658083C78703178722
:10E3A000FF1F2305F780B7E70400BC4B82976F304F
:10E3B0001FEA9777FF1F23A1A77E8280EF325FE5D8
:10E3C00037E404007C4CA1451775FF1F0345057D0C
:10E3D00082977C48A1451775FF1F0345257C9774DC
:10E3E000FF1F9384247B8297DC4489E7EFF05FDD95
:10E3F0006F305FE503D567FFEF903FBCAA897DD5FD
:10E40000D84891476310F7027C4C91451775FF1F60
:10E410000345C57882977C4891451775FF1F0345D2
:10E42000E577829703A9490103D409018947B7E930
:10E4300004001777FF1F2329F77683A7091D2104FE
:10E440004204829783C784011755FF1F13050520D7
:10E4500061191757FF1FA30BF71E83A7491C4180A3
:10E4600082979777FF1F2385077483A7C91C81466E
:10E4700009469375F40F4A85829711E99787FF1F24
:10E4800083C7478389C79750FF1FE780208EB7E770
:10E490000400BC4F2146A1451775FF1F03450570B9
:10E4A0008297B9B7EF327FD893F7052001112E84F8
:10E4B00081CBEFF03FEB1345042005616F303FD96E
:10E4C00093F70510A9CB9774FF1F9384A46CDC48C5
:10E4D000EFF07FC61777FF1F1307475D184383C709
:10E4E0008401034787036316F700DC4499C3EFF008
:10E4F0009FE385471777FF1F2328F76AB7E70400D4
:10E50000BC4B930500021775FF1F034525698297D1
:10E51000134504105DB793F70508ADC79777FF1F44
:10E5200083C75769E91719469775FF1F9385A56833
:10E530001305D10093F4F70F1779FF1F034989677B
:10E54000EFA0902393970401C1831777FF1F130750
:10E55000E766231DF100231CF1009777FF1F9387C7
:10E5600067633ACE3ACAD8432306010009CBDC439D
:10E570009315890154080D46E1856800829713457B
:10E58000040825BF93F72500B1CF9777FF1F938726
:10E590006760D84B89476306F7029777FF1F83C7E9
:10E5A000A75C13F7270011EF918B99CFB7E7040011
:10E5B000BC4F1306000A89451775FF1F0345055E0A
:10E5C000829713452400D5BD9777FF1F9387074E89
:10E5D0009C4383C787031777FF1F2309F75CEFF07E
:10E5E000FFDDC5B793F7050291C7EFF03FDD134597
:10E5F0000402E1B593F7850091C7EFF0BFD613454C
:10E60000840065BD93F7150091C7EFF07FBB1345FC
:10E61000140065B593F7450091C7EFF07FBA134535
:10E62000440061BD93F7050485C39777FF1F83C737
:10E63000675681CBEFF07FAC91471777FF1F2325FB
:10E64000F7561345040495BD93F705010145E3868C
:10E6500007E69777FF1F9387E753D84B91476310DF
:10E66000F7049777FF1F938727509C4313D7270002
:10E670008583D98F858B91E7B7E7040083A7071DB2
:10E680008297B7E70400FC4F91451775FF1F0345BC
:10E69000E550829785471777FF1F2327F7501345CB
:10E6A000040121BD9777FF1F2386A7608280EF3288
:10E6B000DFB79777FF1F23A5074E9777FF1F23A389
:10E6C000074E85471774FF1F1304443E1777FF1F3B
:10E6D000232CF74C1C4083C787031777FF1F2307A2
:10E6E000F74CEF90FFDF39C19757FF1F23A4A7F620
:10E6F0001C4017050000130525DB83C78703177728
:10E70000FF1F2305F74A1757FF1FA301F7F4977759
:10E71000FF1FA3810748B7E7040083A70708829774
:10E720009777FF1F238CA7466F307FB2B7C7898EBC
:10E73000938767ED1757FF1F232EF7F055BF177705
:10E74000FF1F03472745795555E39777FF1F9387A9
:10E75000674403C7170005079776FF1FA38CE6429F
:10E7600003C717008D463377D7029776FF1FA38321
:10E77000E64283C617001777FF1F13072733184396
:10E7800093F6F60FA9EA834787031777FF1F230F36
:10E79000F74085471777FF1F230EF73E9777FF1F38
:10E7A0009387873C9C430145998BA9E3EF32FFA7F0
:10E7B00037E404007C48C1451775FF1F0345053E3B
:10E7C00082973C4885451775FF1F0345253D829775
:10E7D00001456F30DFA783C7170085466395F600B4
:10E7E000834797035DB78347A70345B78280977731
:10E7F000FF1F83C7273AA1CBEF323FA337E40400C2
:10E800009777FF1F238807387C4885451775FF1FBA
:10E810000345C53882977C4C91451775FF1F03450A
:10E82000E53782977C4891451775FF1F03450537EB
:10E8300082973C48C1451775FF1F034525368297CF
:10E8400001456F30DFA079558280EF321F9E2A8408
:10E85000035565FFEF906FF69777FF1F9387873318
:10E86000D847BE841DEBEFA05F989C48232004008E
:10E870008DEB9777FF1F23A787329777FF1F23A181
:10E880008732B7E70400BC4B89451775FF1F034566
:10E89000E530829701456F309F9B630A87001843DC
:10E8A000D1B780C39777FF1F23AE872ED9BF795585
:10E8B000DDB7EF329F979777FF1F9387E73F884336
:10E8C00023260500232405005105EF80D02E6F304C
:10E8D0001F98EF329F951774FF1F1304E43D1C40EF
:10E8E000411189CF9C472302B5002AC61CC1EFF015
:10E8F0005FFC1C409C4B99C33245829741016F30AD
:10E900001F95EF329F924111444D328532842EC6BD
:10E91000EFA00FF92AC42285EFA0EFF903A8440065
:10E92000630C0800B245835744001840224683D543
:10E930004500AA862685029841016F305F91EF322B
:10E94000DF8E404D1DC408C0970500009385E50289
:10E9500013054401EF8090189777FF1F9387C73501
:10E960009C43014589E79777FF1F23A787346F30C2
:10E970001F8E7D55EDBFEF325F8B0111680093054F
:10E98000F00F02C602C802CA02CC02CEEFF07FF43A
:10E9900005616F30DF8B9777FF1F9387E7319C43CB
:10E9A000D847A1679D076311F702EF321F88011155
:10E9B0003285EFA0EFEE230AA10081456800EFF059
:10E9C0005FF105616F30BF8882809777FF1F938763
:10E9D000A72E9C43D847A167938777036311F7025B
:10E9E000EF32BF8401113285EFA08FEB230AA10023
:10E9F00081456800EFF0FFED05616F305F85828033
:10EA00009777FF1F9387472B9C43D8479547631CF5
:10EA1000F702EF329F81011132853284EFA04FE877
:10EA2000230AA1002285EFA00FE983574400231B8E
:10EA3000A10081453ECC1C4068003ECEEFF07FE94E
:10EA400005616F30DF808280930785FF89CF832740
:10EA5000C5FF91CBDC4B81CBEF322FFD032585FF2A
:10EA600082976F30CFFE8280EF322FFC2A8432856E
:10EA7000EFA00FE3BD4763EBA70018449377F500C1
:10EA80000345B70041995D8DA305A7006F302FFCAA
:10EA9000EF32AFF901117C003ECAB70707003ECC48
:10EAA0007C003ECE5C4D8DCF2A8413858700AE84DA
:10EAB000EF807004A1652A899D054808EF80FFBD9D
:10EAC0009305803EB345B902480893F5F50FEFA0D2
:10EAD000CFD2014781465008A6852285EF807FDC92
:10EAE00005616F30CFF6EF324FF4EFF07FFA6F3001
:10EAF0000FF6EF328FF301117C00AE843ECAA165A0
:10EB0000B70707002A843ECC48087C00938575032C
:10EB10003ECEEF809FB81C44480883C5B700BD892E
:10EB2000EFA0AFCD500801478146A6852285EF8032
:10EB30005FD705616F30AFF1EF322FEF2A84AE84DB
:10EB4000EFF09FF2A6852285EFF0BFFA6F302FF02D
:10EB5000EF32AFEDEFF0FFF96F306FEFEF32EFEC28
:10EB60000329C5014111630409022A843285B28454
:10EB7000EFA00FD32AC62685EFA0EFD38327490045
:10EB80002A8691C7DC4781C7B24522858297410119
:10EB90006F30EFEBEF326FE9444D81CC2A84328540
:10EBA000EFA06FD1DC40AA8589C79C4799C3228515
:10EBB00082976F30CFE9EF32AFE5032AC5014111EB
:10EBC00063030A062E89AA84954532853284EF8034
:10EBD000DFAC85452285EFA0CFBDAA89CA852285F5
:10EBE000EFA0EFC283274A009DC7DC438DC7228573
:10EBF000EFA0AFBA83274A00104083564400DC439D
:10EC00007115A307A100B2961307F1004E86CA85BD
:10EC10002685829701C52380090031A08345F10034
:10EC20002285EFA00FB941016F30CFE1EF32EFDF66
:10EC300065711C083EC2B70780013EC41C083289BA
:10EC40003EC62A84AE84EFF07FF14A85EFA0AFC6BE
:10EC50008357A10089CFAA8550002285EFF0BFF528
:10EC6000014781465000A6852285EF809FC35961E8
:10EC70006F30EFDDEF32CFD965711C088329C501F4
:10EC80003EC2B70780013EC41C082A84AE84328984
:10EC90003EC6EFF03FF0638409024A85EFA0AFC1A2
:10ECA0008357A100AA8581CF50002285EFF0BFF0E5
:10ECB000014781465000A6852285EF809FBE59619D
:10ECC0006F304FD8EF326FD665711C083EC2B70760
:10ECD00080013EC42A841C0832853EC6AE84EFA063
:10ECE0008FBD8357A10089CFAA8550002285EFF000
:10ECF0009FEC014781465000A6852285EF807FBAB0
:10ED000059616F30CFD4EF324FD2444D91E88347F1
:10ED1000450093B71700B307F0403E856F302FD3FF
:10ED20001845FD577DDB97070000938707032A846A
:10ED30005CCB97050000938565D113858400EF8037
:10ED4000E05980C003474400814761FB1777FF1FEC
:10ED5000232697F6D9B7EF32AFCB8329C5014111EE
:10ED6000032985008147638B090803240901914524
:10ED70002A8A2285EF807F9285452285EFA06FA3A6
:10ED80008945AA8A2285EFA0CFA2AA84EF809F9608
:10ED900083A749002A8B9DC79C438DC72285EFA07E
:10EDA000CF9F83A74900A306A100104083564400CB
:10EDB0009C431307D100B296D6851306E100528515
:10EDC000829709CD83570B002380F400A183A38091
:10EDD000F40023800A00A306010029A88357E1005C
:10EDE00022852380F4008345D100A183A380F40011
:10EDF000EFA02F9C8347D100B337F0000347B90041
:10EE0000920701453D9BD98FA305F90041016F3061
:10EE10006FC3EF328FC141111DE99777FF1F9387B1
:10EE2000E7E9804305C80440130984009DC55C40A0
:10EE300099C79C4B89C726852EC68297B2459307F2
:10EE4000803EB385F5024A85EF80605521A0404D94
:10EE5000AA8479F841016F308FBF4A85EF80A055B1
:10EE60005C40EDDBDC4BFDD726858297E5B7EF32C2
:10EE7000CFBB2A843285EFA0AFA2AA852285EFF00E
:10EE80005FF96F30CFBCEF324FBA2A84AE84EFF017
:10EE90001FFEA6852285EFF0BFBF6F304FBB084134
:10EEA0003355B50005898280EF322FB81774FF1FE4
:10EEB0001304C4E21C5C0111231701008D83858BB0
:10EEC000A303F1008327040B231801002319010079
:10EED00003D7C7013ECA3C002314E1007D57231528
:10EEE000E1000357C4023ECC02CE2316E100EF80BE
:10EEF0002FE38357E101231EA10093F707E093E777
:10EF00001710231FF1009777FF1F83C7C7DF85C343
:10EF100005470145638AE7008347840393E7270099
:10EF20001777FF1F2308F7DE05616F304FB2814767
:10EF300017D700001307871985461306710085450A
:10EF40004808EF70E04B6DF183478403F59B17771A
:10EF5000FF1F2301F7DC85471777FF1F2305F7DA2B
:10EF6000E1B7EF328FA9977DFF1F938D2DD703A6B1
:10EF7000CD0639712A8981478144930600023357AF
:10EF8000F600058B01C7850493F4F40F8507E39819
:10EF9000D7FE83A70D0B231701022318010203D705
:10EFA000C7013EDA3C102314E1027D572315E1022C
:10EFB00003D7CD023EDC231901022316E10202DE53
:10EFC000EF800FD68357E103231EA102014593F77B
:10EFD00007E093E71710231FF1029777FF1F83C7FE
:10EFE00087D2A9EF9777FF1F83C7D7D23EC69779FD
:10EFF000FF1F9389A9CE0144014D9D4A054B954BB6
:10F00000177CFF1F130CCCD4977CFF1F938CCCD3A1
:10F0100003DAC90563090A00EA85631459036685A2
:10F02000EFF0FFE71DC1050DA1478909E312FDFEC1
:10F030002DE09777FF1F23AB07D0014521616F308B
:10F040008F9F6285EFF0BFE579DD3247B38784009B
:10F05000E3F0E7FE9C001306140006043E94131729
:10F060008A0093578A00D98FC207C183A30EF4FC8C
:10F07000A183230FF4FC03A70D07B317AB01D98FAE
:10F080001777FF1F2324F7CC63047601328461BF16
:10F0900015449777FF1F83C7E7C613871700977636
:10F0A000FF1F2381E6C693161400230EF10017D725
:10F0B00000001307A701814785067008CA85481814
:10F0C000EF700034E34705F68347C1010545177724
:10F0D000FF1FA309F7C29777FF1F238627C3B9BF76
:10F0E000EF320F930111AA892E84EFD0EF9C2A8969
:10F0F0009774FF1F938484BE6399090A9C5C4147FF
:10F1000093F707036393E70A1777FF1F0347F7BFD8
:10F11000894763ECE70883A7040B23170100231832
:10F12000010003D7C7013ECA3C002314E1007D570C
:10F130002315E10003D7C4023ECC23190100231696
:10F14000E10002CEEF80CFBD231EA100EFC06FCD46
:10F150008357C101230FA100914613D78700A2074F
:10F16000D98F2312F1009777FF1F83D7C7BA13D720
:10F170008700A207D98F2313F10017D700001307C8
:10F1800067F48147500095454808EF70602705886F
:10F190009317240003C484036D985D8C9777FF1F39
:10F1A000238A87B605616F30EF89EF70B0781775E5
:10F1B000FF1F1305A5B6EF80002083A7040B9775EA
:10F1C000FF1F83D565B403D5C701EF10E0279777FC
:10F1D000FF1F83C727B493F60702014789E6177715
:10F1E000FF1F035767B29776FF1F2397E6B2177783
:10F1F000FF1F130767AD184309CBC18B99C789451A
:10F200001775FF1F035545B002979777FF1F23AD72
:10F2100007AE9777FF1F238807AE9777FF1F23A5B9
:10F2200007B29777FF1F23A307B29777FF1F23A18A
:10F2300007B283D7840393F7270C93E71700177758
:10F24000FF1F2319F7AC83572903A18B99C3EF70D4
:10F25000E03F11C49777FF1F23A407AAA1B78D47EA
:10F260001777FF1F232EF7A8EF902FA59305803E59
:10F27000B305B5021775FF1F130545AAEF802012CD
:10F2800015B79777FF1F938767A5D85325C791C9EF
:10F290009777FF1F238907A69777FF1F23A807AA41
:10F2A0008280EF229FF883C7F70241112EC685079F
:10F2B0001777FF1FA30BF7A49777FF1F239FA7A420
:10F2C0009D471777FF1F232DF7A2EF900F9E2A84EB
:10F2D000EF90AF9DB24501E5EF902F9DAA85B30554
:10F2E000B4401775FF1F130565A3EF80400B410164
:10F2F0006F20FFF582809777FF1F9387279ED85353
:10F3000031C7EF229FF203C7F70205079776FF1F69
:10F31000A38DE69E11CD8C5F0D47014589818589BE
:10F320009776FF1F23AEE69CEFF09FDB6F203FF246
:10F3300085479305C0441775FF1F1305259E177752
:10F34000FF1F232FF79AEF808005CDB78280EF2231
:10F35000DFED1777FF1F0347079B8547631EF70005
:10F360009777FF1F9387879783C7870393C7870084
:10F370001777FF1F2300F79A1775FF1F1305059ACC
:10F38000EF806003EF807FEF99471777FF1F2329F6
:10F39000F7969777FF1FA38A07969777FF1F238417
:10F3A0000796EF90AF8F930740063305F5029777E6
:10F3B000FF1F23ADA7946F209FE99777FF1F83C797
:10F3C0006795C18B99C7EF225FE6EFF0FFAD6F2025
:10F3D0001FE8695582809777FF1F93872790DC533A
:10F3E00081CBEF229FE48545EFF09FCF6F203FE672
:10F3F00082801777FF1F1307678E01468146BA8503
:10F400002148631E06019DCA2390A60083C7850379
:10F4100093E717001777FF1F230EF78E05A083577A
:10F42000C705631DF502F8598547B397C70093C711
:10F43000F7FFF98F1777FF1F232CF7909C5D9183BF
:10F44000858B85C79777FF1F83C7E78B99EFEF22DF
:10F45000DFDD1D45EFF0FFB06F207FDF81E699E330
:10F460009306C7050506090769BF8280EF227FD989
:10F470008605AA84B309B500977AFF1F938ACA8CC0
:10F48000054B977BFF1F938B6B8C214C639434034C
:10F490009777FF1F938787849C5F9183858B89CBA8
:10F4A0009777FF1F83C7278681E72145EFF07FAB62
:10F4B0006F20BFD803DA0400630B0A041779FF1F1B
:10F4C0001309C9810144CA8C8357C905639D470349
:10F4D000A2855685EFF0BF9C11E5A2855E85EFF011
:10F4E0001F9C05C903A74C07B3178B00D98F17774B
:10F4F000FF1F232FF78483C78C0393E71700177729
:10F50000FF1F2309F78005040909E31F84FB890411
:10F51000B5BF231E0904C5BF1767FF1F0347A77E9A
:10F520008547631AF700EF225FD0EFF05FE2EFF05C
:10F53000BF976F20DFD18280814785451306000287
:10F5400093861700B397F500E98F13F7F60F89E755
:10F55000B687E397C6FE01473A858280FD47854519
:10F560007D56B396F50013871700E98E1377F70FD2
:10F5700089E6FD17E397C7FE01473A85828089E94E
:10F5800001473A85828001473A8541016F203FCC8F
:10F59000EF22BFC941112AC62E852EC4EFF0DFF934
:10F5A000A2457D158547B397A700E39EF5FC32463B
:10F5B0009377360099C3719A11069767FF1F938757
:10F5C000A77194433E871768FF1F1308287089EAC4
:10F5D000832708009107F19B9766FF1F23AEF66E05
:10F5E000032588001843B307A700B3F7B702B38712
:10F5F000F540FD15FD8D83274800AA95B306B6009A
:10F60000E3F3F6F8E371D5F82E979767FF1F23A36E
:10F61000D76C3DDB3A858145EF203FC42A87ADB7E3
:10F6200018419767FF1F9387676A23A4070098C351
:10F630005841D8C39767FF1F23A0076A8280EF2233
:10F640003FBDAA8401441769FF1F13092969930963
:10F65000400EEF807FD56345A40001456F209FBE1B
:10F66000330534038327090B3E958357C501E38790
:10F6700097FE0504F9BFEF22DFB89769FF1F938952
:10F68000E9653E84BA848347060003A70900411157
:10F690009D83058B3D8F83C74401AE8A2A89F99BE0
:10F6A000D98F238AF4001C44B685231204001CC0A1
:10F6B0002285328A36C6EF90DF8FB246D2853686F3
:10F6C000EF90900BDC4883A509000840858B568697
:10F6D0009D8DEFD03FCC61E918407D5583475700A1
:10F6E00003476700A207D98FC207C1872394F4009C
:10F6F0006358F00A83C7440193F70703B5CBD0489A
:10F700009377160003A609001D8E9777FF1F938736
:10F71000A7939C43ADEB814641A003A70B00931731
:10F720002A00BA97184094438347570083456700DF
:10F7300033F65601A207CD8F6311F60283473700D7
:10F740000346470003472700A207D18F4207D98FFE
:10F75000BD82B3F76701638AF604050AEF80DFC351
:10F76000420593170A014181C183E3E8A7FA41BF2B
:10F77000A16A370B0200014A976BFF1F938BCB6383
:10F78000FD1A7D1BE1BF83C74401130700038546B3
:10F7900093F70703E391E7F8A2854A85EFD0FFCFFF
:10F7A00041016F209FA96155E5BF7955D5BFEF2273
:10F7B0003FA69764FF1F9384A43A9C40D9EF9767B4
:10F7C000FF1F938727509C436399070CEF80DFBE90
:10F7D000930780023305F5028945EFF05FDA41C9EE
:10F7E0009767FF1F23A2A75AEF801FBC9307400E05
:10F7F0003305F5029145EFF09FD835C99767FF1F94
:10F8000023A6A758EF805FB201CDEF80FFB19145ED
:10F810000E05EFF0DFD621CD9767FF1F23AAA7566D
:10F82000EF801FCB11CDEF80BFCAD9473305F5025A
:10F830008945EFF0DFD405CD9767FF1F23A4A754B8
:10F84000EF809FB591450A05EFF07FD30DC1976713
:10F85000FF1F23A3A756014521A8EF803FC29307AE
:10F8600080063305F5029145EFF07FD101E565553E
:10F870006F205F9D9767FF1F23A2A7480144130ACB
:10F8800080061769FF1F13096945B14AEF801FBF42
:10F890006364A4029C40E38407F2EF803FBE9307B9
:10F8A000A0043305F5028945EFF07FCD69D1976754
:10F8B000FF1F23A7A75019BFEF805FBB894506052F
:10F8C000EFF0FFCB4DD5B3094403032709024E9750
:10F8D00008CBEF80BFB8330555039145EFF03FCA21
:10F8E00059D58327090205041374F40FCE9788DBDA
:10F8F00071BF9767FF1F9387673E8847058982809E
:10F90000C167FD176319F5009767FF1F9387073DD0
:10F9100003A5070B8280EF225F91EFF05FD26F208B
:10F920001F93814709C58347E501B337F000176787
:10F93000FF1F1307A73A18470983058B19C393E7DD
:10F9400027003E858280EF225F8E2A84EFF07FFDC4
:10F950008347E401AA851305940899E3130504037A
:10F960009766FF1F93868637944213061502130786
:10F97000840213059504EFD0CFC06F205F8DEF2276
:10F980003F899764FF1F9384643598442A892E84A5
:10F990000983058B9C4019C76314F5006380050E2D
:10F9A000014401A2E3FEA7FE1387A702E36AA7FEB4
:10F9B000850763FCA70883A9440BEF80FF96131605
:10F9C000350081454E85EF205F899767FF1F23A78C
:10F9D00027319767FF1F23A5073049CC9C4493E745
:10F9E00047001767FF1F232FF72E9767FF1F2383FB
:10F9F0000736630F040C9767FF1F23A1272F0144CD
:10FA00000549EF807F926341A40AEF80FF9493053C
:10FA10000006B3C5A502B7F73600938707E8176558
:10FA2000FF1F13056533416901449309400E7D1999
:10FA3000B385F502EF70B016EF801F97634FA408EF
:10FA40000145EF3040700544A9A86398A7029DE5E1
:10FA500083A9440BEF805F8D1316350081454E85D9
:10FA6000EF20AFFF9767FF1F23AA27279767FF1F86
:10FA700023A807269C44ED9BADB785C51767FF1FDC
:10FA80000347472D9307F005E3FCE7F021F8EF600B
:10FA9000F03C6DD19C4493E707021767FF1F2323B7
:10FAA000F72422856F200FFA83A7440B1315340027
:10FAB0003E958357050081CB8347250099C7214692
:10FAC0008145EF208FF905042DBF23012501E5BFF6
:10FAD0009767FF1F23A607200DBF3305340383A7B5
:10FAE000040B3E958357C50163842701EFF0BFE502
:10FAF000050499B7EF226FF3EF801F861304000609
:10FB00003345A4029764FF1F9384441D83C7840771
:10FB10003E951375F50F9767FF1F238DA722930757
:10FB2000F00563E7A7020545EF30E061EF80DF8273
:10FB30003345A402B7F53600938505E8B305B50251
:10FB40001765FF1F13054521EF7070056F202FF01B
:10FB50009C4405458983858B81CBEF904F888840F5
:10FB60008145EFF0DFE1DDB7EF30E05DC5B7EF22B3
:10FB70002FEA130495082A8913069005A285130518
:10FB80000503EF90603F1306900581452285EF2025
:10FB9000CFEC4A85EF30C0548144176AFF1F130A27
:10FBA000EA13930A8002EF803F8163C4A4006F20B0
:10FBB0006FE9338454038327CA0A3E940357040031
:10FBC0008357C9016317F702834744009DC3930914
:10FBD00064014546CE8513055400EF90E039454653
:10FBE00081454E85EF206FE7228523020400EF3028
:10FBF000005785044DBFEF224FE39767FF1F9387A0
:10FC000027F69C432A8491C70DC50355C501EFE033
:10FC10000FC29767FF1F938727439C4389CBEFB0A1
:10FC2000DFD085476315F5002285EF50C05D6F205A
:10FC30000FE241657D15E1BFEF222FDF1764FF1F43
:10FC40001304C4094440938714001767FF1F232936
:10FC5000F708EF30605E1C448983858B9DE7584030
:10FC6000B7E7B0009387075063F1E7020145EFF073
:10FC70001F9D01CD0545EF809FF608408545050590
:10FC8000EFF0FFCF0145EFF01FF726856F202FDC47
:10FC9000EF220FD8A1642A8901449769FF1F938935
:10FCA000A911FD14338AA500EF800FEF6344A4006F
:10FCB0006F204FD903A7090093172400BA979843E0
:10FCC000658F42074183634C2701635A47012380B4
:10FCD0000700A380070023810700A3810700050414
:10FCE000E1B7EF228FD183594500C547411163F534
:10FCF00037310441C1E533853401834785FF03472C
:10FD000095FF0348B5FFA207D98F0347A5FFC20798
:10FD1000220733670701D98F0347C5FF0348D5FF83
:10FD20002207336707010348E5FF0345F5FF420754
:10FD300022083365A800498FB98F1767FF1F130783
:10FD400067051768FF1F1308E8063A858328070030
:10FD50006384172B1107E31B07FF1767FF1F1307A8
:10FD6000670518431318270042951CC10507A147D2
:10FD70003367F7029767FF1F23AEE70293F735005B
:10FD80001397470083474601C16B368993F7F7FC09
:10FD9000D98F32842E8A230AF600814A176CFF1FFE
:10FDA000130CCCF3FD1B976CFF1F938C6CDB176D52
:10FDB000FF1F130DED00EF802FDF63C7AA00E15492
:10FDC000268541016F202FC71308400EB3870A0311
:10FDD00003280C0BB30DF800638E0D2083D7CD01E3
:10FDE000638A772183A70C00014B639707169767F7
:10FDF000FF1F938727ED9C436390071683C704007A
:10FE000003C70D0493F7F707631BF71ACA87228706
:10FE1000CE86268693859D0613851D04EFF0BF854B
:10FE2000631F051883D7CD01032709002320B401E0
:10FE30002312F400FD572313F4008347170093F6B1
:10FE4000F7078347D40093F707F8D58FA306F4008C
:10FE500093F7F707B337F000B307F0402307F40038
:10FE6000834717009D839396370083474401DD9BAA
:10FE7000D58F230AF4008347370083464700A20743
:10FE8000D58F83462700C206D58F1CC883477700CD
:10FE900003478700A207D98F2315F4000D47630499
:10FEA000EA00BD5491DF93870710C207C18313078F
:10FEB000B00FBD54E376F7F0EF800FC98144E31132
:10FEC00005F09766FF1F83C666EF938716001767D6
:10FED000FF1F2305F7EE1767FF1F1307E7ED231B2F
:10FEE000D40093972600144303578400E175BE960F
:10FEF000A1671386F7FFB377C70098426D8FD98F3C
:10FF00009CC21848F18F3E07D98F9CC2EF80CFC8A2
:10FF10009767FF1F83C787EA33F5A7029767FF1F1D
:10FF2000238EA7E871BD9307A004B308FB028327C3
:10FF30000D00BE9803D7080083D7CD01631DF700DD
:10FF400083C7040003C7880093F7F707630BF70024
:10FF500083C7FD019DEB050BEF804FD2E345ABFC62
:10FF600071BD9385980113859800CA872287CE8634
:10FF7000268646C6EFF02FF0B24879F98347440150
:10FF800093E74700230AF40071BD83C7040003C749
:10FF9000980293F7F707E310F7FCCA872287CE860B
:10FFA00026869385A8031385A802EFF0CFEC45F5CC
:10FFB0008347440193E72700230AF400C1B783C7AE
:10FFC000FD018DCB83C7040003C79D0993F7F70795
:10FFD0006312F702CA872287CE86268693852D0C68
:10FFE0001385AD09EFF02FE911E58347440193E74D
:10FFF000270049BF850AC1B3FD54D9B3EF226FA0D2
:020000040001F9
:10000000797183544500AA8B2E84B28AEF80CFBBCE
:10001000590563499504B7E4040003A90407EF8078
:10002000AFBA59054205418102992A8905CD2AC6F0
:1000300023180100EF804FB959052319A10061462B
:10004000814528089769FF1F938949C94ACAEF204B
:10005000CFA02302810203A48900058819E4BC54BF
:100060004A85829745616F204F9D74003008D68580
:100070005E85EFF01FC765F56800EF807FF1176AB6
:10008000FF1F130A6AFC83270A00AA84035B01018D
:1000900089CB89476397FA00835501025E85EF504B
:1000A000203003552102EF704FC819E50355210296
:1000B000EF708FD43334A000931764000344C1025F
:1000C0002C0868001374F4FB5D8C23068102EF603A
:1000D000B056E9576314F5028356E1029767FF1F94
:1000E000938787CD9C43139726006176BA979843F0
:1000F000718F98C39767FF1F2382D7CC8317210284
:100100006345F00085476396FA00B25793F7070CF2
:1001100095E7D247C2040347C102C180BE9426C6F8
:100120002318610113770703C147631DF700834755
:100130005102054793F7F7076390E704B7E7040018
:10014000BC5739BF92570544A18393F7F707E3776C
:10015000F4FE15C78347C1021307000293F7070394
:100160006397E700EFB06FFC8547E319F5FC834721
:10017000C10293F7070389CFEFB0AFCA21A8EFB050
:100180008FD7E30985FCEFB04FFAE31985FAD9B7A9
:10019000EFB0EFD8AA8501460545EF707FF82A84B5
:1001A00051DD8347C102414793F707036384E702A8
:1001B00032478347170093F707F8A300F700324749
:1001C000925783461700A18393F7F707FD17D58F42
:1001D000A300F70003560101B245130BC4005A8572
:1001E000EF80DFDFE24A130690058347C10283C434
:1001F000EA01918BB384C40213851404569595C308
:100200005444B3879A0083C7070403C706001377D3
:1002100007F82380E600584483460700D58F230063
:10022000F700B25703A609008146858B1D8EDA853B
:10023000EFD0EF9B15E9B25783A509004844138618
:100240009406858B56969D8DEFD0CF9411ED832724
:100250000A0099EFB257054791838D8B6387E704B6
:100260009DCF09476389E7042285EF80DFF8F9B560
:10027000EFB0AFEB85476309F5008347C102414703
:1002800093F70703E398E7FC835521025A85EF4073
:10029000907C69D183172102E35EF0FAF1B7EFB0E9
:1002A0008FC57D151335150061D101468145228525
:1002B000EF70FFEF55BFEFB04FE7E5B7EF12FFF676
:1002C0009764FF1F938404A32685EF809FEB2A8405
:1002D00019E16F10DFF71305C40005468145EFF003
:1002E000FFD12285EF803FF1C5B7EF121FF4411116
:1002F000AE842A8493079503130715019306F10032
:1003000005466C00268523060100EFD0CFBE1DED0B
:10031000A68541462285EF8030468347F10093054C
:10032000140226852308F400EFD06FC805E1976713
:10033000FF1F938767D19C4389EF1306940497C5E9
:100340000000938525D92685EFD08FD441016F1009
:100350001FF01306940297C50000938525D82685C3
:10036000EFD00FD379D9DDB7EF129FEA9767FF1F60
:10037000938787A48043AE84B289368AAA8AEF80A5
:10038000AF811316250081452285EF101FED976779
:10039000FF1F238507A29767FF1F9387279403A456
:1003A000070B13F714003E89230FE400CE8525C701
:1003B00013059408EFF07FF301C555556F109FE8C2
:1003C0008947A30FF4009767FF1F9387E7C79C43F4
:1003D00003278900858093B7170086072300F4025E
:1003E000231E54019767FF1F23AA478F85889377A1
:1003F000B7FF99C0936747001767FF1F2324F78E45
:100400002285930700061767FF1F2305F794EFF077
:100410008FD3014565B713050403EFF01FED45D5F4
:1004200069BFEF129FE0FD572310F500231105006F
:10043000231205002313050013062004814521051E
:10044000EF10BFE16F10BFE0EF129FDC4111AA84F3
:1004500001441769FF1F1309A9969309A0042EC62A
:10046000EF80CF81B2456344A40061550DA03305F0
:100470003403832709003E9583572500639CB7000A
:100480008357050063989700EFF0BFF901454101DC
:100490006F105FDB0504E1B7EF129FD79767FF1F6F
:1004A000938747829C434111AA842E84B2890359C1
:1004B0002500C1C39767FF1F83D70785639B270765
:1004C000EF700F862A8903D5240093051002B30527
:1004D000B40285472302F10093578900A302F1007B
:1004E00093578500A303F10083D744002304A100A0
:1004F000254613D787002305F10083D76400A304A2
:10050000E1004E8513D78700A305E1002306F10023
:100510001387950093879501A105B386B400A6972C
:100520004C00269723032101EFD0EF9C41016F106F
:100530007FD1EF60FFFE51BFEF129FCD4111AA8422
:1005400001441769FF1F1309A9879309A0043AC63C
:1005500036C432C22EC0EF707FF282451246A246E8
:1005600032476344A400615599A0B30734030325BF
:100570000900AA9703D8070003D5C4016310A80493
:1005800095E91DEE91CA03C6E401930510023306F6
:10059000B60225063E9690C2014511CB83C6E40102
:1005A00013061002B386C602E506B6971CC34101C6
:1005B0006F105FC903D52700E305B5FC050441BFF3
:1005C00083C5E40113051002B385A502BE9583C55A
:1005D00085002300B6007DB7EF129FC35C41411137
:1005E0002A8403DA2700C167FD17AE843289630CC1
:1005F000FA002685EF807F9A8D4763EDA7007D5531
:1006000041016F103FC42E85EF803F999D47E3E283
:10061000A7FEF5B75C40268583D54700EF809F9005
:10062000835584002685EF80FF8F8D452685EF80DA
:100630003F8EAA89EFF04FE0935705012380F90020
:1006400093578500A380F9002381A9005840C16712
:10065000FD178345A7006314FA0093E50508268576
:10066000EF801F8F9757FF1F9387C7659C430840F4
:10067000D9CF8347B400858BD9CB780034001306DB
:1006800071008145EFF05FEB1DC98347B40018404E
:1006900093069005F99BA305F4008347E701B38710
:1006A000D702B306F70083C60604A303D1009386DE
:1006B000170493879706BA96BA9736C43EC617545E
:1006C000FF1F1304A4611C440C4026858983858B7D
:1006D0009D8D834771009E05DD8D93F5F50FEF80AD
:1006E0003F871C44104022458983858BCA861D8E16
:1006F000A685EFC0DFCFE31505F01C440C40324661
:1007000089838840858B9D8DEFC0DFC8D5BD834729
:10071000B40013079005F99BA305F4008347E50196
:10072000B387E7023307F50003470704A303E1009B
:1007300013871704938797062A973E953AC42AC6CB
:10074000BDBFEF12FFAC032A45009307F00FAA8448
:100750000347AA00AE89328436896316F700EFB0EA
:100760006FAB2305AA00938AC9000146D68526856A
:10077000EFF09FE62A8A21E51767FF1F1307C78C52
:100780001843DC4039C383C6A7000547638FE602E0
:1007900083D547005685EF40102C05C9DC40839770
:1007A00047006354F00201CC1C4089C74A8681454A
:1007B000014582975C4081C7CA85014582974E8575
:1007C000EF807FA352856F10FFA7DC4003D5470061
:1007D000EF60BFD501E9DC4003D54700EF60DFE102
:1007E00081471DCD19C41C4089C74A8681450145F2
:1007F00082974E85EF807F9FAA851755FF1F1305AF
:10080000654FEF80DF9511C45C4081C7CA85014503
:1008100082971755FF1F1305254DEF60F03685476A
:10082000D84085460346A700E30BD6F803174700D8
:100830006353E000C9F74A86A2854E85EF703F9763
:10084000BDBFEF12FF9CAA8401441759FF1F130973
:1008500029579309A004130A9508EF703FC2634417
:10086000A400014535A033053403832709003E95D4
:100870008357250099E30504CDB70357050083D7B7
:10088000C401E31AF7FE52868545EFF0FFC065D537
:100890006F105F9BEF12DF97AA8401441759FF1F67
:1008A000130909529309A004EF705FBD6344A400CB
:1008B0006F105F9933053403832709003E958357F2
:1008C000250081CF83570500639997009305950212
:1008D000130610022105EF80206A0504F1B7EF121C
:1008E000DF940347E5012A848347F5016307B700D6
:1008F00089E781452E856F109F95230FB40005472A
:1009000081C9E398E7FE8947A30FF4008545DDB769
:10091000638BE7020947E39FE7FC2285EFF02FA5F1
:100920009757FF1F9387073A9C4399E79757FF1FF5
:10093000938707239C4389C70355C401EFF09FF5B4
:10094000A30F0400E1B755D6C9BFEF127F8CEFA00B
:10095000FFEE85476312F508EF80EFCC1754FF1FB9
:100960001304846E1C4081CBEFA03FFC89476304D5
:10097000F5001C4082979757FF1F9387A7349C432D
:10098000B9CF82979757FF1F9387871D9C4391C3C9
:1009900082971754FF1F130464348327040B83D4F6
:1009A000C701EF60FFB78327040BAA85144003C675
:1009B000E7011C448983858B99C31366260026852D
:1009C0004169EF40C03D8144D9497D19EF705FB066
:1009D00063CAA4006F101F87EF800FCA41B7EF7082
:1009E0005F884DB7B38734030327840ABA9703D5CA
:1009F00027006308250103C6470183D50700EF40A0
:100A0000A03B8504E1B7EF12BF8001449754FF1F5C
:100A10009384C42C1309400EFD59EF70FF98634F67
:100A2000A40401449754FF1F9384442B13098002AC
:100A3000FD59EF707F98634CA40401449754FF1F45
:100A40009384C4295949FD59EF709FA8634AA404AF
:100A500097F5FFFF9385450A1755FF1F1305C52F0F
:100A6000EF60D00797050000938585851755FF1F18
:100A700013058527EF6050056F10CFFC3307240363
:100A800083A7040B0504BA97239E370179B7330770
:100A9000240383A7C40A0504BA972390370151BFE2
:100AA0003307240383A7840A0504BA9723913701E7
:100AB00061BFD4410387350085473356F50263771C
:100AC000E600A54899E7238006008280B387E70205
:100AD000EDB73358F502038735003375F502B3D708
:100AE000E7021307000363DA080103C605001307D2
:100AF0007003118A19E21307700585064297A38FC8
:100B0000E6FEC9B718451C416376F7005C41BA9709
:100B10002380B7001C4585071CC58280EF12EFF0CB
:100B20004111AA872E85B285368636C682976348DC
:100B30000500B246158D3335A0003305A0404101B4
:100B40006F10EFF0EF12CFEC056941112A8A2320D4
:100B5000060001448149975AFF1F938AEA28056BD2
:100B60007D1932C62EC4EF703F85AA84EF70DF83F3
:100B70002695A24532466346A4004E8541016F107A
:100B80006FEC03A70A0093171400BA9703D7070066
:100B90003377670101E71CC20504E1B703D70700FB
:100BA0009356D700858AE39946FF33772701E315EB
:100BB000B7FEBE89D5B7EF124FE701112EC6B2843A
:100BC0003689EFB02FEE2A84615501C8B24589E914
:100BD000232E040023200402014505616F102FE736
:100BE000A1463008CA852685EFF05FF37DF583576F
:100BF00081010357A101231EF4008357C101231073
:100C0000E4022311F4028357E101D207D1832312B6
:100C1000F4028357E1011397370163560700FD572C
:100C2000231FF4005DBF231F040045BFEF124FDEFA
:100C30001754FF1F1304840A8327040B03D7C7012B
:100C4000C167FD17630EF7109757FF1F9387074083
:100C50009C4381C70545EF406077C1690149930A0C
:100C6000400EFD19175BFF1F130B0B3EEF70CFF308
:100C7000634BA90E1757FF1F0347C70D9307F005D6
:100C800063E4E702EF704FED93050006B3C5A502DC
:100C9000B7F73600938707E81755FF1F1305C50BF5
:100CA000B385F502EF60A06F8145170500001305BD
:100CB0008520EF60DFF8EFB0EFDE01CD0357C5010F
:100CC00009CB0357E50111C78347050299C3EF60BC
:100CD000A06BEFB06FDE31C51757FF1F03474714F6
:100CE0009757FF1F9387C7130DCF03C71700230420
:100CF000E50003C72700A304E50003C73700230569
:100D0000E50003C74700A305E50003C75700230616
:100D1000E50003C7670083C77700A306E500230744
:100D2000F5001C4493E717001757FF1F232CF7FA11
:100D30005C4085E7EF708FEF0DC1EF702FEF4440FF
:100D40002A89EF70AFEE33F5A4025C40FD17CA9715
:100D5000898F1757FF1F2325F7F80145EF70DF9F95
:100D600001456F102FCEB30459038327040BBE94A3
:100D700083D7C40163883703138A0403D28552855D
:100D8000EFF0AFD605E183C7F40199CF93859408BE
:100D90002E85EFF08FD509C9130690058145528540
:100DA000EF10AFCB0509D9B583270B00268593B784
:100DB000170086072380F402EFE0FFB8E5B7854708
:100DC00063F8A7009307F5FFBE953305A040E98DB2
:100DD0002E8582809841C167BA9713D707016304B3
:100DE000A7009CC182804207998FE5BFEF12EFC335
:100DF00041112EC63284B684EFB00FCCE15701C941
:100E0000B24591E99757FF1F238C070081473E8524
:100E100041016F10CFC39D461756FF1F13065600A2
:100E2000A6852285EFF09FCFAA8775F105479756D3
:100E3000FF1F2387E6FEE1BFEF128FBD411191E94D
:100E40009757FF1F23AE07E80144228541016F1029
:100E50006FBFB68532858D467000EFF03FCC2A8497
:100E60006DF58347D1000347E1001759FF1F1309B0
:100E7000E9E6A2074207D98F0347C100D98F175768
:100E8000FF1F232FF7E4EF706FDA61D1EF700FDAF5
:100E900083244900AA89EF706FD933F5A402832710
:100EA0004900FD17CE97898F1757FF1F232AF7E2B6
:100EB00069BFEF128FB71C45AA8491CFD84B01CFE1
:100EC00083D7470089CBEF601F92AA8509C5884464
:100ED0006105EF60C04C9757FF1F9387A7DE9C43C7
:100EE000014489EF6F10AFB69C4813171400BA97EE
:100EF00003D5070019C1EFE0CFCF0504EF70CFC7CE
:100F0000E344A4FEC5B7EF124FB2011185E9EF60CB
:100F10005FDA01449757FF1F23AE07E49757FF1F7F
:100F200023AC07E49757FF1F23AA07E49757FF1F37
:100F300023A807E4228505616F106FB1B68732855B
:100F4000C9467000BE85EFF07FBD2A8465F5414635
:100F50009305E1001755FF1F1305C5E1EF80C001A0
:100F60000355C100EF608FD7F1B78DE19757FF1F91
:100F700023A607D69757FF1F938747D69C4701455F
:100F8000ED9B1757FF1F232FF7D48280EF12EFA995
:100F90004111B685328595463000EFF03FB815ED2A
:100FA000A2471757FF1F232BF7D29757FF1F93878F
:100FB000E7D29447B24713F7B6FF13F6170019C2EA
:100FC00013E74600858393F7F7079756FF1F23AB78
:100FD000E6D01757FF1F230FF7D641016F102FA739
:100FE000EF120FA303841500DC412A89AE84850724
:100FF0000387F7FF19C36340800C8387240091C7E0
:10100000635580007D14620461849C40370700FFB3
:101010000907F98F3707001009076392E70A63553C
:10102000800079146204618483C70400858B95E392
:101030009379F40F4E8A93178A01E187634AF00887
:10104000A2876353040081473384F9407D1462040E
:1010500061848385240081C54A85EFF0BFAA9C4046
:10106000370700FF0907F98F370700100907639A50
:10107000E706930500034A85EFF0DFA883C7040065
:1010800093058005918B99E3930580074A85EFF0DE
:101090007FA783C70400858B81CB1374F40F93174C
:1010A0008401E1876347F004C04005048305F4FF31
:1010B000A1E96F102F997D14620461840DBF370779
:1010C00000080907E392E7F6E35080F67D1499BF24
:1010D000930500024A857D1AEFF0DFA2137AFA0F1A
:1010E00099BF370700080907E395E7FA930500035E
:1010F00071BF930500034A85EFF0DFA07D1471BF37
:101100004A85EFF03FA055B7EF122F92EF70CFAAAC
:101110002A84EF706FA9229589450605EFE02FC656
:10112000E55711C59757FF1F23A0A7CC81473E85E0
:101130006F10EF91930700026306F5005D151335FC
:101140005500828005458280EF128F8C4111AA895B
:101150002A89130419008304F4FF32C62EC426859D
:10116000EFF05FFDA245324659E19307D00263924A
:10117000F408830404000548130429009377F6FE5D
:10118000C9E793070003639FF40E83070400130766
:10119000800593F7F7FD6399E70683041400414641
:1011A0000904B70600806314080093C6F6FFB3FE77
:1011B000C6028147254F654EFD5F33D3C6021387B4
:1011C00004FD6368EF06BA8463D5C408630DF501B6
:1011D0007D55636AF3006394670063C69E0005450E
:1011E000B307F602A69705048304F4FFC9BF22895A
:1011F0008DB79307B0020148E392F4F8830404002A
:101200002A88130429009DBF01CA8947E31BF6F809
:1012100093070003E397F4F88307040013072004FF
:1012200093F7F7FD639BE704830414000946090460
:101230008DBF13E704021307F7F9636CEE00938880
:10124000F4FB1307700363741E0113077005998C78
:10125000A5BF7D576300E50263040800B307F040B3
:1012600091C519C19309F4FF23A035013E854101C1
:101270006F005FFDB687FDF5D5BF9304000315F23F
:10128000214605B719FE294629BFEF027FF8011153
:1012900061540DC53284AE89414681453689EFF0EF
:1012A000BFEA93140501C180639E09002685EF30D3
:1012B000102B014401C58145EF20501622850561A0
:1012C0006F005FF82285CD467000CA85EFF01F855C
:1012D0002A846DF52685EF30902809E90356C10070
:1012E0008345E1012685EF20500B01C94146930556
:1012F000E1001105EF705048D1B75D54C1B7EF025E
:101300003FF10111E15401CDB284AE8941468145DE
:101310003689EFF07FE32A846397090081442685AC
:1013200005616F003FF22685D1467000CA85EFF057
:10133000EFFEAA846DF58357C100EDD3EF700F8ED9
:101340004205931704014181C18363F9A702EFB0FD
:101350008FB64204E14741803304F40241460C0851
:101360002A9413054400EF7030418357E1002311A4
:10137000F4008357C1002310F40055B7E55445B776
:10138000EF021FE97971E15415C53284AE894146F7
:101390008145B684EFF05FDB13190501135909018C
:1013A000639E09004A85EF401065814401C581456F
:1013B000EFB02FB1268545616F00DFE8A685930663
:1013C000300270002285EFF06FF5AA8465F54A853A
:1013D000EF4070622A8411E54A85EFB04F8C2A8471
:1013E00031C58357C10023112401930964002310E0
:1013F000F4008347E1009305F10041462302F40025
:101400004E85EF7070371309740141469305F10161
:101410004A85EF707036930554004E85EFC04FBF7C
:10142000930564014A85EFC0AFBE69B7DD5459B773
:10143000EF021FDE797111E5E154268545616F00E9
:101440007FE0B284AE89414681453689EFF0DFCF37
:10145000131A0501135A0A015285EFE06FCA2A8454
:101460006398090071D98145EFB02FB48144F1B779
:101470002685930610027000CA85EFF02FEAAA8431
:101480004DFD31C8B2479305D1004146858B230FEE
:10149000F400B24713050403858393F7F707A30FFE
:1014A000F400EF70702D41469305D10113059408A7
:1014B000EF70902C59B73304690383A70A0B3E944D
:1014C0008357C401638337030509EF60FFEDE344ED
:1014D000A9FEDD549DB7C1690149974AFF1F938A50
:1014E000EA7F130B400EFD19CDB7231E440159BFEF
:1014F00049CDEF02FFD14111B289AE844146814509
:10150000368AEFF07FC4931A050193DA0A01014984
:10151000174BFF1F130B8B7CEF601FE1634AA90081
:101520000145ADCC81441749FF1F1309297B81A8D0
:1015300083274B0B131439003E94835704006388B0
:1015400057050509D1BF8327490B139434003E94F6
:101550008357040085E72310540191467000D2851B
:101560004E85EFF0AFDB1DE9B24713978700E183AB
:101570002183858B58C02301F4000DA08504EF6002
:10158000BFDAE3C2A4FC5D5511A861558280F1F475
:10159000214681452285EF005FCC014541016F0066
:1015A0007FCA1971D2C4130AC10686CEA2CCA6CABC
:1015B000CAC8CEC6D6C2B6D6BAD8BEDAC2DCC6DE75
:1015C00052C463810524FD151C102ACC2ECA02CEFC
:1015D0003EC89304B0021549A949830506001304C7
:1015E00016009DE1F2465247E24763FBE620B697BC
:1015F000238007007245F6406644D6444649B64902
:10160000264A964A09618280930750026386F50054
:101610004808EFF02FCFF5A88357C100230701003A
:10162000014593F7C70F2316F10081450148014793
:10163000014681469308D00213030003130E3002C3
:1016400005048307F4FF99C7638C970463C3F4040C
:10165000638BC70501CA0346C100858A799AD18E7A
:101660002306D100630908008346C100098BF59A5F
:10167000558F2306E10019C12307B100138707FD29
:101680001377F70FA54663E2E6068146A54529458F
:1016900035A0E38717FBE39F67FA0546FD564DB774
:1016A0000545854571BF05487D5759BFB386A602DC
:1016B00005048307F4FFBA96E206E18613F7F70FF5
:1016C000130607FD1376F60F63E5C500138707FDC4
:1016D000F1BF1306F7F91376F60F636EC90213878D
:1016E00097FAE30537FDA306D1001307900663853B
:1016F000E704634BF706130780056384E70A634535
:10170000F702E38107EE1307500293055002E381CD
:10171000E7F02286D9B51307F7FB1377F70FE364D9
:10172000E9FC138797FC75BF130730066386E70A49
:1017300013074006E39FE7FC03250A00A947A30718
:10174000F100930A4A00635805009307D00233055D
:10175000A0402307F1006C00EFF0AFB56C00480823
:10176000EFF01F88568A75B713073007638EE706B8
:101770006341F7021307F006638EE70413070007BF
:10178000E399E7F80347C100136727002306E10048
:1017900009A813075007638BE70213078007E39A32
:1017A000E7F6938787FA414793B71700A307E1004D
:1017B000139727008347C100ED9BD98F2306F100C3
:1017C000930A4A006C0003250A0079B7A947A307CA
:1017D000F100FDB7A147E5BF83050A004808930A59
:1017E0004A00EFF02FB2BDBF83270A006C00480803
:1017F0003EC8EFF0EFFE1C10930A4A003EC89DB7AA
:10180000BA97FDB30145C5BBEF023FA22A883685D2
:1018100083464800BA8703475800A206D98E32870C
:1018200017B600001306C68D89E517B6000013062B
:10183000E68DBE85EFF0FFD66F007FA19747FF1FB3
:101840009387875D9C4381CFEF023F9ED843B2864A
:101850002E861847AA853E8502976F005F9F6155C7
:101860008280EF029F9C8357050039712A84231ED2
:10187000F100834745009305650041461305F101DA
:10188000230FF100EF70406F93057401414613057B
:10189000F102EF70606E8356240017B60000130645
:1018A000268FE5450A85EFF0DFCF6C08130630027E
:1018B0000A85EFF0BFF821616F007F99EF02FF9674
:1018C00039712A849305050341461305D101EF7050
:1018D000A06A9305940841461305D102EF70C069D0
:1018E0008347E4010347F4018356C401858B06074F
:1018F000D98F17B600001306668AE5450A85230EC0
:10190000F100EFF01FCA6C08130610020A85EFF011
:10191000FFF221616F00BF93EF029F8F3704000138
:10192000B70400FF0111814A1749FF1F1309093B42
:101930007D149389F4FF17BA0000130AAA8AEF6096
:10194000BF9E63C5AA0005616F00DF8F8327490B27
:1019500013973A003E978347370095CF5C43A30126
:1019600007005286B3F687008247E5454800E58FB9
:10197000D58F3EC083462700B3F73701858AE2063C
:10198000D58F835607003EC0EFF0BFC111468A8550
:101990004800EFF0BFEA850A5DB7EF021F890146F4
:1019A0008145EFF0BFE96F009F8A83576500638E22
:1019B000071A1D71A2CCA6CACAC886CECEC6D2C48A
:1019C000D6C2DAC05EDE801013F717003289AA840F
:1019D00031CBF99B2313F500EF601F9906053D05F8
:1019E00041990A8BC16A3301A1408A8B8149014A1E
:1019F000FD1AEF607F97634CAA0C7947930604FBAE
:101A000017A600001306067DCA852685EFF0DFDFE6
:101A1000638F090C13961900DE85130504FBEFF0A4
:101A2000FFE15A8183D7640013F7270021CBF59B90
:101A30002393F400EF605F9406053D0541998A8A7F
:101A40003301A1400A8B8149014AEF60FF9263454F
:101A5000AA0A6547930604FB17A60000130606783A
:101A6000CA852685EFF05FDA6387090A13961900A5
:101A7000DA85130504FBEFF07FDC568183D7640021
:101A800013F7470005CBED9B2393F40065479306BE
:101A900004FB17A600001306A674CA852685EFF07E
:101AA000BFD69C4481C703D747003DEB130504FB19
:101AB000EFF0BFEE130104FAF6406644D6444649FF
:101AC000B649264A964A064BF25B25618280DC4481
:101AD00013171A00BA9703D70700630857019397A3
:101AE0001900DE972390E7008509050A19B7130549
:101AF00004FBEFF09FEA35B79C4813171A00BA971A
:101B000003D7070019C793971900DA972390E700C6
:101B10008509050A1DBF130504FBEFF01FE8B1BFDF
:101B20002314E4FA03D767008326C4FA2146520738
:101B300051832315E4FA370700F0758F9447930516
:101B400084FA130504FB92069182558F2326E4FA4A
:101B500083C7770013F707018347F4FABD9BD98F3A
:101B6000A307F4FAEFF09FCDB1B78280EF026FE9DF
:101B70001744FF1F130484160444797193F7F4FB90
:101B80001747FF1F2320F71693F70404A1C7858882
:101B9000A1E097A900009389E964EF60EFF863DBA7
:101BA000A4028327440B139934003E9983560900FD
:101BB00091CE4E86E5454808EFF0BF9E4808EFF00D
:101BC000DFDD214681454A85EF002FE98504F1B725
:101BD000EFF09FD41C4413F7F7F79746FF1F23A39A
:101BE000E61093F707086397071E1C4413F7F7EFF7
:101BF0009746FF1F23A8E60E13F707106318071E6A
:101C000018449377F7DF9746FF1F23ADF60C9376C2
:101C1000072095C6058B630A072018408983858BAA
:101C20003ACA0347840715464C080607D98F17A5FB
:101C300000001305E557230CF100EFF03FC01C44F2
:101C400013F7F7BF9746FF1F23AEE60893F7074049
:101C50008DC3835744000D464C08231AF100835767
:101C6000640017A500001305E554230BF100EFF005
:101C7000FFBC1844FD749387F47FF98F9746FF1FCC
:101C800023A2F6069317470163DF0700EFA08FE159
:101C900019C98356C5016391061A17A500001305DB
:101CA000E551EFF09FCF1C447D777D177D8F9746E0
:101CB000FF1F23A9E60213973701635A0702858B9A
:101CC0006388071CEFA04FDF1DC118458347E5005F
:101CD0001D463ACA0357C5004C0817A50000130556
:101CE000654E231CE100230DF100EFF03FB51844D1
:101CF000F977FD17F98F9746FF1F23A5F6FE931777
:101D0000270163D90700814517050000130525CA7F
:101D1000EF50FFF21844E177FD17F98F9746FF1F48
:101D200023A2F6FC9317070163D30702EFA0BF9825
:101D30002A84814417A9000013094949EF600FEE76
:101D4000939704014205C183418163EAA714456169
:101D50006F00AFCE83A70A0093141900BE9483D7F7
:101D6000040033F767011DCF1396170133F777018E
:101D7000B3F637016352060417A600001306464166
:101D800009E717A6000013066641E5454808EFF08D
:101D90005F814808EFF07FC083D70400B3F74701A5
:101DA0002390F4000509EF602FE1AA84EF60CFDFF4
:101DB0002695E341A9FA15BD368519C7EF40A04322
:101DC00061DDEFF01FAAC9BFEFD09FB371D5EFF06F
:101DD000FFAED9B785697D7A0149974AFF1F938A7B
:101DE000AA00056B896BFD197D1A75BF858B9DC790
:101DF000EF500FF3231AA10041469745FF1F93852B
:101E000065F713056101EF70201749464C0817A5C7
:101E1000000013056539EFF07FA2DDB317A50000C0
:101E200013058538EFF07FB7E1BB17A50000130558
:101E30002538EFF09FB621B50357E501C177850737
:101E40003E978357A101FD14133717003207E58F22
:101E5000D98F231DF100231AD100835605020357A1
:101E600025022146231BD100231CE1000357450214
:101E70008566FD16758FFD76F58FD98F4C0817A5F1
:101E800000001305A533231DF100EFF03F9B21BD9A
:101E900017A5000013050533EFF03FB089BD5C487E
:101EA00013F7E7FF58C8858B89CFA6864A86C945B0
:101EB0000A85EFF00FEF8357040099E70A85EFF0EA
:101EC000DFAD850461049DBD231AF1008357240012
:101ED0009305440041462808231BF100EF70C00918
:101EE00051464C080A85EFF07F95E1BFEF02EFB352
:101EF00085473395A7009747FF1F938727DE9C47A9
:101F0000411181455D8D9747FF1F23ADA7DC937776
:101F1000057085E393576500858BA1CBC1679387D7
:101F200007887D8D05EDEF606FD19305803EB30589
:101F3000B5021745FF1F130565EB2EC6EF50A03BFA
:101F4000B24519C16349B50085C51745FF1F130583
:101F5000E5E9EF50C04441016F006FAFEF600FCE75
:101F60002A84EF60AFCEE360A4FCEF602FCE75BF94
:101F70000145EFF0BFBFC5B7EF022FAB7971AA865D
:101F800001441749FF1F130969D536C6EF60CFB961
:101F9000B246635CA4028327490B93143400BE94B9
:101FA00083D704006396D70285C617A600001306E0
:101FB0006623E5454808EFF0CFDE4808EFF0FF9DC7
:101FC000214681452685EF004FA945616F002FA866
:101FD000050465BF19C223200600814701C5930689
:101FE000D00389E53E858280850505058387050048
:101FF0000307050099CF6394E700E397D7FE814775
:10200000D5B79306D0038547E30ED7FC9337170067
:10201000D1BF9307F002E316F7FE854761D60505A9
:1020200008C2C9B799C123A0050081470DC1130893
:10203000D0031306F0023307F5008306070081CAB8
:10204000638706016397C60099C1050798C13E855D
:1020500082808507CDB731C9EF02AF9A41112E8A30
:102060006C002A89368BB28A97A400009384440BB3
:10207000EFF05FFB2A8C0144A689B14B8840628651
:10208000CA85EF70E01701ED0E044E945C403245B6
:10209000DA865686D285829741016F000F9A050431
:1020A000A104E31D74FD6155C5BF7D55828099E58E
:1020B00061558280615505616F00CF98EF024F95A1
:1020C0002E8A2A8401118145B28452854146BA89FB
:1020D0003689EFF06F8793150501C1811376F50FEF
:1020E000A1812285EF507FB12A8469D552854C08A1
:1020F000EFF05FF3524A2A8BE30E0AFA2A8697A57D
:1021000000009385250D5285EF70800FAA8A0DED92
:102110007D5AEF606FA563C5AA0099E8014561BFCC
:102120005C4413971A00850ABA9723904701D5B7E4
:102130004C442EC6EF604FA3B245131615004E85D2
:102140000299E34DA0FC85BF5A8697A500009385B0
:10215000E5085285EF70C00A0DE1032A0401EF6023
:10216000AFA11316150081455285EF000F8FDDD406
:102170000C482EC6EF604FA0C1B75A8697A5000045
:10218000938505065285EF70A00741E11C44A5CF59
:1021900081ECD443370700E0758F9447D8C33707E5
:1021A000001F758F98C701BFA1463008CE854A85AC
:1021B000EFE0DF96E31105F01844835781017D7647
:1021C0002312F7008357A1019396470183576700B5
:1021D000D182F18FD58FF2467D767D16F182858A88
:1021E000B206F18FD58F2313F7008347E1018356A1
:1021F000C1012305F7008347B7002314D700FD8BE7
:10220000A305F7004DBD7D557DB55A8697A5000005
:10221000938585F05285EF60B07EE31D05E81C4C88
:10222000E38A07E89C43E38707E8CE864A86A685CB
:102230002285829749B5EFF25EFF3687B2862E86F9
:10224000AA850545EFF0BFE66F006F80EFF2FEFD57
:102250003687B2862E86AA850145EFF05FE56FF0DE
:102260001EFFEFF2FEFA411199C123A00500974726
:10227000FF1F938767B9804381441DC82E89AA89AF
:1022800031141DC40C4070004E85EFF0BFD419CD41
:1022900081E8A284630C0900B2472320F90039A029
:1022A0008C4008400146EFF0FFD265F5404869F8E0
:1022B000268541016FF01EF9184111CBEFF2FEF6B1
:1022C000AE873E85B285368602976FF05EF835554B
:1022D0008280EFF29EF58357C50013D70501C20532
:1022E000B387E7021841C1814849BA95BE95EFF01E
:1022F000BFFC6FF0DEF5584111CBEFF21EF3AE8755
:102300003E85B285368602976FF07EF43555828021
:10231000184509CBEFF27EF1AE873E85B285029774
:102320006FF0FEF2355582805C4599C7EFF2FEEF03
:102330002E8582976FF0BEF135558280EFF25EED0B
:1023400083290500035AC5002A844849AE84814583
:10235000EFF09FFD2A890DE193D50401B385450374
:102360000356C4004848CE95EFF09FFA2A8909E544
:1023700048488545EFF05FFB4A856FF0BEECEFF211
:102380003EE92A890441035BC500484979712E84DE
:102390008145B28A368AEFF03FF941E19359040151
:1023A000B3896903420441802694A2990344090138
:1023B000330480403374440111CC03254901A286C3
:1023C0005686CE85EFF03FF3AA8431E1330A8A4086
:1023D000A299A29A8144630C0A025286D685080803
:1023E00003244901EF605039834609011C08930515
:1023F000F00F338646413385470136C6EFF0FEE5E0
:10240000B2461008CE852285EFF0FFEEAA840325A0
:1024100049018545EFF05FF1268545616FF09EE249
:10242000EFF2BEE02E864C41A1462A84EFF03FF544
:10243000AA8403450401A145EFE07F985C40338501
:10244000A74048C026856FF09EE0814797A6000010
:10245000938606CA6393C70082803387F5000347DB
:1024600007008507398D1357450036970347070046
:102470001205398D1375F50F13574500369703472D
:1024800007001205398D1375F50FE9B7EFF2FED984
:102490002A84AA851D461305F00FEFF01FFB834722
:1024A00074003385A7403335A0006FF05EDAEFF299
:1024B000DED74111A1463000EFF0BFE109ED03572F
:1024C0008100C167FD1705456317F7002800EFF08D
:1024D000FFFB3335A00041016FF07ED7EFF25ED3F2
:1024E000AE848C414111A1462A8903440501EFF0D5
:1024F0005FDEAA8939E9A1452285EFE05F8C9C4027
:102500000357C9002A8AAA97939607019CC0C182E3
:10251000098F639CE602C16513D70701B385B740F5
:1025200011E78355E900FD15C205BE958CC0A14693
:102530000A864A85EFF0FFD9AA8901E90A85EFF0FA
:10254000FFF401C9832749009CC04E8541016FF00B
:102550007ECF0357C900835721008040330747418E
:1025600063DBE70033FA470363170A004177798C8E
:102570003E9480C0D9BF03450901A145417AEFE0EF
:102580001F84098CAA8A80C0337A4401417B63642A
:102590008A0081495DBFA1463000A2854A85EFF0DF
:1025A0005FD3AA895DF12800EFF05FEE11E9835750
:1025B000A1000357C100337A6A0180C0BA973E9ADE
:1025C00033045441E9B7EFF25EC62A84AA851D465A
:1025D0001305F00FEFF07FE7A303A4006FF03EC7F1
:1025E000EFF23EC22A84034505015D71A145EFE08B
:1025F0000FFD5C402A8B0355E4004179B3F72701B6
:102600006C003EC6EFE00FFD8355C400B247A14603
:102610003008BE95B385654122852EC8EFF07FCB8B
:10262000AA84634B05002808EFF05FE611C9B245A4
:102630002285EFF0BFD0AA84268561616FF0FEBFCE
:10264000C2470357A101417C338B6741B3F7270190
:10265000BA973EC810100C082285C24BEFF01FE855
:10266000AA8479F90810EFF07FE22DE95C403ECAB8
:1026700030104C0822855249EFF05FE6AA844DFDE8
:1026800003578102835701026316F7002810EFF009
:10269000FFDF09C55840D247E31CF7FC63902B05C8
:1026A0008357410285CF83572102B3FA8B0108106B
:1026B000BE9A1C442311F102EFF0FFF0834904019C
:1026C000035A4102B309304193F90902631B0A001E
:1026D0000C102285EFF0DFD4AA8439FDE31C7BF7D0
:1026E000B9B74E8963733A015289CA861018D685E4
:1026F0002285EFF01FBEAA8421F1630909000C4472
:10270000CA8610182285EFF09FC7AA8403450401EA
:10271000CA85EFE0CFEA1C443E9508C4E39E04F06E
:10272000330A2A41CA9A5DB7EFF29EAE411191E594
:10273000FD54268541016FF0FEB0C44983D72501C1
:102740004CC904C12316F50003C705012A842317C9
:10275000E50003C5150193160701130700022308BE
:10276000A400C182E366A7FCE1D7B3E4F402E9F078
:102770008547E3FFD7FAA145EFE06FE4AA89014A54
:1027800001498357C400931509012285BE95B3857D
:1027900035412EC2EFF0BFD119ED0355E4004C00D6
:1027A000050AEFE02FE39245420A2285135A0A01F7
:1027B000EFF0FFCF09E905098357E40042091359F7
:1027C0000901E360F9FC8357E40063944701D154A5
:1027D0008DB7639427039245A1463000B3853541F8
:1027E0002285EFF01FAF35E12800EFF03FCA11C599
:1027F0000355E4004C00EFE0EFDD9247C17A3387E8
:10280000374158C04177F98F1CC44C401C4463EEDB
:10281000F500A14630002285EFF0BFAB1DE5280092
:10282000EFF0DFC6032A44001DC15C400355E400FD
:102830004179B3F727014C003EC2EFE0AFD9924592
:102840002285EFF0DFC6635C0502AA84DDB5124580
:102850000359A100035BC10033F5AA002A9903457F
:102860000401DA85EFE0AFD54A9508C46314450149
:1028700063130B04330A3A412322440179B709C593
:102880008547A308F40075B54C402285EFF01FABD7
:102890004DFD48408357C40086093375A9003E9515
:1028A0003305354148C03375250108C42285EFF052
:1028B0003FD379D559BF4D5549BF83471501C9CF7E
:1028C000EFF23E942A840345050141112E8AA14569
:1028D000BA893689328BEFE08FCE8357C400060564
:1028E000898F7D5563E727075C4081443EC23000F5
:1028F0004C002285924AEFF07FBE21ED835B810080
:1029000063994B012800EFF07FB801E58504C2040C
:10291000C18058409247630BF702E3FA99FC835653
:10292000C10061559DC663E63403C175B3FABA00B0
:102930006373D900CA868355A1005A862285D6952D
:10294000EFF03F9919E50355C10021A06155E388D7
:102950004BFD41016FF07E8E49558280EFF2FE8C77
:102960000147EFF09FF56FF09E8EEFF21E8C3284E0
:10297000B2862E86835545000841EFF03FFE635333
:1029800085002A8422856FF09E8CEFF21E87834794
:1029900015013971C954BDC7034B05012EC62A84E0
:1029A000A1455A853689328AEFE06FC10D4733075A
:1029B000E5028357C400AA8DFD54998F63E427056F
:1029C0006304090063000A045C403ECA30084C08F6
:1029D0002285524DEFF09FB0AA8945ED83578101C2
:1029E00032476397E7002808EFF05FAA63060510F7
:1029F0005840D247E31CF7FC8144631B090019A02F
:102A0000814499E7268521616FF0FE82E35CA0FE98
:102A10005A85CA85EFE0AFBA014B11C5330BB5013A
:102A2000420B135B0B01014D7D5CC17B930C440099
:102A30008357E4006380A70D1C4444403307FB0028
:102A400063EBE40432472311F1020810FD57231011
:102A5000E102231221032303F102EFF0DFB6630941
:102A600009000C44CA8652862285EFF05F91AA893C
:102A700003450401CA85EFE08FB41C443E9508C4A9
:102A8000639909000C102285EFF09F99AA89CA84E6
:102A900035D9CE8485BF03450401A145EFE02FB2AF
:102AA000B387A4002311F1028357C400B3F4740167
:102AB00023108103BE94898C44C0081023120102A4
:102AC000EFF07FB00C102285EFF09F95AA8403559C
:102AD000E400E685EFE00FB05C40B3F777011CC47B
:102AE000E39204F22285EFF0BFAFAA84E31C05F065
:102AF000050D3DBFC15439B78357C101E30209F049
:102B0000E39827F1C177034C0401B377FD00035D1F
:102B1000A101330C8041137C0C023E9DD28ACA8CE9
:102B2000E28B63F38C01E68BDE861010EA8522854A
:102B3000EFF02FFAAA84E31B05EC5E860C10568595
:102B4000EF602041AA84E31505ECB38C7C415E9DC7
:102B5000DE9AE3970CFC7DB5EFF22EED814601463F
:102B6000EFF0BFE26FF0AEEE638C050EEFF26EE9B0
:102B70005D71054D19C213BD160003590502B68BD0
:102B8000328B05094209135909012E8A2A84CA8900
:102B9000216C930A8500E15C9304F9FFC204C180B3
:102BA000638F84059306A0045000A6855685EFF038
:102BB000FFDA6357050063139501A6892689E9BFEB
:102BC0009C083E95230A05FA4C005285EFF06EF3FF
:102BD00075F563040D08835704026395970893877E
:102BE000F4FF2310F402894613060402A1655685FA
:102BF000EFF0BFD96358050661616FF00EE401453F
